:020000040800F2
:200000002A18002405030008A9020008A9020008A9020008A9020008A9020008A902000838
:20002000A9020008A9020008A9020008A9020008A9020008A9020008A9020008A902000828
:20004000A9020008A9020008A9020008A9020008A9020008A9020008A9020008A902000808
:20006000A9020008A9020008A9020008A9020008A9020008A9020008A9020008A9020008E8
:20008000A9020008A9020008A9020008A9020008A9020008A9020008A9020008A9020008C8
:2000A000A9020008A9020008A9020008A9020008A9020008A9020008A9020008A9020008A8
:2000C000A9020008A9020008A9020008A9020008A9020008A9020008A9020008A902000888
:2000E000A9020008A9020008A9020008A9020008A9020008A9020008A9020008A902000868
:20010000A9020008A9020008A9020008A9020008A9020008A9020008A9020008A902000847
:20012000A9020008A9020008A9020008A9020008A9020008A9020008A9020008A902000827
:20014000A9020008A9020008A9020008A9020008A9020008A9020008A9020008A902000807
:20016000A9020008A9020008A9020008A9020008A9020008A9020008A9020008A9020008E7
:20018000A9020008A9020008A9020008A9020008A9020008A9020008A9020008A9020008C7
:2001A000A9020008A9020008A9020008A9020008A9020008A9020008A9020008A9020008A7
:2001C000A9020008A9020008A9020008A9020008A9020008A9020008A9020008A902000887
:2001E000A9020008A9020008A9020008A9020008A9020008A9020008A9020008A902000867
:20020000A9020008A9020008A9020008A9020008A9020008A9020008A9020008A902000846
:20022000A9020008A9020008A9020008A9020008A9020008A9020008A9020008A902000826
:20024000A9020008A9020008A9020008A9020008A9020008A9020008A9020008A902000806
:20026000A9020008A9020008A9020008A9020008A9020008A9020008A9020008A9020008E6
:20028000A9020008A9020008A9020008A9020008A9020008A902000800000000000000002C
:2002A000FFECC2925D7D05C5EFF305801EF0040F02D0EFF309818D466A4602F16802EFF3D3
:2002C00011831EF0100F0CBF2DED108A90B02DE9FC4F6946DFF828D000F070FAB0E8FC4F82
:2002E0001EF0100F0CBFB0EC108A40301EF0040F0CBF80F3088880F3098883F311887047A7
:200300000004002408B51E4B1E48DA1CC11E121A22F00302994288BF0022002100F0A5FC1B
:20032000194B1A48DA1CC11E121A22F00302994288BF0022164900F083FB00F01BF900F0DA
:2003400055FA00F075F9BFF34F8FBFF36F8F4FF0E023D3F8902F22F00102C3F8902FD3F88A
:20036000942F22F00102C3F8942FBFF34F8FBFF36F8F00F0C2FC00F00CFA00F0CBFC00BFCD
:200380003C150024000100240001002400000024C0A50008704A82B0D2F8003423F4802369
:2003A00043F48033C2F800346C4B0193019B002B00F3C980019B002B40F3C380664BD3F85E
:2003C000182422F4706222F00F0242F00802C3F81824D3F81C2422F4E06242F04002C3F811
:2003E0001C24D3F81C2422F4E06242F48062C3F81C24D3F8182422F0700242F04002C3F88D
:200400001824D3F8202422F0700242F04002C3F82024534AC3F82824524AC3F83024524AAF
:20042000C3F8382402F50032C3F840244F4AC3F82C24D3F8002442F0A852C3F80024D3F8F4
:2004400000249001FBD5D3F800241101FBD5424BD3F800249200FBD5D3F80C2842F006022F
:20046000C3F80C28D3F8182842F44042C3F81828D3F818289004FBD5374BD3F80428910452
:20048000FBD5D3F8F4244FF0B04142F00202C3F8F424D1F82C2442F00102C1F82C24D3F84E
:2004A00018289204FBD5324A22211160D3F8102422F0070242F00302C3F81024264BD3F8EA
:2004C000102402F03802182AF9D1D3F8542422F4405242F40052C3F85424D3F8582422F4AD
:2004E000407242F40072C3F85824D3F8502422F4E04242F48052C3F85024D3F8502422F468
:20050000E02242F48032C3F85024D3F8582422F0E04242F08052C3F85824D3F8542422F4B3
:20052000401242F40012C3F85424D3F8582422F44032C3F85824D3F8502422F04052C3F84A
:20054000502402B07047D2F800349B033FF532AF019B013B29E700BF0040025848BE2100A5
:2005600012202000770203072F0201018808BF000020005210B52A4C00200122D4F8003434
:2005800043F00103C4F80034264BC3F80821C4F81004254BD4F80024134043F01003C4F85A
:2005A0000034224BC4F82C34D4F8003423F48023C4F80034C4F8600400F07CF8FFF7EAFE72
:2005C000D4F8D83443F0006343F00103C4F8D834D4F8DC34C4F8DC34D4F8D434C4F8D4346E
:2005E000D4F8E03443F0805343F09F03C4F8E034D4F8E834C4F8E834D4F8EC34C4F8EC34E8
:20060000D4F8F03443F01003C4F8F034D4F8E434C4F8E434D4F8F434C4F8F43410BD00BFA8
:20062000004002580080005167EFFEEA0000FF017047FFEC30B4EFF3118400238022EFF36D
:20064000108372B682F3118883F31088BFF34F8F164B174AD3F80038118803F4807578B1C0
:2006600001311180128875B1C2B10023BFF34F8FE4B284F31188BBB1042030BC00F04DB8BA
:2006800051B10139EDE7002AEFD043F48073074AC2F800380123E9E7002DE6D023F4807313
:2006A000024AC2F80038E0E730BC70470040025800040024EFF3118200238021EFF3108322
:2006C00072B681F3118883F310880749D1F8003823F48073C1F800380021044B1980D3B2FD
:2006E00083F31188FFF7A6BF004002580004002430B5EFF3118400238025EFF3108372B60D
:2007000085F3118883F31088036823EA0101E3B20A43026083F3118830BD82B0002245F275
:200720006161B0F57A7F0BD8002240F6A201642811D800220A2818D8002200BB02B070477C
:200740000192019B8B4202DDA0F57A70E9E7019B01330193F5E70192019B8B4201DD6438B9
:20076000E5E7019B01330193F6E70192019BDC2B01DD0A38DEE7019B01330193F6E701927D
:20078000019B152B01DD0138D7E7019B01330193F6E7BFF34F8FBFF36F8F4FF0E0230022C3
:2007A000C3F8502FD3F8142D42F40032C3F8142DBFF34F8FBFF36F8F7047FFEC37B50A4D6A
:2007C0000C462B680BB91C462960019000F0F5F82968019800F080FB14B900232C682B6073
:2007E000204603B030BD00BF04040024EFF3148343F0040383F314884FF0E023D3F8342FD3
:2008000022F04042C3F8342FD3F8882D42F47002C3F8882D7047FFEC0F2810B531DDA0F151
:2008200010041F2C0ADC03F1604303F561430B60012303FA04F4146000201CE03F2C08D8E1
:200840001C4C30381C440C60012303FA00F01060F2E75F2C04D8184C50381C440C60F3E7A9
:200860007F2C04D8154C70381C440C60ECE7952C02D94FF0FF3010BD114C90381C440C6081
:20088000E2E7104B04280B6003D14FF480331360D2E7052802D14FF40033F8E7062802D151
:2008A0004FF48023F3E70F28E3D1074B0B600123EDE700BF04E100E008E100E00CE100E0BE
:2008C00010E100E024ED00E010E000E008B54FF0E02320494FF0FF305B6803F00F035A1C72
:2008E00003F1382361339B0041F8040B8B42FBD14FF0E0231849C3F8081D4FF08031C3F86B
:20090000181DC3F81C1DC3F8201D5301134A03F1604303F5644342F8041B9342FBD1104B7A
:20092000002210490B201A6000F0AEFA00220E49032000F0A9FA4FF0E022D2F81C3D23F059
:200940007F4343F0E043C2F81C3DF02383F3118862B608BD80E100E00000000800E400E060
:2009600004040024ED090008BD09000813B5802301AA69460446FFF74FFF20B90F2CDDE952
:20098000003102DD196002B010BD1A6822EA01021A60F8E713B5002301AA69460446FFF7E0
:2009A0003BFF20B90F2CDDE9003102DD196002B010BD1A680A431A60F9E7704708B54FF03F
:2009C000E023D3F82C2DD3F8283DEFF3118300238022EFF3108372B682F3118883F31088CC
:2009E000AD21014800F034F99C9F0008CA6E012A08B508D0022A0AD01AB9D422086F00F052
:200A00001FF8002008BD0A6F034B1A60F9E70A6F11604A6FF8E700BF04040024FFECC2920D
:200A200018DF88DFCD06CD767CD30CD3D982D9122C00050A0F14191E232800BFAFF300800D
:200A400000B501B400F004F801BC00BDAFF3008000B5042A60DB00F0030E61F3830E7A4BDB
:200A6000D3E80EF0AFF30080AFF30080AFF3008011F8013B00F8013BA2F1010211F8013B03
:200A800000F8013BA2F1010211F8013B00F8013BA2F101022DE9F01F282A07DBB1E8F81F74
:200AA000A0E8F81FA2F12802282AF7DADFF89CE14FEA920BDEE80BF051F8043B40F8043BCD
:200AC00026E0B1E81800A0E8180021E0B1E83800A0E838001CE0B1E87800A0E8780017E029
:200AE000B1E8F800A0E8F80012E0B1E8F801A0E8F8010DE0B1E8F803A0E8F80308E0B1E85B
:200B0000F807A0E8F80703E0B1E8F80FA0E8F80FBDE8F01F02F00302002A08BF00BD11F8DB
:200B2000013B00F8013B013A08BF00BD11F8013B00F8013B013A08BF00BD11F8013B00F811
:200B4000013B00BDAFF30080AFF30080AFF3008011F8013B00F8013BA2F1010211F8013BE2
:200B600000F8013BA2F1010211F8013B00F8013BA2F10102282A35DB2DE9F01FB1E8F81F65
:200B800020F8023B4FEA134364F31F434FEA144465F31F444FEA154566F31F454FEA164687
:200BA00067F31F464FEA174768F31F474FEA184869F31F484FEA19496AF31F494FEA1A4AC5
:200BC0006BF31F4A4FEA1B4B6CF31F4BA0E8F80F4FEA1C4C20F802CBA2F12802282ACDDA1B
:200BE000BDE8F01F042A97DB51F8043B20F8023B4FEA134320F8023BA2F10402BAE711F89D
:200C0000013B00F8013BA2F1010211F8013B00F8013BA2F1010211F8013B00F8013BA2F1B3
:200C20000102042AFFF678AF51F8043B00F8013B4FEA132320F8023B4FEA134300F8013B24
:200C4000A2F10402EDE70000200A0008300A000808B501F09BFA012000F004F8012008B585
:200C600000F000F808B500F07DFB002A43D010F0010F034639D0013A03F8011B012A38D93A
:200C8000F0B541EA01259E07ADB22BD0023A23F8025B032A18D95C0745EA054616BF141FA8
:200CA000144643F8046B224603EB040C072A13D8E2086FF0070707FB02423C40032A234401
:200CC00084BF043A43F8046B012A02D9023A23F8025B02B11970F0BDACEB0207083AC7E9B4
:200CE0000066E3E7032AD6D8F0E7012AC8D1197001E0002AFBD17047704700F008B80020B0
:200D000070470021084601F005BA04F0EBBC70477047FFEC3C4C01233C4D8C2204F17006BB
:200D20002B7083B500212046FFF79FFF03231822374923773046374B374FC4E905330623BF
:200D4000E38303F0A3FD354920463E6003F0A9FB334B01A96846334E1C6002232B7001F0FD
:200D600009FADDE9000103F0ADF9042333603368012B45DD3068800003F0C2F92A4B1860BA
:200D8000336804602048A17F00F008FBA3681E48DB685F6001F04EFB1B4800F0F1FA1A488C
:200DA00000F01AFBA36805221A7200221F4B1A6003232B7000F0C0F806F07AFC1C4B0BB172
:200DC00000F032FB1B4B0BB107F095FA1A4B0BB100F080FF01F09CF901F06CFA05F061F893
:200DE000042309482B7000F01AFB05232B7000F039F806232B7000F0AFF801F019FBFCE7B4
:200E000033685B00B2E700BF10040024AC040024B49F0008150D000808040024BC040024DF
:200E2000C4040024A8040024B8040024A404002429140008F7820008D51C000813B500249F
:200E4000FFF75FFF054B40F67A4264210094044800F0D9F8204602B010BD00BFB1980008E1
:200E600000A0000813B50024054B4FF40062FE210094044800F0E0F8204602B010BD00BF7E
:200E80003D0E000810A00008A52870B505460C461AD8EFF3118600238021EFF3108372B6EC
:200EA00081F3118883F310881CB9FFF75FFD2246074C0848F6B240F8354000EBC50042603E
:200EC00086F31188002070BD6FF01500FBE700BF150F0008E0040024A52808B50CD8094AA9
:200EE00052F830305BB102EBC00252689847064B1A68064B1A6008BD0022054BF6E71A46E2
:200F0000FBE700BFE0040024BC040024C4040024150F000808B5EFF3118300238022EFF352
:200F2000108372B682F3118883F3108836210148FFF78EFE1BA00008054B1B682BB1054AF7
:200F4000126812B91A8C01321A840020704700BFBC04002404040024134B10B51A68C2B117
:200F6000124B1B68ABB9EFF311848021EFF3108372B681F3118883F31088B2F92030002B37
:200F800009DC002313840A4B1B6853B9E4B284F31188002010BD013B9BB21384002BF5D12A
:200FA000EFE701F09FF9F1E7BC04002404040024B004002470B586B005468C200E46CDE9B6
:200FC000043203F09DF80446D0B10021C68303910C9902910B9901910A99DDE904320091EC
:200FE000294600F033F8051E05DA204603F078F8284606B070BD2046E56800F077F9F7E75A
:201000006FF00B05F4E71FB5069C00920A46CDE9013400231946FFF7CDFF04B010BD1FB5AA
:20102000079C0294069CCDE9003413460A460221FFF7C0FF04B010BD13B5049CCDE9003497
:2010400013460022FFF7EBFF02B010BD2DE9F347867F88460546914631461F46DDF828A0F8
:2010600000F09CF9041E3ADB284606F0030600F0D8F9041E0CDB87B152463946284601F0CF
:201080009FF9041E05DB284600F07AF9041E13DA57B1284600F0A6F921E032465146284653
:2010A00001F0C6F8041EEEDAAB6B002BF1D03146284601F031F9ECE70B9B49460A4A2846CB
:2010C000009600F013F8041EE2DB0C9A4146284600F0A0F8041EDBDB284600F07DF920466B
:2010E00002B0BDE8F08700BF111300082DE9F74F04460E4601929946EFF31187002380228C
:20110000EFF3108372B682F3118883F31088DFF8FCA0DFF8FC80DAF800500020D8F800300E
:201120000135384A116888420DDB1068C00002F0E7FF344A0546002845D1FFB287F31188F1
:201140006FF00B0039E0012D1168B8BF01250139294053F821B003EB810EBBF1000F2FD1D1
:20116000CEF80040FFB2E560CAF8005087F31188019BF6B29DF8302059460320267402F0D7
:2011800003026674C4E90539E38B23F06303134304F14402E38300F083F9204684F81CB08D
:2011A00001F048F9FFF7C8FE1749204603F079F904232377FFF7D0FE584603B0BDE8F08F1C
:2011C00001350130AEE711684FF0000C0D4B490011601A68D8F8000002EBD272BCEB620FA2
:2011E00004DB02F07DFFC8F8005094E750F82C000CF1010C1A68C168013A0A4045F822000A
:20120000E7E700BFA80400249C040024A4040024B8040024344B2DE9F74F002914BF89465B
:20122000994607460024154649461822703003F051FB484687F8884003F044FB461C4DBBEA
:201240002C460234384606EB840101F077F806464FEA8408002844D000EB080AA8F108089F
:20126000B346043DC0F800A0484603F02BFB0446B04449460134504603F000FB5444D845FA
:201280001BD100204AF8040CBA68D268566003B0BDE8F08F40F2011855F824000028D0D083
:2012A00003F010FB01307B6B06449E4216D201344445F1D16FF00600E9E74BF8044F55F86F
:2012C000041F0846019103F0FDFA81460199204609F1010903F0D2FA4C44D0E76FF05A0097
:2012E000D5E76FF00B00D2E733A0000810B5EFF3118400238022EFF3108372B682F3118888
:2013000083F3108801F03EF8E4B284F3118810BD38B5134B1C68E38B03F00303022B02D0F0
:20132000204600F0ABFBA368012040F20111DB685A6852F820304BB9E38BA56903F0030329
:20134000022B08D11146A847FFF78CFC01308842EFD10120F8E70146284603F0BBF8F8E7CE
:20136000BC0400240446002208B5E4B2034B2146186800F0ABFB204600F080FFBC04002446
:2013800010B51821044600F0D9FF20B1A368DB680360002010BD6FF00B00FBE770B5064611
:2013A0004FF48E7002F0ACFE044690B100F0B3FB051E04DA204602F093FE284670BD04F1AD
:2013C0002400B46006F0A5F92046002503F08FF9F3E76FF00B05F0E7D0E902321A60012291
:2013E0005A72704738B58468054634B1637A012B04D9013B63720023AB6038BD204600F0F1
:201400009BFB204600F032F904F1240006F085F9204603F08BF9204602F062FEEBE700F0D1
:2014200098BB00F096BBFFEC0023044A044942F833100133A62BFAD1FFF748BAE004002422
:20144000150F000838B5044618B3C068B0B1EFF3118200238025EFF3108372B685F31188EA
:2014600083F310880C4B00251B68013B03400B48006840F82350D3B283F31188A36B13B114
:20148000204600F049FF2046FFF7ACFF204602F027FE002038BD00BFA8040024B8040024A6
:2014A000F8B51746194B06460C461D68FFF744FD0FB16B6C3B60D4B1EFF311830022802174
:2014C000EFF3108272B681F3118882F31088022E11D0032E14D0012E14D16A6C21680A4370
:2014E00000246A64DBB283F3118800F011F8FFF733FD2046F8BD21686A6C22EA0102EFE7E0
:201500002268EDE76FF01504ECE700BFBC040024184B30B51D6885B0FFF70EFD6C6C284636
:2015200000F0F4FCE4430440039424B9FFF714FD204605B030BD03A800F070F8431C014634
:2015400010D0019003A803F00FF80199284600F013F8044630B1011D284600F09BF82046D2
:2015600000F02EF8039B002BE5D1FFF7F5FC0120DFE700BFBC04002438B58368EFF3118515
:2015800000228020EFF3108272B680F3118882F3108800209C6974B122798A4206D103F158
:2015A000180130B9084602F057FF04E020462468F1E702F05BFFEDB285F31188204638BD8E
:2015C00010B5037B83B9EFF311848022EFF3108372B682F3118883F310880E4902F01CFF56
:2015E000E4B284F3118810BD022B0CD1EFF3118400238022EFF3108372B682F3118883F311
:2016000010880549EAE7012BEDD1BDE8104002F067BD00BF300A0024280A002438B5054673
:2016200001242146284602F0B0FF20B90134202CF7D14FF0FF34204638BD38B5044600F1F8
:201640004C05284602F008FF50B904F15405284602F002FF38B94FF0FF32C4E9112038BDE6
:2016600000F0AEFCEDE700F0ABFCF0E738B5044600F11005284602F0EFFE28B91834204671
:2016800002F0EAFE18B938BD00F082FBF2E7FFF797FFF4E72DE9F0410D460978044629B3BC
:2016A000443002F072FF012807467ED1EFF3118600238022EFF3108372B682F3118883F32F
:2016C0001088237FF6B2062B12D1297804F1480002F05BFF60B12B682046E3656B6823663C
:2016E0000023A36400F04EFE86F311880026B4E086F31188A4682978EFF3118200238020C1
:20170000EFF3108372B680F3118883F31088A36913B11879884208D1D2B282F3118833B198
:201720002A685A606A689A60E0E71B68F0E7564B1B68FBB1554802F08FFE20B9544802F01D
:201740008BFE0028D2D02B6843606B688360EFF3118500238022EFF3108372B682F3118862
:2017600083F3108804F11801EDB202F055FE85F31188BBE7EFF3118600238022EFF3108303
:2017800072B682F3118883F310884048F6B202F063FE86F311880028D5D1102002F0A8FCDC
:2017A0000028A3D001230373CDE7FFF7C5FB2978A06800F0C7FB064600282CD0406848B31C
:2017C00000F0D2FB00284BD073684360B2688260F3689B0604D4297801238B4013438360F2
:2017E0002B68C3606B680361EFF3118600238022EFF3108372B682F3118883F3108804F110
:201800004C01F6B202F008FE2249204600F04EFE86F311880026FFF79FFBEFF31188002368
:201820008022EFF3108372B682F3118883F31088237F062B08D12B682046E3656B68236604
:201840000023A36400F09EFD5FFA88F888F31188002F08D001DA6FF015063046BDE8F081FE
:201860006FF00B06D7E7237F052B03D10421204600F012FA237F072BEFD12B78082BECD1E6
:20188000204600F0C6F9E8E704040024300A0024280A0024B918000807B5019100F072F902
:2018A00028B1019903B05DF804EBFFF7F3BE6FF0020003B05DF804FB2DE9F04F87B00446D9
:2018C00002F0A0FD03684FF0800904F14C0A019304F15408B4F922300293EFF31183039F6A
:2018E000EFF3108772B689F3118887F31088E28B0397DFB212F400720AD087F3118802F031
:2019000081FD019B0360029B638407B0BDE8F08F5046059202F0A0FD059A06460028ECD060
:20192000E18B059241F40071E183414602F074FDD4F844B0B5684BEA0505656487F31188B8
:20194000736806F10C01059A307B9847EFF31183049A0593EFF3108272B689F3118882F3AD
:20196000108804924146E28B304622F40072E283626C554082EA0B02154085EA0B05656469
:2019800002F054FD059BDBB283F31188FFF7C0FD304600F015FBA0E77047FFEC054B10B561
:2019A0001C68FFF7C9FA204600F012F9BDE81040FFF7D2BABC04002408B5024B01201B6880
:2019C000FFF750F9BC04002408B58068203002F0DCFD0028D4BF0020012008BD0023084AEE
:2019E00012F83310814206D102EBC3035878C04300F00100704701330B2BF1D101207047CE
:201A00003CA0000838B585685AB100231A4A12F83300814219D102EBC30305F120005C68FF
:201A2000BCB9EFF3118400238022EFF3108372B682F3118883F3108805F12000E4B202F09E
:201A400093FD84F31188002413E001330B2BDED1E7E7EFF3118500238022EFF3108372B60E
:201A600082F3118883F3108802F071FDEDB285F31188204638BD00BF3CA000082DE9F043F3
:201A800086680024104D4FF002092036A04685B0304602F076FD6B6873B12F7801A90022D7
:201AA000CDF80C903846CDE90138012300F086F93946304602F04BFD013408350B2CEAD132
:201AC000002005B0BDE8F0833CA0000810B5C38B04461B0515D43AB9806828B1437A012B32
:201AE00002D12C3002F06DFD204600F00BF82046FFF778FC2046FFF7A0FDE38B43F4006331
:201B0000E38310BD10B5044600F020F82046BDE8104000F0A8B838B50546382002F0F0FA64
:201B2000044630B10122002102F0DFFC0020EC6038BD6FF00B00FBE710B5C468204600F075
:201B40007AF82046BDE8104002F0CABA243000F065BA002307B5024601900121184606F0B1
:201B6000A5FA019A00230621012006F09FFA0023019A0621022006F099FA002003B05DF879
:201B800004FBFFEC0346EFF3118100228020EFF3108272B680F3118882F310880A4A10685B
:201BA00060B1002B0EDB094A1268013A1A4050F8220018B1C2689A4218BF0020CBB283F37B
:201BC000118870470020F9E7B8040024A804002438B50446EFF3118500238022EFF310831C
:201BE00072B682F3118883F31088037F043B032B0BD800F05BFA042307212046638400F0FE
:201C000041FAEDB285F3118838BD072100F0E4FAF7E710B5EFF3118400238022EFF310839A
:201C200072B682F3118883F3108800F0ABFBE4B284F3118810BD30B103881B0401D40123D3
:201C40000380002070476FF01500704710B5FFF7F2FF041E05DA644202F0D4FB04604FF048
:201C6000FF34204610BDEFF3118200238021EFF3108372B681F3118883F31088037F052B5B
:201C800006D1016C0B8801331BB20B8000230364D3B283F31188704738B5EFF31184002286
:201CA0008025EFF3108272B685F3118882F31088027F052A09D1056C2A88013212B22A8077
:201CC00000224184026400F05DFBE4B284F3118838BDFFECF8B50024284B294E6020C3E902
:201CE0000044284BC3E90044274BC3E90044274BC6E90044C3E9004402F0FAF9054648B15D
:201D000000F160072C7528461835314602F084FBAF42F7D1602002F0EBF9044658B100F1D4
:201D200060050227174E277520461834314602F073FBA542F7D1402002F0DAF9044658B164
:201D400000F140050027104E277320461034314602F062FBA542F7D1402002F0C9F90446B1
:201D600058B100F140050227084E277320461034314602F051FBA542F7D1F8BD100A00240A
:201D8000180A0024200A0024300A0024280A002410B5EFF3118400238022EFF3108372B65D
:201DA00082F3118883F310880349E4B202F034FB84F3118810BD00BF100A00242DE9F74FCE
:201DC0001546504A1F280746D2F800B00E46DBF808A004D96FF0150003B0BDE8F08F41B90F
:201DE0003946504600F0AEF8044665B916BB0020F2E7002BF4D10B68012BF1D0FFF7EEFDD5
:201E00000028EDD1E6E739465846FFF7DDFD30B100230122C5E900230223AB60E6E72CB150
:201E200063682B60A3686B60E368F6E7C5E90044AC60DBE73568012D11D12A463946584654
:201E4000FFF7E0FD054685B9002CD0D020460AF1100102F0EBFA2046FFF79AFFC7E700224C
:201E600039465846FFF7CEFDEDE7D4B9EFF311834FF0800B00930022EFF3108272B68BF314
:201E8000118882F31088204802F0E6FA009B0446DBB283F3118850B10AF11001077402F067
:201EA000BBFA65607368A360B368E3609FE7502002F01EF914490446C0B1EFF31183EFF3FD
:201EC000108972B68BF3118889F3108800F1500220461434CDE9002302F09EFA009A0A49D5
:201EE0009442019BF4D1DBB283F31188EFF311830093EFF3108872B68BF3118888F310883A
:201F00000846C1E7BC040024100A0024002337B582680193EFF311858021EFF3108372B666
:201F200081F3118883F3108894692CB9EDB285F31188019803B030BD217901A802F007FB84
:201F40002468F2E738B50D46044640B1FEF7F4FF246914B1237CAB4203D1FEF7FDFF2046B0
:201F600038BD2468F5E7FFEC124B10B51B6843B1114802F071FAE0B91048BDE8104002F0F2
:201F80006BBAEFF3118400238022EFF3108372B682F3118883F310880748E4B202F05CFAFA
:201FA00084F3118828B9182002F0A2F808B10123037510BD04040024180A0024200A00248A
:201FC00010B5037D83B9EFF311848022EFF3108372B682F3118883F310880E4902F01CFA4F
:201FE000E4B284F3118810BD022B0CD1EFF3118400238022EFF3108372B682F3118883F307
:2020000010880549EAE7012BEDD1BDE8104002F067B800BF180A0024200A002438B504468F
:20202000EFF3118500238022EFF3108372B682F3118883F31088F0B14368E3B1104B00204F
:202040001B68DBB1A3420FD123681BB19A68A1680A449A6058B10A4902F008FA00206060D2
:20206000EDB285F3118838BD18461B68E9E7044802F0F2F9F2E76FF01500F1E71B68FFDE5C
:20208000380A002438B50C46074B054653F8311003EBC4031B79DB0703D500F015F82C77CF
:2020A00038BD02F0F3F9FAE7C09F0008054B027F10B553F83210044602F0FEF900232377F2
:2020C00010BD00BFC09F000810B50B68027CB3B11C7C944206D25A6862B9C0E9003258603D
:2020E000086013E01B68F2E7C0E900321060486000200CE0C0E9003210605860F8E74A6896
:20210000002AF1D1C0E90033C1E90000012010BD7047FFEC37B5124D2C682CB1114802F0B6
:202120003DFA012003B030BD0F4802F037FA40F2011369464FF60C70ADF800308DF80240DB
:20214000019503F075FE011E04DA4942074802F025FAE6E7064802F021FA2046E2E700BF85
:20216000400A002494A00008B7A00008E2A0000821A10008044B1B680360C3F1105303F5BE
:2021800000230B60704700BF989F000808B504F0DBFB04F0D9FB04F0D7FB0D4B186818B93E
:2021A0000C4B1B681B6873B9002007F06BFCEFF3118300238022EFF3108372B682F3118832
:2021C00083F31088FEE7BDE8084007F05BBC00BF04040024BC040024F7B50646114D01915A
:2021E0002F6806F0BFF8019904463046FFF74AFF0D4B1B681BB106F0C9F82043C4B234B1E6
:202200000A4B1A682AB1FA662A68D26E1A6003B0F0BD2B6807F16C00D96E03B0BDE8F0403A
:2022200000F0A7B8BC040024B00400240404002438B5836B0C46054611469BB9204601F0ED
:2022400057FFA863A86BB0B10119E86321F00701091A696300F0CCF8EB8B002043F48053E8
:20226000EB8338BD436BA342ECD000F055F8AB6B002BE7D1E2E74FF0FF30F2E7094C08B554
:202280002368EFF3118300238022EFF3108372B682F3118883F3108806F0D0F92368D86E2F
:2022A00000F002F8BC0400240146012000B500DF5DF804FB08B5084AC0230849013B42F847
:2022C000041BFBD1064B0BB1AFF3008000F042FBBDE8084001F08ABC00010024EFBEADDE36
:2022E0000000000038B50A4C256806F04FF830B1084B1A6822B1EA662268D26E1A6038BDBF
:20230000236805F16C00D96EBDE8384000F031B8BC0400240404002410B50446806B20B1B8
:20232000E38BDB0401D501F0DBFEE38B23F48053E3830023C4E90E33636310BD38B5073129
:20234000836B044621F007057BB1436BAB420ED9C36B2A4600211846FEF787FCE26B03464F
:202360002A44E263626B521B6263184638BD0023FBE703460A460220194600B500DF5DF850
:2023800004FBFFEC70B505460B4C2668FFF78EFE284605F0C3FF30B1084B1A6822B1F26676
:2023A0002268D26E1A6070BD236806F16C00D96EBDE87040FFF7DDBFBC0400240404002480
:2023C00070B5836B06460D46144623B1C18B01F00301FFF7A1FF2C44284624F00704611BCD
:2023E000C6E90E55716300F003F8002070BDFFEC90B5C41D83B024F0070400AF224679B913
:20240000391DB94228BF394621F00703191A074B21F0030121448A4204D10C37BD4690BDB7
:202420000144F1E742F8043BF5E700BFEFBEADDE7047FFEC38B50025C16804464566856676
:20244000C56661B9184B186840F2EE23A0F2EE206363C4E90E00BDE83840FFF7C9BF406BAA
:20246000D4222946A0F1D403E06B1844E066FEF7FCFBE36B616BE26E0B4413606369E26E6E
:2024800023F00103C2F884304FF08072E36EC3F888206FF01602E36E9A62F022E36EC3F8F0
:2024A000CC50E36E5A6038BD989F000810B5436E044603BB1B4B1A6882421DD11A4C2368B8
:2024C00013B9BDE810400847A3F1D400C2E919132060D4221946FEF7B3FA236803F1D402E1
:2024E0001A60124A2368C3F8842080225A604FF08072C3F8882010BD4166D422C16E8166AC
:20250000A1F1D400E066FEF79BFAE36E03F1D4021A60064AE36EC3F884208022E36E5A6043
:20252000E36EE4E7BC040024040400243125000838B50D4B1C68F023A56E83F3118862B6FB
:20254000636E20469847EFF3118300238022EFF3108372B682F3118883F3108800232846E0
:202560006366FFF7A1FE00BFBC04002410B5846E01F4D873A0F8501001F00101226822F4D8
:20258000D87213432360826E936823F001031943916010BD10B5EFF3118400238022EFF319
:2025A000108372B682F3118883F31088FFF7DEFFE4B284F3118810BDF0B5C26BEFF31184B5
:2025C00000238021EFF3108372B681F3118883F31088916E0B6823F0010003F00105086098
:2025E000D66D576E710801EB4701B1FBF6F1642933D9013123F40040490820F00100936E0E
:202600001860936ED96092F856101F4B012903EA00032CD143F4C06392F85700092802D059
:20262000082829D141B343F48053916E0B60906E92F85860416821F440510EB141F4005134
:2026400041602B43906EE4B2816821F440718160926E136084F31188F0BDC1F3420321F00D
:202660000F0140F400400904090C1943C7E7022908BF43F48063CFE7B2F85610B1F5E06FE3
:2026800008BF43F08053D0E7FEE9FFEFC36B9A6E506AB3F8522040EA0242C0B20A60002268
:2026A000A3F85220704710B5C06BEFF3118400238022EFF3108372B682F3118883F3108871
:2026C000B0F8503039B143F02001E4B2FFF762FF84F3118810BD23F4907121F00101F4E7C4
:2026E000C36B9B6ED869C0F340107047C36B9B6E9962704710B5C06BEFF311840023802293
:20270000EFF3108372B682F3118883F31088B0F8503041B143EA020189B2E4B2FFF73AFFB6
:2027200084F3118810BD23F08001F5E7C36B9B6ED869C0F3C010704738B583685D6940F2CA
:2027400001139942EC6B05D0B1F5817F21D06FF0180038BD002A3CD094F85630BBB1012B7B
:202760004FF480710CBF4FF4007300230B4394F858101046002914BF402100210B4343F0EA
:2027800030039360E16D02F0B7F80020E1E71946ECE7F2B1936803F03001302919D113F4FE
:2027A000807113D013F4007F14BF0123022384F8563093681046C3F3801384F8583002F011
:2027C000BBF8E0652846FFF7F7FEDEE784F85610EFE76FF01500BCE710B5C46B94F8600034
:2027E000FEF7C4F8002294F860001146BDE81040FEF74ABB38B5C56B06492A4695F860000B
:20280000FEF742FB044618B995F86000FEF7C2F8204638BD1928000810B51446926ED369D0
:202820009BB29806A4F8523013D5B4F8501089060FD5204604F041F8B4F852301A0606D56C
:20284000B4F850301B0602D5204604F000F8002010BD13F00E0FEFD00E231362ECE7FFECD2
:2028600038B5C46B00210546A36E1960C36B9A6E1B4B9A4203D110221A48FDF739FFE06EEC
:2028800001F020FB206F01F01DFBA26E94F85810536823F47D5309B143F400535360284689
:2028A000A26E114B11680B401360A26E94F85510936823F4E06323F0010343EA4163936044
:2028C000FFF77AFEA26E0020136843F0005343F00D0313600123A4F8500084F8543038BD9E
:2028E00000100140F044025803BEFF33F8B50026C46B054684F85460EFF3118780223346F4
:20290000EFF3108372B682F3118883F3108831462046FFF72BFEFFB287F31188EB6B9A6EE0
:202920000A4B9A4204D1324610210948FDF7E0FEA26E136823F00D031360E06E01F0A4FBC6
:20294000206FBDE8F84001F09FBB00BF00100140F04402587FB50B49684601F08FFF00234A
:20296000094D1C4655F8041B39B15E1C303368468DF8093003F088FD33460134082CF1D1E4
:2029800004B070BD5CA1000868A10008704738B50A460169044629B14B69036103B9436146
:2029A00000234B61637E207EC3F3C00520B9E068007C60F3C3036376CB6820464A8198477C
:2029C000637E65F3C303637638BD37B50446C0680A4680B10368B4F85E10009121469D68C9
:2029E00004F11D03A847002803DA237C43F00103237403B030BD6FF00400F6E7F0B5047E5A
:202A000044B313466401154FE5592E0415D4AE03134E48BF45F080652E40334343EA81433C
:202A200001F04F0143F0805343F40043E351437EC28023F04F0319434176037E0020094933
:202A400003F110020123D1F81C4893402343C1F81C38F0BD21462346D4E700BF000B08408F
:202A600000F8F3FF00000840E0B590F818C0144E4FEA4C17BD592B0417D4AB03114B48BFF0
:202A800045F080652B40134343EA814301F04F0143EA8C5343F0805343F40043BB51437ED0
:202AA000C28023F04F0319434176007E0123064A83400020D2F81C180B43C2F81C38E0BD90
:202AC0000009084000F833FC00000840437E8A88DB06C97801F0030101D5FFF7C5BFFFF706
:202AE0008DBFFFEC417E027ECB064FEA42124CBF084B094B890713441A6822F4001248BFB8
:202B000042F080521A60437E6FF3C30343760020704700BF00090840000B084001F07F01EA
:202B2000F0B5EFF3118400238025EFF3108372B685F3118883F310888618F57CC9B106293D
:202B400022D8012303FA01F12940D1B101239C460CFA03F73942BE4610D025EA0E05E4B260
:202B6000F57484F311881C214B4322B160331844F0BD2946E9E703F59273F8E70133072B21
:202B8000E6D1E4B284F311880020F1E710B5C0B1B9B1EFF3118200238024EFF3108372B667
:202BA00084F3118883F310884B7E097EC3F30013184401238B40C17C0B43C374D3B283F3D6
:202BC000118810BD024BD3F80808C0F30D20704700000840037C61F3410303740020704723
:202BE000EFF3118200238020EFF3108372B680F3118883F310880848D0F8043841B123F08D
:202C00000203C0F80438D3B283F311880020704743F00203F5E700BF00000840084601F0F6
:202C20005FBA10B5182001F063FA044618B118220021FEF71AF8204610BDFFEC70B5EFF396
:202C4000118600238022EFF3108372B682F3118883F31088037CDA0611D50B4CD4F80838B7
:202C6000DB070CD5D4F80458052045F0010325F00105C4F8043801F0F9F8C4F80458F6B256
:202C800086F31188002070BD0000084070B54B7E05460C465B070CD422695AB9237E1A481F
:202CA0005B01195841F000611950637E62F38203637670BDD18819B92046FFF768FEEBE7CC
:202CC000E388124E5A1E1144227EB1FBF3F152014B43905943EAC1430B4900F06040034307
:202CE0009351237E5B015A5842F004425A50637E43F004036376237E002BDAD16B7C0622A5
:202D000062F307136B74D4E7000B0840100B0840002882B006DD0023034904330A689842C5
:202D20000192FADC02B070470010084030B503460B4C1A1D1B1A994200DC30BD2368C3F393
:202D4000072502F8043C02F8035CC3F30745C3F3076302F8025C02F8013C1346E9E700BF1B
:202D600000100840054B064AC3F8102BD3F8002B42F00442C3F8002B704700BF0000084053
:202D8000180008601023054A1361054B1169C90601D5013BFAD10320FDF7BFBC000008406D
:202DA000400D030040F02000054A064B10611169890601D5013BFAD10320FDF7AEBC00BF3C
:202DC00000000840400D030038B5036904460D4643B1437EDB0606D5007E8001FFF7E2FF1E
:202DE00023691BB938BDFFF7CDFFF9E729462046FFF7CDFDF4E710B5EFF31184002380226B
:202E0000EFF3108372B682F3118883F310886FF06D01E4B2FFF7D8FF84F31188002010BDCC
:202E200070B5437E0446DE063CD5037E3E495B015B581D0434D5EFF3118500238022EFF30D
:202E4000108372B682F3118883F31088027E5201535823F4004343F090435350334A037E1C
:202E6000590102EB431318688007FCD58B58EDB243F002038B50207E8001FFF793FF207E03
:202E80002B490122D1F81C388240204623EA0203C1F81C386FF06D01FFF796FF85F31188CE
:202EA000002070BDEFF3118600238022EFF3108372B682F3118883F310881D4DD5F804385B
:202EC00043F40073C5F80438D5F804381B07FBD5227E0A201749F6B25201535823F400432A
:202EE00043F090435350FDF718FC237E124A02215B0120469950D5F8043843F48063C5F876
:202F00000438227ED5F81C3802F1100101228A406FF06D0123EA0203C5F81C38FFF754FF8A
:202F200086F31188BCE700BF000908400809084000000840000B0840080B0840F0B5057E55
:202F40001F4F6D01EB5903F0004392B3C688541E3444B4FBF6F4467E134306F0030643EABF
:202F6000C443012E174E08BF43EA4473EB51457E047E05F003056401012DA35908D1124DC6
:202F8000D5F80858ED0554BF43F0805343F0005323F08043033243F004439210A351037ED7
:202FA00000201B0303F1804303F50123824202DCF0BD0124CFE751F8204001301C60F5E7A4
:202FC00010090840000908400000084010B504466030FFF7B3FF0422637C62F30713637465
:202FE000BDE81040FFF7BEBE00221146FFF7EEBFF8B50E6907460C465EB90B7E30495B0116
:203000005A5842F000625A50637E66F382036376F8BDF3881BB94B7E43F040034B76328969
:20302000F588AA4208D3637E590605D420460021BDE8F840FFF7ABBC637EAD1A6FF38613CF
:20304000002D63760ADDE388AB4207DC18D13379DB0703D5637E43F040036376217E194BC6
:203060004A01D258EB1C92B2B2EBA30F0ADA164A0123D2F834088B400343C2F83438C7E7EE
:203080001D46EBE733892A46316820461944FFF755FF637E43F004036376237E23B97B7CC1
:2030A000052262F307137B743289F3881544ADB2AB423581ACD8637E5A06A9D4B6E700BF5C
:2030C0000009084018090840000008401A4B024670B5C0688B60EFF3118500238024EFF3E8
:2030E000108372B684F3118883F31088537E13F008031DD114694B613CB9537E13F004062E
:20310000C2E9041109D0204603E05069416118465161EDB285F3118870BD13F01004114617
:2031200003D0FFF765FF3046F3E7FFF7AFFDEAE76FF00F00EDE700BF000089FF344A002078
:203140002DE9F047D2F80438324C23F00103C2F80438FFF727FEE06818B103682146DB6850
:203160009847FE232C4E2D4F00254FF0FF0A4FF01C09E374237509FB05483046C7F800A073
:203180006FF06D01C7F800A20135FFF71DFE98F8793006F1C4006FF06D0123F04C03203740
:2031A0001C3688F87930FFF70FFE98F83D31072D23F04C0388F83D31DDD1154B4FF0FF3291
:2031C00000211548C3F818284FF00112C3F81C280B22C3F81428C3F81028D3F8002822F405
:2031E000FE62C3F800284022238A23F4706323F00403238202232372FFF736FC402200216F
:203200000748FFF7FBFBBDE8F047FFF7ABBD00BF00000840C80D0024280E00240809084086
:20322000EC0E002438B5124D0446D5F8043843F40073C5F80438D5F804381B07FBD5227E93
:203240000A200C495201535843F0804343F400135350FDF762FAD5F80438002043F480637B
:20326000C5F80438637E43F00803637638BD00BF00000840000B0840427E0346D20601D458
:20328000FFF7D0BF027E06485201115841F40011115000205A7E42F008025A76704700BFFE
:2032A0000009084010B5EFF3118400238022EFF3108372B682F3118883F3108829B1FFF733
:2032C00011FCE4B284F3118810BDFFF7D5FFF8E72DE9F041437C044603F0F003202B40F014
:2032E000828000F592756FF046012846FFF76CFD6FF0460104F16000FFF766FD94F83D310F
:203300006FF3C30384F83D3194F879306FF3C30384F87930238A23F001031B051B0D43F4D6
:2033200040532382637D13F0600F05D004F115012046FFF74AFB39E0B4F81770B4F8191061
:20334000B4F81B200FFA87FE94F816C008B216B2BCF10C0F26D80FF2080858F82CF000BF12
:20336000953300084F340008A5330008A7340008A533000845350008893500088935000841
:2033800091350008AF3500082D3300082D330008AD330008207C460704D5022A02D11E06D6
:2033A00000D517B3237C43F001032374237CDB0716D594F8783028468C495B015A5842F4DA
:2033C00000125A5094F8793043F0080384F87930FFF728FF237C43F001032374FFF7C2FC5B
:2033E0000023A4F85E30BDE8F08103F01F03012B2AD0022B0CD0002BD4D10029D2D1C0F3D7
:203400000013C0F34000A17740EA4300607715E001F07F03062BC5D8C3EBC3030F064FF04C
:2034200002024FEA83034CBF603303F5927323445B7EC3F3C00363770023A37704F11D014B
:203440002046FFF7C3FDB1E76777A777F6E7207C4607A7D5002AA5D103F01F03022B17D1B0
:20346000002F7FF463AF01F07F0006283FF65EAFC0EBC0000E064FEA80004CBF603000F5F0
:2034800092702044FFF72EFB2046FFF7ADFD8DE7002B7FF44BAF012F7FF448AF034662F35D
:2034A00004132374F0E7267C70077FF57BAF002A7FF478AF03F01F03022B12D1002F3DD1AA
:2034C00001F07F00062839D8C0EBC0000E064FEA80004CBF603000F592702044FFF7CCFE4F
:2034E000D2E75BBB012F03D146F010062674CBE7022F23D1CBB20BBB090AA37C0139042960
:2035000014D8DFE801F0030B0D0F1100012262F30303A374237C43F02003C2E70222F6E798
:203520000322F4E70422F2E70522F0E76FF30303A374237C43F001032374EBE731077FF524
:2035400031AFF3E6DA067FF42DAF50EA06037FF429AF7F2F3FF626AF637C03F00F03022B2C
:203560003FF420AF224AE17DD2F8003823F4FE6343EA0113C2F800381E4B228A134009B1B0
:2035800043F4827323827FE7DB067FF40BAFCDE6217C4F077FF506AFDE067FF403AF5EEAC6
:2035A00000037FF4FFAE012A7FF4FCAEBEE6227C51077FF5F7AEDA067FF4F4AE50EA0603B5
:2035C0007FF4F0AE04F115012046FFF7FEF900287FF4ECAE218AFFB2074A0A401FB142F44A
:2035E00002722282E2E642F48072FAE70009084000000840FBF0FFFFF7F0FFFF2DE9F04F26
:2036000085B0DFF8B0B2DBF81440DBF8182042F4403343F440732340144023F0E96323F44A
:20362000E02323F47D7323F00103CBF8143000F0AB8025030FD5DBF81868DBF81C381E4063
:20364000360C40F0AC80DBF81838FF21984A1B0C002B40F09D80660312D5964BD3F818589C
:20366000D3F81C281540AAB20192002A40F02C81D3F81838FF21904A9BB2002B40F01281A0
:20368000002C12DA8B4A01218C4DD2F80438284623F00103C2F80438FDF73AFBE86820B177
:2036A000026852690AB12946904721050AD58349C86818B103681B6903B1984700217F48B0
:2036C000FDF726FBE20659D57A4B1D6A05F00F09B9F1060F52DC05F4F012B2F5002F00F0B8
:2036E0009681B2F5402F00F0A081B2F5802F45D1C5F30A15002D41D0DFF8C0811C2606FBB0
:203700000986D6F83471002F40F06C8196F83CA1BAF1000F40F06281D6F830717B7C03F0CA
:20372000F003102B40F05A81402DAB4607F11D00A8BF4FF0400B1FFA8BF10191FFF7F6FADF
:20374000A5EB0B00FFF7E4FA96F83D31022238466AF3820386F83D317B7C62F307137B7439
:203760000199A7F85E10FFF7B3FD1C2303FB098898F83D316FF3820388F83D31504B1C4262
:2037800000F06981FFF7DAFC002005B0BDE8F08FD80701D5106811605B08203258E70027D1
:2037A000464DF30741D5424B4FEA471959F80320DBF8143802EA030818F0010F1FD001238B
:2037C0003B4A17F0FF0A49F802306B7C42D103F0F003602B13D1D5F834215ABB95F83D3160
:2037E00062F3820385F83D3195F83D3113F0040105D1FFF7B7FA6B7C61F307136B7418F048
:20380000020F03D002232A4A49F8023018F0080F0BD06B7C03F0F003202B02D12846FFF76F
:2038200057FD0823224A49F80230760807F10107B7D110E751462348FFF7A9F895F83D3199
:2038400020496AF38203A1F5927085F83D31FFF71DFAC9E703F00F03022BD0D11C2000FBD3
:203860000AF005EB000ADAF834210AF59C7A32B99AF8053062F382038AF80530BFE700F53A
:203880009270002128440190FFF781F89AF8053001986FF38203014628468AF80530FFF7F0
:2038A000F5F9ACE7DD0700D511605B082032E4E6080B08400000084008090840C80D0024E9
:2038C00000108000EC0E0024DFF8C8814FF00009DFF8C4A1A8F16005019BD8076DD56B4A26
:2038E0004FEA491BD2F81038D2F8346801225BF80A7002FA09F23242029218BF43F0800337
:203900001F4017F00103039338D0029B5FFA89F21C2126EA03065D4B01FB0251C3F834688A
:20392000012360314BF80A306B7C002A4ED103F0F003502B0DD12846FFF75AFB95F87930F7
:2039400013F0040105D1FFF70DFA6B7C61F307136B742A7C910611D54C486FF34512AB7CC1
:20396000D0F8041803F00F0E6FF3030301F0700141EA0E11C0F804182A74AB743A0702D596
:2039800008234BF80A30FB0606D541462846FFF72FFB10234BF80A3038060ED5039B4BB91B
:2039A000029B4146284626EA0306384BC3F83468FFF71EFB80234BF80A30019B09F10109B3
:2039C00008F11C085B08019386D159E603F00F03022BD3D12846FFF70BFBCFE72846FFF7E3
:2039E00097F9C2E63889FE883B68361A1844AE42A8BF2E461FFA86F84146FFF797F9A81BC7
:203A0000FFF786F939898844A7F80880B6E6204A527C02F0F002102A7FF4B0AED3F8002BC3
:203A200042F08062C3F8002BA8E6194D082105F11500FFF77BF995F91530002B08DBB5F86C
:203A40001B302BB16B7C012262F307136B7495E66B7C0222F8E7A3047FF5D3AD0B4AD2F8C8
:203A6000003923F4FF6323F0070343F04003C2F80039D2F8043843F48073C2F80438D368AD
:203A800023F4705343F4C053D360BAE500000840C80D0024280E00240809084038B50B4CF8
:203AA000E060214603681B689847054618B10023E360284638BD7520FCF76CFF012120463A
:203AC000FFF78EF802232372F3E700BFC80D002470B50446EFF3118580260023EFF31083F9
:203AE00072B686F3118883F31088FFF727FBEDB285F311880E4D2046236829465B68984759
:203B0000EFF311840023EFF3108372B686F3118883F310887520E4B2FCF728FF002128467A
:203B2000FFF75EF80846E96084F3118870BD00BFC80D002470B52B4DE86808B1FFF7C8FF4A
:203B4000EFF3118600238022EFF3108372B682F3118883F3108800212248FFF741F875201F
:203B60000C462972FCF702FF752021462246FDF78BF91D4BFF204FF0FF32F6B2C3F808091D
:203B8000C3F8080BC3F82809C3F8280BC3F84809C3F8480BC3F86809C3F8680BC3F88809BD
:203BA000C3F8880BC3F8A809C3F8A80BC3F8C809C3F8C80B4FF48060C3F81048C3F8144876
:203BC000C3F83448C3F81C48C3F81828FFF7EAF8FFF7D8F86B7C64F303036B7486F31188C1
:203BE00070BD00BFC80D0024000008408F4AF8B5D2F80C3823F0007343F08073C2F80C385A
:203C0000D2F80C385901FBD58948402700F05AF9884800F057F9884800F054F9874EFFF709
:203C200089FF874B4FF4F47200211846FDF71DF88449024603464FF01C0C42F8601B014638
:203C40004260FE22C274027500220CFB02141C335E64196504F1780594F8794044F0100428
:203C60006C70D4B2013283F85C4064F07F04072A83F848406C786FF301046C70A3F84A7011
:203C8000E3D100231C274025DAB2C0F82461C0F830111C3080F8202180F80C2107FB031222
:203CA000013392F83D41072B6FF3010482F83D41A0F80E51E8D1002263497520FDF7E4F854
:203CC000002803DABDE8F840FFF734BF5F4C80235F4DA360E36843F04003E3600320FCF702
:203CE0001CFD2369002B01DB013DF7D1236943F001032361564B554C2269D20701D5013B13
:203D0000FAD103200025FCF708FDA36B142043F48033A36300F0AAF82368322043F0C00301
:203D20002360E36823F0005343F08043E36000F09DF8C4F8005ED4F800384FF4806023F439
:203D4000C053C4F80038D4F8003843F00303C4F8003840F20123636203F59203A362493302
:203D6000C4F804314933C4F808314933C4F80C314933C4F810314933C4F814314933C4F83E
:203D80001831FFF70FF8FEF7FDFF4FF0FF33C4F81058FF21C4F814582E4AC4F83458C4F893
:203DA00018382D4BC4F81C58186820330028B4BF4FF00840002043F8200C43F8105C43F8AD
:203DC000181C9342F0D1254B0022FF2024491C682033002CB4BF4FF00844002443F8204C2F
:203DE00043F8102C43F8180C8B42F0D1174B14489A614FF0FF325A6059691A4A21F07F4185
:203E000021F47C0121F47C4121F0FF010A4300215A61154A9A6181229A60FEF7E1FEFFF743
:203E20008DF97520BDE8F840FCF7B4BD004002580BAC08000CAC08000AAE0900D4A10008CF
:203E4000C80D0024B8A10008FD35000800000840400D0300E009084000090840000B084061
:203E6000E00B08400AFCB0F810380C0082B0002245F261610092009B834201D302B0704791
:203E80000192019B8B4203D9009B01330093F2E7019B01330193F4E702064FEA10130CD48C
:203EA00003F00F03064A52F8232032B100F00F00012319B103FA00F0906170471030F9E79B
:203EC000F0A100082DE9F04705090446C0F3031715F0080540F0D2806A4B53F82760002E8E
:203EE00000F0CC8000F4402300F00F08B3F5002F00F0B180B3F5402F00F0AF80B3F5802FA3
:203F000040F0AD80C0F30021FFF7C6FF0121EFF3118200238020EFF3108372B680F31188B2
:203F200083F31088022940F09C8014F4704FC4F3033017D023074FF00F094BBFA8F1080335
:203F400043464FF0240C4FF0200C9B005CF806E009FA03F900FA03F32EEA090E43EA0E03CD
:203F60004CF806304FEA48090323D6F800E0032903FA09F32EEA030E6FEA030C01FA09F3BC
:203F800043EA0E0333606ED004F44033B3F5803F6BD0B3F5003F0CBF02230023D6F80CE051
:203FA00003FA09F30CEA0E0E43EA0E03F36080B923074FF00F0A4BBFA8F10803434624202F
:203FC00020209B0050F806E00AFA03F32EEA0303835101F1FF3EBEF1010F0DD804F440657C
:203FE000B5F5006F43D0B5F5406F42D0A5F5806ADAF1000545EB0A05B36805FA09F501205E
:20400000BEF1010F0CEA030C00FA08F045EA0C05B56073682FD8A5052DD5034301297360C4
:2040200013D0E30511D504F00C044FEA88030F2004F1B04403F00C03D4F8081498409F404E
:2040400021EA00010F43C4F80874D2B282F311880020BDE8F087022159E7032157E72946C8
:2040600055E700207EE7002398E7012396E70225C2E70325C0E723EA0003CFE76FF0150063
:20408000E7E700BFF0A10008C0B2FFF71BBFFFEC02064FEA101310D403F00F03084A52F8E4
:2040A000233053B11A6900F00F00012303FA00F0104214BF1846002070470020704700BF26
:2040C000F0A100080A460146034808B500F052F8024B186008BD00BF10A20008B00F002488
:2040E000024B0146186800F0C7B800BFB00F0024024B0146186800F01BB900BFB00F002421
:20410000024B0146186800F070B900BFB00F0024F8B50D460446164600F05AF805F11F03D0
:204120006168AA19082523F00F03012622F00F02A3F11007D01B01441038C4E9011743F834
:20414000105CA1684E60A3F1080143F8080CA2F108004D60E060204642F8085C53F8083C35
:20416000E2683343536000F05FF82046BDE8F84000F052B801F10F03A2F5A27223F00F0374
:2041800070B5541818464FF4A27200211D46E41A03F5A276FCF769FD034600F1200200F59D
:2041A000A071A2F110009A6110321033D8618A42F7D1284600F007F8284622463146FFF75E
:2041C000A7FF284670BD0122002100F099B9FFEC104B37B51C6805464CB101A900F0AAF9DD
:2041E00001980028D4BF0020012003B030BD04F049FA00280CDB284604F068F9002801DB7D
:204200000120F2E700F0FEF80368002BF3DCF7E72046EAE704040024024B1B680BB904F090
:20422000A1B970470404002438B5054608680C4600F015F8421C05EB021205EB0015AB69CF
:2042400023B1196811B12068814205D39460C4E9023203B1DC6038BD1A469B68F0E7B0F58B
:20426000800F07D203090020012B00D8704701305B08F9E71220704770B505460C46A9B176
:20428000FFF7A6FF98B9EFF3118300228021EFF3108272B681F3118882F31088D5F8402115
:2042A000DBB22260C5F8404183F3118870BD54F8043CA4F1080123F0010344F8043C54F86C
:2042C000083CCA185068C60713D4CB58D2E902061344B06008B1D668C660126854F8080C08
:2042E000104444F8080C5A6802F0010202435A601A4654F8043CCB1A5868C00710D4D3E96C
:204300000210816009B1D868C860196854F8080C08441860516801F00101014351601946E3
:204320002846FFF781FF2846BDE87040FFF774BFF8B506460F46EFF3118300228021EFF344
:20434000108272B681F3118882F310880022D0F84041DBB2C0F8402183F31188002C39D133
:20436000002F35D007F1170525F00F05AF422FD83046FFF72DFFB5F5800F32D22846FFF79B
:204380006EFF06EB00108469FCB12268A368AA4229D3E26893600BB1E268DA602368581B1D
:2043A0000F280CD92344611960514D6025605A6802F00102024330465A60FFF735FF6368FC
:2043C000083443F0010344F8043C3046FFF724FF2046F8BD2568214630462C46FFF74CFF27
:2043E000BCE71220CDE71C46CEE713B50191FFF79FFF044618B1019A0021FCF736FC2046D5
:2044000002B010BD08B500F099FA08B1143008BD0048FCE7B40F0024002303600B6813B944
:204420000860486070474B681860FAE70B6802468BB180B1834208D11A680A604A689A4269
:2044400009D100234B6070472BB118461B689342FAD100F00BB8704703682BB11A6802600B
:2044600002B9426000221A60184670470A68036852B14BB14A689A424FF0000215BF19682E
:204480004860016002601A6018467047002303604B6843600A6812B90860486070471860CA
:2044A000FBE7002343600B68036013B9C1E900007047586008607047D0E9003232B90B6039
:2044C00033B94A600023C0E9003370471360F7E75A60F7E707B504460191009200F03AFA59
:2044E000DDE90010A047FCF7BDFB30B1B2F5004F03D212B20280002070476FF01500704760
:2045000008B530B1B2F5004F03D212B20280002008BDFFF777FF162303604FF0FF30F7E7B3
:2045200028B121B1038800201BB20B6070476FF01500704710B5FFF7F3FF041E05DA6442B7
:20454000FFF760FF04604FF0FF34204610BD1F299FBF012303FA01F103680B439ABF0360CF
:2045600000206FF0150070471F299FBF012303FA01F103688B439ABF036000206FF01500AE
:20458000704700230360184670471F299DBF0068C84000F001006FF0150070470FB41FB502
:2045A00006AB53F8041B0191039303F01BFF039A5030019900F079F805B05DF804EB04B0E6
:2045C000704770B5044630B300F0D4F80121201D002600F022F8012104F1500000F01DF81B
:2045E000012104F19C0000F018F8D4F8E85025B9204600F0C7F8304670BDB5F844309B07AB
:2046000007D50121284600F008F836EA200628BF06462D68EBE70646EDE7F8B5436805469B
:204620000F46002B3EDBB0F844309B073AD500F0BCF86C69FCB1EE69B44207D1284600F06B
:20464000D3F8EC696969641A2046F8BD2B6A9C4226D1361B32462146686803F0F5FB00285A
:204660000DDA95F8463043F0020385F84630FFF7C9FE04686442284600F0B6F8E4E7044437
:20468000361A0FB1002EE5DC6B692644EB61B442D4D0EB695A1CEA6114F8012B1A70F6E743
:2046A0000024E8E76FF00804CEE730B589B004460D46014603A8019200F0C6F8204600F0A3
:2046C00074F82946019A03A800F066F90546204600F08AF8284609B030BD08B5FDF7B6FAD2
:2046E000002803DABDE80840FFF78CBE08BD38B50122044600212C30FFF702FF4FF0FF3582
:20470000002304F130006563C4E9453300F03CF804F17C00C4F8805000F036F804F1C80068
:20472000C4F8CC50BDE8384000F02EB838B504462C30FDF78BFA0023C4F81831D4F8145149
:204740006DB904F13800FFF7C8FF04F18400FFF7C4FF04F1D000BDE83840FFF7BEBF284654
:2047600050F8083BC4F81431FFF7B7FF2846FFF7B7FCE3E710B50446204603F0A7FE0028EB
:20478000FADB10BD03F0EEBE08B500214FF0FF330122083001814360FFF7B2FE002803DA5E
:2047A000BDE80840FFF72EBE08BD70B5044603F0A5FF0546E368984212D004F10806304694
:2047C00003F084FE031E07DAFFF71CFE0368042BF5D08C2BF3D05B422BB90123E56001E0AE
:2047E000238A0133238270BD10B5044603F086FF238A012B0ED1002304F1080023824FF0C3
:20480000FF33E36003F0AEFE002805DABDE81040FFF7F8BD013B238210BD01210069FFF7AE
:20482000FCBE38B504460D462169284600F0B6FD013003D0E3680133E36038BDFFF7E2FD09
:204840000368042BF0D0F8E7094B03604B6963B1B1F84430074A13F4807F074B18BF1346AA
:2048600083600023C0E903317047034BF8E700BF234800081B480008DB530008421E11F835
:20488000013B02F8013F002BF9D17047034610B592B10A44084604460130904203D10022C6
:2048A00020461A7009E010F8014C03F8014B002CF1D1401A013810BD084610F8013B002B78
:2048C000FBD1F6E703461A46013311780029FAD1101A704710B5024404464B1E904208D08C
:2048E00013F8011F00F8011B0029F7D1121AFCF7BCF9204610BDFFEC0E4B002230B5D3E97A
:2049000000548C4209D1C561836823F4805323F00F0319438160002030BDA94202D1C16151
:204920002146F1E7013208331F2AE8D1C1614FF48051E9E718A20008C06970471FB500202C
:2049400001A903F069FD0028ACBF0298002005B05DF804FB2DE9F0410A4D2B6843B90A4C7B
:204960000A4E0B4FDFF82C80B44203D101232B60BDE8F08154F8043BBB42F5D34345F3D2D6
:204980009847F1E7B80F0024B8A50008B8A5000800000008B8A5000807B5009200220B467D
:2049A000114600F003F803B05DF804FB2DE9F04F8FB005460026DDF8609093F800A0BAF10E
:2049C000000F00F0EF83BAF1250F08D0013302932B68514628460136CB46984725E193F896
:2049E00001A09A1CBAF1250F0292F1D04FF000080A22474644463F2C4CD8BAF12B0F3ED020
:204A000013D8BAF1200F3CD0BAF1230F3FD0AAF13003DBB2092B4FD8E0054EBF02FB0838F4
:204A200044F0800402FB073707E0BAF12D0F2BD0BAF1300FEBD144F00104029B13F801AB87
:204A40000293BAF1000FD6D1AAF14503022B72D80AF1200A44F400545FFA8AFA14F4807F71
:204A600008BF4FF00608BAF1650F5FFA88F140F08280013144F48044C9B2002283E044F09D
:204A8000020444F00404D8E744F00804D5E744F01004D2E7B4F5007FB9D3BAF17A0F2AD036
:204AA000BAF1740F27D0BAF16A0F21D124F48064A4B244F42064C0E7BAF12A0F0FD1E0055D
:204AC00059F8043B02D523EAE378B6E7002BA7BF44F080041F465F4244F08804ADE7BAF11C
:204AE0002E0FDAD1E00500F15D8344F48074A4E7BAF16C0F09D1A30548BF44F4006424F4FE
:204B00008064A4B244F4007497E7BAF1680F09D1600548BF44F4006424F40074A4B244F413
:204B200080648AE7BAF1700F02BF24F42064A4B244F4007488E7AAF16503022B8ED9BAF1E6
:204B4000630F00F0A8810AF0DF03532B40F0C981CB469D4B5BF8049BB9F1000F08BF9946AC
:204B600014F4807F484614BF41464FF0FF3100F036FC804698E1BAF1660F7FF47EAF0A4666
:204B800044F400440F2109F107090F2908A829F0070B28BF0F21BBEC020B00F035FB9DF8CC
:204BA000243003F00902012A42D0A20743D414F0040F0CBF4FF000094FF0200913F00C0FF6
:204BC00043D0B9F1000F14BF04230323BB420CDA2107A7EB030709D4B8462B682021284625
:204BE0009847B8F10108F8D13E440027B9F1000F04D02B6849462846013698479DF8243096
:204C000004F40054714A13F0080F714B0CBF90469846A6EB080909EB080618F8011B69B946
:204C20003C46002C40F0B8823E44D946029BC4E64FF02D09C2E74FF02B09BFE70CB1203927
:204C4000C9B22B6828469847E5E7C3B2DDF820A00193604B019A1C421BD1134608A90433BE
:204C60000B44019919B113F8011930292CD01AF1040F2EDB92452CDABAF1000F44F40044CD
:204C800002DB019B9A4528DA0AF10108019BA3EB080823B2002B0393B6BF2AEAEA730523D8
:204CA0000133B9F1000F00D00133B8F1000F17D008F101021344BB42B4BFFF1A002714F05D
:204CC000090F1CD13B4615E00199481EC1B20191C7E7019B03F1FF38DBE74FF00008D8E717
:204CE000E20648BF0133E6E72021284604939047049B013B2A68002BF6D13E441F46B9F1B7
:204D0000000F04D02B68494628460136984723070CD4B94604E009F1FF393021284698474D
:204D20002B68B9F1000FF6D13E444F46039B002B52DA2AEAEA79C8F10003AAEB09020493EA
:204D4000019B09F1FF3904999A4237BF08AB4FF03008D31893F80580731C894503932B686B
:204D60001CDAE40606D5B9F1FF3F03D12E2128469847039ECA450BD19DF82530352B20D852
:204D800006D19DF8243013F0100F08BF4FF0310801362B6841462846984741E74146284637
:204DA00005929847B9F1FF3F059A07D1B31C2E212846059203932B689847059A0132039E80
:204DC000BEE74FF03108E3E718A3000810A3000814A3000800C0FFFF9DF82510284631295F
:204DE0001EBF9DF8243023F010038DF824302B689847B8F1000F2B683DDD02364FF0010996
:204E00002E2128469847C8452B6821DA14F4005F2B68284614BF452165219847BAF1000F9B
:204E200004DB31D19DF82430D9062DD5CAF1000A2D212B68284698473021BAF1090F25DCBF
:204E40002B682846984704362B680AF13001A2E7019A284601364A4588BF09F1380209F1AC
:204E6000010994BF30216A445FFA89F988BF12F8131C9847C7E7E00601D40136C6E72E2100
:204E8000284602369847C1E72B21D2E70131AAF10A0AC9B2D1E7CB464FF001080DF120094C
:204EA0005BF8043B8DF8203022070FD509EB08044C450DD14644B3E6013F2B68202128466A
:204EC00098474745A4EB0706F6D8EFE7BC19F8E72B68284619F8011B9847002FE8D0013F3F
:204EE000E6E7BAF1640F04F4206302D0BAF1690F78D1B3F5206F63D109F1070929F0070970
:204F0000CB46D9F804105BF8080B24F48059002929F0100906DA404249F4805961EB4101E3
:204F20001FFA89F919F4807F06D0B8F1000F03D150EA010300F0C28008AC0A23224600F0BF
:204F400035F9041BE4B219F4807F019400F0B88029F0010A44451FFA8AFA80F2B48044F27F
:204F600010025FFA88F309EA0202102A03D129F011091FFA89FA1AF0100F00F0AE8004F13B
:204F800038026A4412F8192C302A40F09E802AF4C04A2AF0100A1FFA8AFA1AF0080F40F0E8
:204FA000AD801AF0010F06D0BB4280F2C480FB1A03EB0408FBB2A3EB06095FFA89F998E075
:204FC000CB46A3055BF8040B4FEAE0719DD462059BD5230555BF40F3C03140F3C01100B2CE
:204FE00040B292E7B3F5206F1DD109F1070929F00709CB46D9F804105BF8080B24F006096F
:20500000BAF1580F1FFA89F945D0AAF16F03DAB2092A47D8092B45D8DFE803F04E254444DD
:20502000444415444436A10509F1040BD9F8000001D50021E2E714F48061DFD0220554BF03
:2050400080B2C0B2F5E724F016040A231FFA84F919F4807F05D0B8F1000F02D150EA010236
:205060002CD008AC6AE7029B1B78562B0AD1029B0133029343681A68079201682846FFF7AA
:205080008BFCD2E549F0100919F0100F01D049F480491023DCE7E30601D549F4C0494FF443
:2050A0000473D5E72B6828462521023698472B68514628469847B8E50823C9E7444642E7BD
:2050C0002346CA4657E7234655E71AF4804F01D1013300E00233DBB25FE741F206021AEA6A
:2050E000020F3FF45AAFF3E72B68202128460136984709EB0603DBB2BB42F5DBBB42B4BF6A
:20510000FF1A00271AF0100F22D02B683021284698471AF4804F10D10136C146A14529DC1C
:20512000A8EB0400A045B8BF002006444CBB019B33441E4674E5A0463DE71AF4005F06F1CD
:2051400002062B6814BF5821782128469847E4E741F206031AEA030FDFD01AF0020F06F1A4
:2051600001062B6814BF2B2120211AF4805F18BF2D21EAE72B683021284609F1FF399847EF
:20518000CCE7631E0EAA284652FA83F2DCB22B6812F8181C9847C9E72B6820212846013C87
:2051A00098473EE530460FB0BDE8F08F2DE9F84313F400791C4606460F461CBF23F400745A
:2051C0004FF0010915464FEAE478304639462246434604F085F8092AB4463B4606460F46F0
:2051E00009DC3032A44505F8012B73EB0803ECD22846BDE8F883B9F1000F01D03732F1E7D6
:205200005732EFE7FFECC2922DE9F74F10EE904A07460E4614F000441CBFB1EE400B0124E9
:20522000B5EE400BF1EE10FA11D121EAE1720530302144F00204FBF718FD0025BB19002275
:2052400030465A713C713D6003B0BDE8F08FB4EE400BF1EE10FA02D744F00804EDE7B0EE8B
:20526000C07B9FED436BB4EE467BF1EE10FA02DD44F00404E1E79FED406BB4EEC60BF1EE01
:2052800010FA5DD5404908230F2501209FED3C6B91ED107B20EE077BB4EEC67BF1EE10FA31
:2052A00005D500FA03FCB0EE470BA5EB0C05013B0839B3F1FF3FEBD132B125EAE5730133F1
:2052C0001A449642A8BF1646304B03EBC60393ED007B30EE070B9FED2A7BB4EEC70BF1EEF4
:2052E00010FA04DBB2EE047B013580EE070B07F10508DFF8A0A0DFF8A0B051EC100B04F061
:2053000007F86FF0040389460090DB1B0193019B43449E4292DD52465B460098494603F07A
:20532000DFFF00F1300C59465046009299460A22002308F801CB03F0D3FF82468B46E6E776
:20534000134908230F25012091ED107B20EE077BB4EEC67BF1EE10FA04DB00FA03FCB0EE96
:20536000470B6544013B0839B3F1FF3FECD1A3E7FFFFFFFFFFFFEF7F00003426F56B0C431B
:205380000080E03779C34143E8A3000820A30008A0A300080080C6A47E8D030037B50A46D9
:2053A0008DF8070004460D460DF10700012100F022F8002804DC4FF0FF34204603B030BD13
:2053C0000A2CFAD195F846305B07F6D501212846FFF723F90028F0DAEDE700207047024615
:2053E000014410B58A42134603D01C780132002CF8D1181A10BD2DE9F84380460F46164628
:2054000042B9FEF7FFFF4FF0FF34092303602046BDE8F883B2F844309B0706D4FEF7F2FF97
:20542000092303604FF0FF3418E053693BB90A460146706802F008FD041EE8DAF2E710464A
:20544000FFF7B3F9304600F04EF800280DDA4FF0FF343046FFF7C8F9002CD8DA96F846306E
:2054600043F0020386F84630D1E7D6E906502D1A202D01D11F2F1CD8BD42414628BF3D469B
:205480002A46A7EB0509FBF7DBFAF369B26908EB05042B449342F36104D2B9F11F0F14D98F
:2054A0004F4607E000213046FFF7B7F80028F4DACDE744463A462146706802F0C5FC002866
:2054C000C5DB0444A4EB0804C3E7B9F1000FF9D021464A46F06908EB0704FBF7B1FAF369D6
:2054E0004B44F361EEE710B5044630B9FEF78AFF092303604FF0FF3010BD4369F3B1FFF76E
:2055000054F9206A6269904213D0E36994F847101B1A2046C4E907220022591A84F847201C
:20552000012200F00DF8002803DA2046FFF75CF9E0E72046FFF758F90020DDE71846DBE725
:2055400000F000B870B504460D461646FFF7CBFF002802DA4FF0FF3070BD204600F010F8C8
:205560000028F7DB002332462946606884F8473002F04BFB01304FF0FF3018BF0020EBE7CC
:20558000426932B1B0F844309B0702D50121FFF744B800207047022901D100F063BB0129C8
:2055A00001D100F0C3BB704708B500F085FBBDE8084000F001BCFFEC38B50F4D04462B780C
:2055C00013F0FD0F09D1C20707D500F081FB002803DB0A4B02221A7004E02B78012B02D93A
:2055E0004FF0FF3038BDA307FAD500F0F1FB0028F6DB024B0122EEE7BD0F0024C4140024C9
:2056000010B5084C606004F00DF8FFF7D5FF002804DB054A13680133136010BD6368002BB3
:20562000F1D1FAE7C8140024C00F002408B5FFF7E7FFA0F120035842584108BD73B504461D
:2056400001AE00256420FFF7DBFF002807DB013506F8010B042DF5D1019B0020236002B0F0
:2056600070BDFFEC70B5094E04460D463378022B01D100F053FB3378012B05D1294620468F
:20568000BDE8704000F0BABB70BD00BFBD0F002410B5114C236801331DD062680F4B9A42A6
:2056A00019D90F4B9B6803F1006303F500339A4211D204F017F803F0E3FFFFF775FF03F025
:2056C000EDFF03F0B1FF204604F026F82046BDE8104004F0E7B810BD00000208FFFF0108F7
:2056E000AC00002410B500230B4C54F8232022B154F82320013A44F823200133042BF4D1C8
:20570000064B1B7833B9A36823B9022004F0ACF83223A36010BD00BFC8140024BC0F002445
:20572000024BD860DA68002AFCD17047C81400242DE9F04FAF4B8FB000250646DFF8BC82E0
:205740001D700395D8F8084003F086FFDFF8C0A20EB1CAF80060DFF8BC924FF0FF37CAF81E
:20576000085089F80050012004F06EF826B1DAF80030002B00F069820020FFF741FF0490BC
:20578000049B002BF2DB012004F04EF8049B213B1F2BE8D801A252F823F000BF1D580008D6
:2057A00033580008215900086757000867570008675700084359000867570008E1590008D6
:2057C0009F5A0008CD5A00080D5B00088F5B00082F5B00085D5B0008ED5B0008F75800083E
:2057E000675700086757000867570008675700086757000867570008675700086757000879
:205800006757000867570008675700086757000867570008675700089B5800080220FFF7D1
:2058200005FF002800F00682039B43F00103039361E04FF47A70FFF7E3FE051EC0F2FA81C4
:205840000220FFF7F3FE002800F0F481681E042800F2F081DFE800F0030B0E111400042180
:205860006548FFF7FFFE039B43F00203DFE704216248F6E704216248F3E704216148F0E7F2
:205880001C252846043503F068FF0421069006A8FFF7E8FE2C2DF4D1E5E701250220FFF759
:2058A000C5FE002800F0C681039B03F00303032B40F0C08101234FF0000B022089F800304F
:2058C00003F0B2FF03F019FF584603F02AFF044640BB022089F8000003F0B6FFD8F80830C7
:2058E000A34226D8039B002443F0040389F800400393CAF80840039B3E4A03F00303032B1B
:20590000137808BF002613B93F4B1B78137041F21203022106A8ADF81830FFF7A3FE22E7FD
:205920000025BBE7584629460BF1010B03F0FFFECAE7204603F011FF013040F05481043413
:20594000CCE73220FFF75CFE051EC0F2738115F0030240F06F812B19D8F808108B4200F214
:205960006981B5F5807F00F26581DFF8A0B05946AA4214D1C820FFF759FE002800F05A81FD
:2059800024B9224B4FF0FF321F681A6025F003052544AC4215D1039B43F0080347E74FF4A5
:2059A0007A70CDE90012FFF72BFE049004980028C0F2408104980099019A01F8010B013243
:2059C000D6E7DBF80010204603F0C1FE204603F0C4FE5BF8042B904240F005810434D8E7F3
:2059E0000220FFF723FE002800F024810025AB4642E000BFBD0F002448A40008AC00002406
:205A0000B0000024B4000024C4140024C4130024C8140024BC0F0024002D3BD1791C39D01D
:205A200006978B494A68C2B98C461346082003F0010E5B08BEF1000F07D083F06D4383F4E1
:205A4000380383F4034383F020030138EFD101324CF8043BB2F5807FE7D106A8002210F8D3
:205A6000013B013283EA0B03042ADBB251F8233083EA1B2BF3D10435D8F80830AB42CBD89D
:205A8000042106A8CDF818B0FFF7ECFD039B43F01003CCE6284603F060FE0690C1E7002311
:205AA00005A80593FFF7CAFD002840F0C3800220FFF7BCFD002800F0BD80059803F057FE3E
:205AC0000421069006A8FFF7CDFD14E7002305A80593FFF7B3FD002840F0AC800220FFF7F8
:205AE000A5FD002800F0A6800598820740F0A280082800F29F8003F08FFE0421069006A824
:205B0000FFF7B0FD039B43F0400390E60220FFF78DFD002800F08E8003F02CFE04210690B8
:205B200006A8FFF79FFD039B43F080037FE60220FFF77CFD00287DD006A9142003F020FE72
:205B400005460421059005A8FFF78CFD294606A8FFF788FD039B43F4807368E60220FFF74E
:205B600065FD002866D0142520223A4906A8FEF7B1FE04210DEB05000595FFF773FD294684
:205B800006A8FFF76FFD039B43F400734FE66420FFF736FD00284DDBC5B21E2D4AD8022075
:205BA000FFF744FD002845D04FF4D07003F0D5FD83464FF4D27003F0D0FD274B9B4539D1BF
:205BC000264B984236D1DFF898B04FF4D07045EA0B0B594603F0BBFD4FF4D07003F0BDFD12
:205BE00058453FF488AE41F2121392E64FF47A70FFF71CFDF0B17B1C0DD141F2120306A887
:205C00000221ADF81830FFF72DFD64200FB0BDE8F04FFFF785BD039B03F01B031B2B09D126
:205C20003946002003F093FD002003F096FD8742E3D0D8E741F21233022106A8ADF818302B
:205C4000FFF710FD002303938DE50FB0BDE8F08FC40F002430A40008FFECC2925D7D05C57D
:205C600000ECC29238B50F4B0F4C002808BF184603F0ACF90D49206003F0B8F90C4B00B1DB
:205C800018604FF0FF320B4D432118682A6002F06CF8002805DB28602068BDE83840FEF7D6
:205CA0001FBA38BD20A10008DC1400244CA40008D81400247400002410B5044C206801F00B
:205CC0002EFE4FF0FF33236010BD00BF7400002413B50F4C2368002B0FDA0E4B4321186881
:205CE00002F043F8002803DA4FF0FF3002B010BD094B20601868FEF7F3F901220DF1070127
:205D0000206802F06CF80128EED19DF80700EDE774000024D8140024DC140024024B0A46F4
:205D20000146186802F090B8740000241E4B70B5002808BF184688B003F048F91B490646D3
:205D400003F054F9054638B31849002003F04EF930B302F0F8FF04464321284602F005F83B
:205D6000031E13DB124D69462B6003F075F9029B2146684623F4B87343F030030293FEF736
:205D8000BBFD6A460021286803F06BF9304608B0BDE87040FEF7A4B94FF4E134054DDBE752
:205DA0004FF4E134D8E700BF20A100084CA40008780000244EA4000810B5044C206801F028
:205DC000AEFD4FF0FF33236010BD00BF78000024094B07B5186800280BDB01220DF1070135
:205DE00001F0FDFF012804D19DF8070003B05DF804FB4FF0FF30F9E778000024F8B5044634
:205E000046184FF47A75094FB44208D1F8BD01222146386802F018F8012804D0013D002D82
:205E2000F5D10134F0E74FF47A75FAE77800002403464FF604720846934210B513D04FF6CD
:205E40000C72934212D04FF60172934226D1FAF756FF002804461FDA6442FEF7D3FA04600C
:205E60004FF0FF3418E003F00DFEF2E70B78012B05D14C78012C05D0022C08D064B16FF01C
:205E80001504E9E74968807801F06CFAE1E74B680024186801F0DEFA204610BD6FF0180483
:205EA000DAE708B500F05CFDBDE8084000F012B8002070471046704708B54AB14B688A6833
:205EC00003F0050313438B6013B1086902F00CFB002008BD00234FF4DB720249024802F039
:205EE00052B900BF64A4000859A4000813B50446A36B204601919B6A984701990028F7D03E
:205F0000A36B20461B6A02B0BDE8104018472DE9F74F458C0446B0F9263088462DB24FF020
:205F2000800B01920135AB42D8BF0025A38C1BB2AB420AD0638C2DB2A26A00201BB202F8E0
:205F40000380658403B0BDE8F08F019B002B30D0EFF3118AEFF3108772B68BF3118887F388
:205F60001088A38C1BB2AB421ED1E27802F0FF09E2B90121A26B20466170526A904704F1D4
:205F80001A0002F06BFAA26B06464946526A204690475FFA8AFA8AF31188E37863B9002E17
:205FA000C4DA6FF00300CDE70026F2E76FF07F06EFE76FF00A00C5E76FF07F00C2E72DE9C2
:205FC000F74F836880460E4601925C6904F12C09484602F043FA051E12DB00254FF0010BB7
:205FE000019B9D4204D2E37873B10DB96FF07F05A36B204601219B699847484602F074FAC1
:20600000284603B0BDE8F08F238EE28D19B212B28A421ED0626B0133525C1BB2B4F9321067
:206020009942D8BF00232386E36813F4E07F05D00A2A07D113F0400F18BF0D22013506F804
:20604000012BCDE70D2AF9D113F4807F18BF0A22F4E7002DCCD1D8F80830002B49D0D8F895
:20606000005015F0400547D1EFF3118A8023EFF3108772B683F3118887F31088A26B294610
:2060800020465FFA8AFA92699047E18D228E09B212B2914225D1A26B01212046926990471E
:2060A000E18D228E09B212B2914202D08AF3118896E7E27892B904F11C0084F802B002F035
:2060C000CDF98AF31188002802DBE378002B87D0E378002B8AD16FF0030589E76FF07F006C
:2060E000EFE78AF31188A36B012120469B69984776E76FF050057BE76FF00A0578E72DE9E5
:20610000F04183685E6906F11805284602F0A6F9041E23DBF378002B36D13378013313F0EA
:20612000FF0734D0012F2DD1EFF3118800238022EFF3108372B682F3118883F31088337982
:206140005FFA88F86BB9B36B30461B689847041E07DA88F31188284602F0C6F92046BDE80B
:20616000F081B36B30469B689847041EB36B03DA5B6830469847ECE79B69012130469847B5
:2061800088F311883770E6E76FF07F04E3E76FF01704E0E7F7B50E4600F1400700F150050C
:2061A00057F8044B8CB16368A26843F0180333401343A3604BB101A92069FEF7B1F9019BAB
:2061C000002B02DC206902F08FF9AF42E8D103B0F0BD2DE9F84383680E4615465C6904F104
:2061E0001E08404602F03AF9071E4EDB002D4FD004F14002002352F8045B002D34D11033BC
:2062000004F1200944F8236004EB83034846736102F054F9638CB4F926201BB201339A42CC
:20622000D8BF0023A28C12B29A4225D1484604F12C0902F059F9484602F040F9E28D238E0B
:20624000484612B21BB29A421EBF736803F001031D4302F049F9E37893B145F018052946A0
:206260002046FFF797FF0DE00133042BC3D100236FF00F07736105E0756805F00405D5E760
:20628000002DECD1404602F02FF93846BDE8F8837369002BF6D01D607561F3E72DE9F0478F
:2062A000836880460F4616465D69464B1B6823B1EB78ABB16FF07F0425E002F09BF800287B
:2062C000F6D105F1200A504602F0C8F8041E1ADBEB7803F0FF018BB3504602F005F9E9E78E
:2062E000EFF3118400238022EFF3108372B682F3118883F3108807EB0608B84506D1E4B23F
:2063000084F3118834462046BDE8F0872B6917F8011BD80703D50D2905D11A0705D4284687
:20632000FFF7E4FDE9E70A29F9D113F0240F03D00D212846FFF7DAFD0A21F0E7D8F8002055
:20634000B146AB6B284682F040085B6AC8F380189847B9F1000F01D1344623E02B6917F866
:20636000011BD80703D50D290AD11A070AD442462846FFF7CCFD041E10DB09F1FF39E8E777
:206380000A29F4D113F0240F01D10A21EFE742460D212846FFF7BBFD041EF6DAB14501D26F
:2063A000A6EB09046A8CAB8C12B21BB29A4204D0AB6B012128465B6A9847504602F094F873
:2063C000A1E700BF040400242DE9F04700F1200804460E46404602F041F8051E1DDBEFF398
:2063E000118700238022EFF3108372B682F3118883F31088E37803F0FF0553B3638C6FF0E1
:206400007F05A384FFB287F311881E4F002DD7F800902CDA404602F067F82846BDE8F087AD
:20642000A36B0121204684F801A05B6A9847484602F014F8A36B054600215B6A20469847F5
:20644000002DDFDB628CA38C12B21BB29A42E7D1D8E74FF0010A04F11A09F3E74FF47A70EB
:2064600002F0D6F83B68A3EB0903B34206D2A36B2046DB6A98470028F0D0CBE76FF0730549
:20648000CBE700BFE41400244FF0FF332DE9F0418B6005460B790C462BB14B6943F00103E4
:2064A0004B6105230B610122002104F1200004F11A07FEF71AF80122002104F12C00FEF7CC
:2064C00014F80122002104F11800FEF70EF80022384604F11C061146FEF707F800223046CA
:2064E0001146FEF702F80122002104F11E00FDF7FCFF0021384602F0D1FB0021304602F02A
:20650000CDFB234628464FF4DB720249BDE8F04101F039BE84A4000810B504460121FFF7EC
:2065200039FEA3783BB1002304F11C00A370BDE8104001F0D9BF10BD10B504460421FFF761
:2065400029FE63783BB1002304F11A006370BDE8104001F0C9BF10BD70B583680E4615464E
:206560005C69A36B1B69F3B9B6F58D7F0DDAB6F58A7FC0F2B680A6F58A73052B00F2B180F3
:20658000DFE803F07995AFAF9CA6B6F5427F36D040F209339E424ED040F207339E420AD08F
:2065A0006FF0180089E0984710F1190FDCD0002800F0998081E0EFF3118100238022EFF39A
:2065C000108372B682F3118883F31088228EE38D12B21BB29A420ADCE38D228E1BB212B2C0
:2065E0009B1ACAB282F311882B60002065E0228EE08D12B2B4F9323000B2121AF0E7EFF3E5
:20660000118100238022EFF3108372B682F3118883F31088A28C638C12B21BB29A4203DC01
:20662000638CA28C1BB2DAE7A28C608C12B2B4F9263000B2E1E7EFF3118100238022EFF339
:20664000108372B682F3118883F31088628CA38C12B21BB29A4206DAA38C628C1BB212B24B
:206660009B1A013BBDE7628CA08C12B2B4F9263000B2121AF4E7EFF3118600238022EFF3CB
:20668000108372B682F3118883F3108835F0020301D1E38D2386013D012D04D8638C204671
:2066A000A384FFF749FFF6B286F311889DE742F210712046FFF788FE70B970BD002D02DA41
:2066C0006FF01500F9E7A368002BF9DAA5608CE74FF0FF33A36088E710F1190F3FF460AF97
:2066E000EBE76FF0180040F201139E420BD0B6F5817FE2D1002DE3D02B68E3606B682361E5
:20670000EB68636171E7002DDAD0E3682B6023696B606369EB6068E770B504460D46EFF3FC
:20672000118600238022EFF3108372B682F3118883F3108881F00103C37089B91821FFF72B
:2067400029FD637823B104F11A00657001F0CCFEA3782BB1002304F11C00A37001F0C4FED4
:20676000F6B286F3118870BD10B5044600211A3001F005FF002104F11C0001F000FF01217F
:2067800004F1200001F0FBFE012104F12C0001F0F6FE04F11E000121BDE8104001F0EFBE0A
:2067A00070B5836805465C6904F11806304601F085FE2378012B06D9013B2370304601F0E0
:2067C00093FE002070BD0021A36B204621709B6998472B685B0604D44FF47A612046FFF78C
:2067E000F3FDEFF3118500238022EFF3108372B682F3118883F31088A36B2046DB6898471D
:2068000023791BB9A36B20465B689847EDB285F311882046FFF780FE2046FFF7A5FFCDE7B4
:20682000436913F0010302D00A44914201D1002070478368002B04DD0B78032B03D01A2B49
:2068400003D00131F1E70A20704707207047F8B5002504462F46628CAEB2A38C12B21BB2FD
:206860009A4210D1628CA38C12B21BB29A4204D1A36B002120465B6A9847EEB12046BDE819
:20688000F840FFF759BEA36B20469B6A98470028E8D0A38C2046A16A1BB2A26BC95C126A60
:2068A0009047A38CB4F9262001331BB29A42A38400DCA7840135CEE7F8BD2DE9F341C58D98
:2068C0000026B0F9323004462DB237460135AB42D8BF0025A36B2046DB69984770B916B17B
:2068E0002046FFF719FE37B13946A06801F06EFE2046FFF739FF02B0BDE8F081B4F83080A1
:2069000001A9A36B20460FFA88F85B69984701228DF803000DF103012046FFF781FFA845B7
:206920000746D7D0E38D01369DF803101BB2626BB6B2D1542BB20135E385B4F93230AB4276
:20694000D8BF0025C6E7FFEC08B5044B186818B103689B6803B19847002008BD8000002404
:20696000002070477047C36B93F85430002B0CBF6FF07F0000207047704700207047C36BE5
:2069800093F85500032894BF00200120704770B5036806460D469B689847044660B1C580F0
:2069A0002846FDF7A5FB0546206028B9336821462C463046DB689847204670BD806890F81A
:2069C000543013B10121FFF7A7BE704700218068FFF7A2BE10B5836840F2093081425B693A
:2069E00000F0A38010DC40F2073081425ED0B1F5427F7ED040F20110814228D0B1F5817FE5
:206A00004BD06FF018000DE040F6025081420AD040F60350814213D040F601508142F0D198
:206A20005A66002010BD002A00F0A080D3F85A101160B3F85E10918093F860309371F0E7A9
:206A4000002A00F0938093F858301360E9E7002A00F08C80D9681160196951605969D160B5
:206A600093F85F10B9B101294FF480700CBF4FF400710021014393F85E0002280CBF402033
:206A800000200143104641F030019160D3F85A10FDF732FFC5E70846ECE7002A66D01168E9
:206AA000D96051681961D2685A61BAE7EFF3118000218024EFF3108172B684F3118881F37D
:206AC00010881C8ED98D24B209B28C4208DCD98D1B8E09B21BB2CB1AC1B281F31188B4E734
:206AE000198EDC8D09B2B3F9323024B2091B5B1AF2E7EFF3118000218024EFF3108172B6A2
:206B000084F3118881F310889C8C598C24B209B28C4203DC598C9B8C09B2DBE7998C5C8C78
:206B200009B2B3F9263024B2E0E7EFF3118000218024EFF3108172B684F3118881F310880C
:206B40005C8C998C24B209B28C4206DA998C5B8C09B21BB2CB1A013BBEE7598C9C8C09B2C7
:206B6000B3F9263024B2091B5B1AF4E76FF0150058E770B50D46044658B151B1086808B120
:206B8000FDF7AEFA236829462046DB68BDE87040184770BD10B590F85430044693B1002155
:206BA00080F85410FFF7B8FDA06E03685B689847E06E03685B689847206F0368BDE81040E9
:206BC0005B68184710BD70B50C468568EFF3118600238022EFF3108372B682F3118883F303
:206BE000108800212846FFF797FD2846FFF7D2FF0023F6B26B84AB8486F3118823685B6965
:206C000023B120460121BDE87040184770BD2DE9F04184680D46002C49D02046FFF7BAFF57
:206C20003220FDF723F9A16E29B12B6828465B6898470023A366616F21B16868FFF799FF3A
:206C400000236367264604F130074FF00008D6F8E41021B1206FFFF78CFFC6F8E4800C3660
:206C6000BE42F4D1216F29B12B6828465B68984700232367EFF3118600238022EFF31083E2
:206C800072B682F3118883F3108804F18808D4F8887077B9F6B286F31188E16E21B12B68C9
:206CA00028465B689847E76600236384A384BDE8F0814046FDF7D0FB41680029E7D0E06E14
:206CC000FFF757FF94F85530013B84F85530DEE72DE9F84F84680D46804621654B68402159
:206CE0009C606868FFF753FE6067002879D03E4B0122C36028462B6894F8AC101E68032385
:206D000041F08001B047A06630B96FF0120429464046FFF77CFF61E0846001222B682846B7
:206D200094F8B0101E68022341F08001B047E0660028EAD0846000222B68284694F8B41034
:206D40001E680223B04720670028DED004F1E00604F5887A4FF0000B8460B1464021206F49
:206D6000FFF715FE706000283BD0A6F808B006610C3656F8082C1D4B5645D360EED104F19C
:206D8000C0064FF0800A6021E06EFFF700FE706038B30661164A7368DA60EFF3118BEFF3AA
:206DA000108772B68AF3118887F3108804F188013046FDF731FB94F855205FFA8BF30132CD
:206DC00084F8552083F3118808364E45DBD12B685C691CB101212846A04700242046BDE86B
:206DE000F88F6FF00B0492E765690008B77100081973000837B50446154608461A4669469D
:206E0000002300F083FB23682A4669461B682046984703B030BDFFEC2DE9F34190F854308E
:206E200004460E468B4204D10025284602B0BDE8F081FFF7AFFE002EF6D0012E41D10022BD
:206E400004F19803A06E11460193FFF7D3FF051E33DBA26E0221019B94600022E06EFFF787
:206E6000C9FF051E29DBE26E3146019B94603246206FFFF7BFFF051E1FDB236F264604F101
:206E80003007DFF844809C60D6F8E410C1F80C80206F03681B699847054670B994F856303A
:206EA0000C360133BE4284F85630EDD10121204684F85410FFF730FCB7E72046FFF76AFEB0
:206EC000B3E76FF01505B0E7B77100082DE9F0410F461178D0F8088011F0600C5488D8F84A
:206EE00074509088D6887BD15378063B052B00F2CC80DFE803F003CA4139634AD378022B6C
:206F000024D0032B2BD0012B40F0BF802C6800F0F9FA00F11002234650F8041B904243F862
:206F2000041BF9D1028812201A80B0424FF001032946A8BF30462B71E880786803681B69BE
:206F40009847002809DA00236B8106E008F19801286800F011FB0028E7DABDE8F0812968A4
:206F6000907800F093FAF6E7002940F08E80E1B24046FFF751FFEEE7802940F086802B68A2
:206F800098F854201A700120CFE701297DD198F85430012B79D1D8F89C30984202D001330E
:206FA000984272D1002C70D14046FFF7F3FD98F854104046FFF730FF0020B6E7812964D1A0
:206FC00098F85430002B60D1D8F89C30984202D00133984256D1002C54D12B681C70D2E79B
:206FE000BCF1200F51D15278203A032A4DD8DFE802F014022D3DA12947D1D8F89C3098428C
:2070000043D1D8F85A2007202B681A60B8F85E209A8098F860209A7187E7212935D1072E88
:2070200033D1D8F89C2090422FD143B11A68C8F85A209A88A8F85E209B7988F86030D8F80A
:207040006430002BB8D000209847B5E721291CD1D8F89C30984218D104F00304D8F8643059
:2070600088F85840002BA7D00120EDE721290CD1D8F89C30984208D1D8F86430002B9BD0F1
:207080000220E1E76FF0200067E76FF05E0064E700230B81006F4968C388CB8003681B69DD
:2070A0001847FFEC2DE9F0470446EFF3118800238022EFF3108372B682F3118883F31088F6
:2070C00000F178094846FAF7A9FF94F85930002B44D004F1900AD4F890502DB95FFA88F8C9
:2070E00088F31188BDE8F0876A6800212B89106817891844B4F93220FF1AE38D0133BFB218
:207100009BB29342A8BF0023228E8EB212B293420DD116B12046FFF7FFF9B7421BD85046BF
:20712000FDF79AF929462046FFF7B2FFD3E7B742EFD9E68D10F801C00131626B36B202F8B4
:2071400006C01AB20133E2859BB2B4F932209342A8BF0023D8E72B891E442E81D4F8903047
:20716000002BBBD02346034AC821484601F0D4FAB4E700BFB371000810B5C06BEFF3118480
:2071800000238022EFF3108372B682F3118883F3108859B190F8593013B9012380F8593065
:2071A000FFF780FFE4B284F3118810BD80F85910F8E7FFF777BF38B584680869EFF3118539
:2071C00000238022EFF3108372B682F3118883F31088B1F90A3013F16E0F0CD08BB9038128
:2071E00004F19001FDF718F92046FFF75BFFEDB285F3118838BD94F85630013B84F8563059
:20720000F5E701462046FFF743FFF0E72DE9F74F0446EFF311834FF0800A01930023EFF358
:20722000108372B68AF3118883F31088D0F86C80B8F80630602B38BF60230093D4F8887079
:207240006FB3D7F804B0DBF80000EFF31189EFF3108572B68AF3118885F310880021B4F8A8
:2072600022C08EB2A28C0FFA8CFC12B2944502D0009BB3421AD8618CA28C09B212B29142CF
:2072800004D1A26B00212046526A904716B12046FFF752F95FFA89F989F31188C6B99DF880
:2072A000043083F3118803B0BDE8F08FA68CA26A36B2925D4254A28CB4F92660013212B2B1
:2072C0009642A28402DC4FF00003A3840131C6E704F18800FDF7C0F894F85520594640463B
:2072E000013A84F855200122ABF80660CBF810708BF80420D8F800201269904700289DD075
:20730000CDE741B1C06B428C838C12B21BB29A4201D0FFF77BBF704770B50D4684680869C5
:20732000EFF3118600238022EFF3108372B682F3118883F3108804F18801F6B2FDF76CF8D8
:2073400094F85530013384F8553086F31188B5F90A3023B92046BDE87040FFF757BF70BD1D
:207360007047FFEC2DE9F04F8FB0242280460F4605A80021F9F779FC04234FF0020A4FF092
:20738000010B0693032343F25420CDF810A0CDE9083BCDE90AA3FCF7ABFE044638B96FF072
:2073A0000B0507B13C6028460FB0BDE8F08F43F2482904AE002104F198054A46F9F755FC3C
:2073C00084F857800FCE0FC50FCE0FC596E80300C2231D4A85E8030084F85B300823102158
:2073E00084F85CB084F860304FF4167384F803B06846638604F58873636342F6E063E384CB
:2074000004F55A73A362114BC4E90E3404F5405383F84CA2C3F848220D4AC3F8504243460F
:2074200001F053FC21466846FFF72EF8051E04DA20460024FCF754FEB3E74C442046FCF788
:207440002DFB0546ADE700BFB4A40008CCA40008A4A4000830B585B085680B4A102195F824
:2074600057300446684601F030FC684600F0ABFE2046FCF72DFB05F17800FAF7CFFD28460F
:20748000FCF72EFE05B030BDA4A4000870B50C4604282BD8DFE800F01C2803242600154D8B
:2074A0002846FDF70FFA002322461946EE5C0133D170023298421670F8DC00284FEA4003AC
:2074C000D8BF0223981C0323C0B26370207006E0032304204B70092308708B70C87070BD52
:2074E000054DDDE7054DDBE7054DD9E76FF01500F5E700BF07A5000879A50008FCA40008BF
:2075000001A500080048704717A50008012810B512D002281FD068BB072305240B704C7064
:207520005269487162F07F028A700322CA7040220A710A228A710CE0072305240B704C7031
:20754000D26988718A700222CA7040220A7100224A71184610BD072305240B704C70926935
:20756000C87062F07F028A7040220A7100224A710122DFE70023ECE72DE9F0410D46044689
:20758000002800F087800021042624274FF003080846FFF7F1FF8023012102224FF0090E79
:2075A000A070E3710012FA23A671E0704FF0100CA672052084F800E0627022716171237211
:2075C00084F809E06B6884F815C04FF0060CE3720023A074E67584F81AC04FF0070CE076EC
:2075E00084F81E8023736173A273E27321746374E7742375A17527766276277761776F6866
:2076000084F820C00F4484F82100E7776F6984F823804FF00A0867F07F0784F8253084F84E
:20762000268084F82270402784F827E084F8247084F828606E6884F82A300E4484F82B20D3
:2076400084F82C8084F8296084F82D3084F82E3084F82F3084F830C084F83100EE6984F883
:20766000332084F8326084F8347084F8353084F8361084F837C084F83800A86960F07F00DF
:2076800084F8390084F83A2084F83B7084F83C3084F83D103E20BDE8F08110B514460846A6
:2076A000114601F0A7F9204610BD0846FBF76EB900F042B9F8B5837804460E468B4223D255
:2076C000CB00FF2B22D88900406801F09FF9074668B1A5788020FCF713FD47F8250070B94E
:2076E000013DA3789D4205DA3846FCF7F9FC6FF016000AE057F82500FCF7F2FCF0E701354C
:20770000B542E7D36760A6700020F8BD6FF01700FBE701220021FCF7E8BEF8B504468578DD
:20772000013D07D26068FCF7DBFC2046BDE8F840FAF781BAAF0070266368D8593044103E2E
:2077400000F01EFA16F1100FF6D16368D859FCF7C7FCE5E72DE9F84FDDF828A08846174691
:207760001D46064600F0D2FD814600F0A7FE041E3EDBBAF1000F514699F80230B8BF0AF17E
:207780000701C9108B428B4609DC01314846FFF791FF041E03DA484600F0A6FE28E0DAF14B
:2077A00000030AF00704D9F804C003F0070358BF5C425CF82B204FEA8B0102EB0412936818
:2077C0002001D3B9C2F8008004EBCB04D9F80420535803445F60D9F804305B5803449E6061
:2077E000D9F804305B5803444846DD6000F07CFE2046BDE8F88FD346DBE701341032082C3D
:20780000DDD10BF1010A99F8023000245345F2DC0BF102014846FFF74DFF041EBBDBD9F80E
:2078200004304FEACA0453F82A30C3F80080D9F8043053F82A305F60D9F8043053F82A301A
:207840009E60D9F8043053F82A30DD60A3E7F8B5002305460F460B6000F058FD0646F0B1AC
:20786000002D1FDB8378B5EBC30F1BDA00F026FE041E0FDB7368EA1005F0070553F822001C
:2078800000EB05153D60AB6833B12B4630463B6000F02AFE2046F8BD6FF00804F6E76FF0F3
:2078A0000A04F7E76FF00804F4E7F0B585B0044600F02CFD054600F001FE002814DB002CDC
:2078C0000DDBAB78B4EBC30F09DAE2106B6804F0070453F8220000EB0414A36833B92846B0
:2078E00000F002FE6FF0080005B0F0BD23466E4604F110071868083353F8041C3246BB420B
:2079000003C21646F6D1102200212046F9F7ADF9284600F0E9FD684600F032F9E4E710B593
:20792000FFF7C3FF041E05DA6442FCF76BFD04604FF0FF34204610BD00F05AB838B50F4C3A
:2079400000F0DCFE05466368984204D1238900200133238138BD204600F0B8FD002807DAEB
:20796000FCF750FD00680428F5D08C28F3D040420028EFD1012365602381EBE78400002486
:2079800008B500F0BBFE0A480389012B0CD1002303814FF0FF33436000F0E4FD002805DA07
:2079A000BDE80840FCF72EBD013B038108BD00BF8400002410B503460446184613F8012B23
:2079C0002AB9001B1C30FCF79BFB18B910BD2F2AF3D1F6E700F11803013C14F8012F12B9EC
:2079E00000221A70F2E72F2AFAD003F8012BF4E708B50348FFF7DEFF024B186008BD00BFB9
:207A000020A10008E014002400232DE9F04116461360027888B0002A45D08DF81C30CDE9D4
:207A2000010301A8CDE90333CDE9053300F04CF8002835DA019FDDE90354384600F036F8FB
:207A4000037880463846D3B1FFF7B4FF48B96FF00B04069808B1FCF743FB204608B0BDE880
:207A6000F0813DB16B68C0E900436860474604460025E2E7A368C0E90043A060F6E7FFF791
:207A800099FF0028E3D035B16B68C0E90043686000243060DDE7A368C0E90043A060F7E7B9
:207AA0006FF01004D5E76FF01504D6E7017803460246013031B12F29F8D113460132197807
:207AC0002F29FAD018467047F8B5036805461A782F2A08D0274A1430274901F0E9F86B697E
:207AE000002B41D02B60254B28681C6803782F2B3DD1002637464CB922466FF001032A615A
:207B0000C5E90004C5E902761846F8BD04F11701431E11F801CF13F8012FBCF1000F0FD15C
:207B20000AB12F2A17D1FFF7C1FF0378BBB1E38903F00F03032B14D0A368264600240BE0A3
:207B400022B12F2A02D0944505D3E2D900246FF001032246D3E7636827461C46CBE702467E
:207B6000CDE702460023CAE76FF00B03CCE76FF01503C9E720A1000840A50008E014002420
:207B800070B5866805467EB134691CB164680CB1A0470446304600F047FB0023C5E9003388
:207BA000C5E90233204670BD3446FBE770B5866804460B4615463EB136692EB136691EB10F
:207BC000B04700280DDA70BD012D05D0022D0AD025B16FF01500F6E762681344002BF8DB20
:207BE00063606068EFE76FF05700ECE71FB50C4603A90192FFF72BFE002804DB019A21460E
:207C00000398FFF7D3FF04B010BD10B5FFF7EEFF041E05DA6442FCF7F5FB04604FF0FF3478
:207C2000204610BDC38913F00F030FD003697BB1CA0701D59A6872B111F002000DD0DB684A
:207C4000002B14BF00206FF00C007047184670476FF0050070476FF00C0070472DE9F04745
:207C6000054688B09246984600295BD012F0060F4FF0000601A8019114BF109B4FF4DB79CB
:207C8000069618BFD3F800908DF81C60CDE90266CDE9046600F0B5FA041E19DB029F5146EA
:207CA0003846FFF7BFFF041E0DDB1AF4006FC5E900A6C5E9027610D00599284600F0BAF902
:207CC0000028044611DA00233846AB6000F0ACFA069868B1FCF704FA0AE0FB8903F00F03EA
:207CE000032B10D13B691C6834B90698A0B90024204608B0BDE8F08729EA080352460599B7
:207D00002846A047DCE7012B09D13B691B68002BEBD028469847D3E7FCF7E2F9E7E76FF036
:207D20000504D0E76FF01504E2E770B5044686B00D46164600F06EFF214603462A4602A8C7
:207D40000096FFF78BFF041E0CDB002304980093059BDDE90212FFF7FDFC041E02DA02A8A1
:207D6000FFF70EFF204606B070BD0EB417B505AA52F8041B0192FFF7D8FF041E05DA64420A
:207D8000FCF740FB04604FF0FF34204603B0BDE8104003B0704710B403688468DB0707D58E
:207DA0005CB123694BB19B683BB15DF8044B18476FF00C005DF8044B70476FF00800F9E72F
:207DC0001FB50C4603A90192FFF741FD002804DB019A21460398FFF7DEFF04B010BD10B54D
:207DE000FFF7EEFF041E05DA6442FCF70BFB04604FF0FF34204610BD10B40468A40708D53F
:207E000083685BB11B694BB1DB683BB15DF8044B18476FF00C005DF8044B70476FF008008C
:207E2000F9E71FB50C46019259B103A9FFF70FFD002804DB019A21460398FFF7DDFF04B0C7
:207E400010BD6FF01500FAE710B5FFF7EAFF041E05DA6442FCF7D6FA04604FF0FF342046B6
:207E600010BDB1F5417F08B5C36805D159681046FCF704FD002008BD6FF01800FBE770B5A3
:207E8000C56806460C462868002956D0212A54D9C38903F00F03032B0BD103690A4629463A
:207EA0005B6B9847002844DB736822200133736042E0A96800293ED021221831601CFCF74D
:207EC000E5FC00232370AB681A6932B1DB8903F00F03022B17D106232370AB689A680AB980
:207EE0001B690BB904232370FFF728FDAC686368AB6013B19A8901329A81FFF741FD2046AC
:207F000000F092F9D0E7072B01D10923E4E7032B01D10423E0E7012B01D10223DCE7042B31
:207F200001D10323D8E7052BD6D0062BD5D10723D2E7831C00D1002070BD6FF01500FBE7E7
:207F400070B5C468D4E90056EB8903F00F03032B0ED12B691B6BA3B12146284698470446CB
:207F6000284600F061F93046FCF7BAF8204670BDA06808B100F058F920460024FCF7B0F874
:207F8000EEE71C46ECE72DE9F04306468BB089461746002A48D1D0F80C804468D8F8005078
:207FA000EB8903F00F03032B20D1A1420CDA2B699B6B2BB96FF0850420460BB0BDE8F083C1
:207FC0003C464146284698472746B94504DC3C46002CF1DB7460EFE72B6901AA41462846A8
:207FE0005B6B9847041EE7DB0137EEE7A142BABFAD681446D8F80850FFF7A0FC0DB1A145C2
:208000000FD1D8F80870C8F8085015B1AB890133AB81FFF7B5FC002FDAD0384600F004F9DB
:20802000D6E701346D68E9E7012A0CBF44686FF01504C1E7F7B5856806460F46EB8903F046
:208040000F03032B19D12B6923B3DC6A14B35B6B03B301AA2846A047041E0BDB019B1D60E2
:20806000019D384600F0B2FF68600D48C6E9020500F0B7F8204603B0F0BD0C20FCF740F8B4
:20808000034650B1019000240560A868986000F0A8F8E5E76FF05704ECE76FF00B04E9E74D
:2080A00090000024C3685968FFF7C4BF2DE9F347061E8946144698465DDB12B900F0A6F99A
:2080C0000446022E18DD01A93046FFF7C0FB051E04DB019B986840B96FF00105B8F1000FAC
:2080E0003DD00023C8F8003039E04946FFF79AFD10B16FF00C05F1E7022EA76836DD4C2064
:20810000FBF7FEFF0446C8B307F12C0A504600F0A5F9051E03DA2046FBF7E2FFDEE7D7F88C
:20812000183103B31C605046C7F8184100F0DCF92046FCF729FB04F1240304F144026660B7
:2081400063612362A4F84490C4E906230C2384F84630B8F1000F14D00025C8F80040284640
:2081600002B0BDE8F087C7F81441DCE74C2404FB06743034DFE76FF00805AFE76FF00B05D6
:20818000ACE74546EBE7F0B585B007460E461D460192FFF7D3FB041E12DB03AA01993846E6
:2081A000FFF732FC041E09DB039B0024DA8922F00F0242F00102C3E90465DA81FFF7E0FBD7
:2081C000204605B0F0BD38B50546FFF7B7FB041E05DB284600F06BF80446FFF7D1FB2046C2
:2081E00038BD38B5044650B1FFF7A8FB051E04DBA3890133A381FFF7C3FB284638BD0546D1
:20820000FBE738B50546FFF799FB041E0ADB2846FFF75AFC041EA1BF6A6893890133938141
:20822000FFF7AEFB204638BD10B50446C8B1FFF785FB0028FBDBB4F90C304BB9E389DB060E
:208240000BD5FFF79DFB2046BDE8104000F044B8013B1BB2002BA381F0DDBDE81040FFF759
:208260008FBB10BD10B5044688B0D0B100240123019001A806948DF81C30CDE90244CDE980
:208280000444FFF721FCA04207DBDDE90242636852B153600023C4E90033069808B1FBF7E8
:2082A0001FFF204608B010BD049A9360F2E710B5FFF7D8FF68B1B0F90C4034B1C28942F049
:2082C0001002C2816FF00F0010BD00F005F82046FAE76FF00100F7E710B5044650B14068E4
:2082E000FFF7FAFFA068FFF7F7FF2046BDE81040FBF7F6BE10BD00F067BBFFEC024A136809
:2083000001331360704700BFE4140024024B1B68986800B124307047BC0400240F4B10B595
:208320001B680446B3F92020002A0ADD1A7C037C9A4206D20A49F9F7C7FE012300202377C4
:2083400010BD06492046F9F7BFFE022320B10322227722681377F3E72377F1E7BC040024F6
:20836000B004002438B5436804465BB90368032201251A7720460449FCF79EF8002328461B
:20838000237738BD0025F5E7BC040024F0B5134D0020134C02262A68032723681BB923601F
:2083A0006360F0BD1268B2B193F810C0117C8C45F8D95168D3F800C0C3E9002139B90120C2
:2083C000536016772B601F771A466346E6E70B6053601E77F8E75368FFDE00BFBC04002499
:2083E000B0040024024B1B6898682C30704700BFBC040024044B1B6823B11868B0FA80F0DF
:208400004009704701207047BC040024014B1868704700BFBC04002438B50F4B0C461D685C
:2084200070B1F9F7AFFBA0B1EB8B03F00303022B07D0AA6883689A4203D06FF00C0007E0BF
:208440002846436B2360836B6360C36B0020A36038BD6FF00100FBE7BC04002438B5164B12
:208460001C68EFF3118500238022EFF3108372B682F3118883F31088D8B103881BB2002B76
:20848000038803F1FF331BB2038005DD00202064EDB285F3118838BD00232064052120467D
:2084A0006384F9F799FEB4F922000028F0D04042EEE76FF01500EBE7BC04002410B5044607
:2084C0002046FFF7CBFF031DFAD010BD10B5FFF7C5FF041E06DA6442FBF794FF04604FF070
:2084E000FF3010BD0020FCE738B5002834D0EFF3118500238022EFF3108372B682F311887C
:2085000083F31088038847F6FF721BB2934205D1EDB285F311886FF08A0038BD038801334F
:208520001BB2038003881BB2002B0EDC0C4B1C685CB1236C83420DD104F12400F9F76EFDF0
:20854000002320462364F9F71DFFEDB285F311880020E2E72468EBE76FF01500DDE700BF11
:20856000D004002410B5FFF7BFFF041E05DA6442FBF748FF04604FF0FF34204610BD70B57C
:2085800005460C46F8F7D8FCEFF3118600238022EFF3108372B682F3118883F310882B88D1
:2085A0001A0409D42B881B040ED5F6B286F31188F8F7D2FC002070BD002CF3DD013C2846A0
:2085C000FFF792FF24B2EAE72C80EEE737B5041E0D4616DB1F2917D8F8F7AEFC0023042281
:2085E000204669468DF800508DF801308DF802200193F9F751F90446F8F7AEFC204603B06A
:2086000030BD6FF05704F9E76FF01504F6E7FFEC07B568B1084A0021B0FBF2F302FB1300AB
:2086200000934FF47A7358430190684600F0EEF803B05DF804FB00BF40420F0038B50F4C28
:2086400025682846FFF78EFE0D4B1B680BB1FFF79DFE246828460421238C013323840223A7
:208660002377F9F70FFD0121E86800F019F803232377238C013B238438BD00BFBC04002407
:20868000B0040024054B186830B1037F032B01D1C06870476FF00200704700BFBC04002435
:2086A00070B50E46EFF3118500238022EFF3108372B682F3118883F31088F9F763FA0446B4
:2086C000EDB2A0B1027F0C4B53F83210FBF7F4FE85F31188002120463246F9F7F7F9E18B05
:2086E000204601F00301BDE87040F8F7ABBE85F311886FF0020070BDC09F0008054B18689C
:2087000030B1037F032B01D1C06870476FF00200704700BFBC0400242DE9F0410C46164667
:2087200098460546002839D0002A37D0002935DBEFF3118700238022EFF3108372B682F324
:20874000118883F3108843680BB1F9F767FC1F4901346E600E68C5F80C801EB92846FBF757
:208760005BFE2CE03046334600229968521801D5196831B9A24214DC196829B9A41A134986
:20878000ECE718460B46F0E78868024418460B46F0E70E4A294600F048FA10E06FF0150067
:2087A00012E099689E42A2EB0102A4EB0204A1EB04019960EDD10549284600F030FAAC6097
:2087C000FFB287F311880020BDE8F081380A002438B50D4C236843B19A680025013A9A6018
:2087E000236813B19B68002B00DD38BD2046FBF733FE23681BB19A6881680A449A6043686C
:208800004560C0689847EBE7380A00242DE9F7430F46054600283BD042681F4B9A4237D852
:20882000EFF3118600238022EFF3108372B682F3118883F31088DFF864906846F6B2D9F84F
:208840000080FBF79EFE2A460021684600F038F810F10B0F044606D186F3118800242046D3
:2088600003B0BDE8F08387B101A9284600F0FAF9D9F8003001983946A3EB080290428ABF2E
:20888000C01A0020404400F0DFF986F31188E6E76FF01504E3E700BFFFC99A3BE4140024F9
:2088A000027F062A0AD140F2FF22A0F85C20742280F85E2000220266F9F764BD7047FFECFC
:2088C000394B2DE9F34707460D4692461C68EFF3118800238022EFF3108372B682F31188DD
:2088E00083F3108806682046F9F710FB30405FFA88F80190A0B101A8F8F790FE014620469D
:20890000F8F73AFE1DB143682B6083686B600679F8F756FE88F31188304602B0BDE8F0875C
:208920003B68A364BAF1000F33D0DAF8043004F124091E4ED917DAF800C09E191C481D4A38
:208940004FF0000341F10001ECFB0061304600F0C7FC23460146184A4846FFF7DDFE20465A
:208960000621F9F739FC4846F9F758FB94F85C1000231F29A36411D83846FBF706FE80B1E2
:2089800094F85C60002DC5D0E36D2B60236E6B60C0E706212046F9F71FFCE7E76FF00A061A
:2089A000F0E76FF00306EDE7BC0400243F420F0000CA9A3B40420F00A188000808B500F022
:2089C00021FC002008BDFFEC10B5084B4FF0E0240022074963610F20A261F8F755FA07237F
:2089E0000F202361BDE81040F7F7D4BFFF520700BD89000838B504464518207808B1AC42D5
:208A000000D138BD0134F9F7C1FFF6E7024B0A460146186800F002B8B00F00242DE9F84F80
:208A2000804614460E4621B91146BDE8F84FFBF77FBC12B9FBF720FC18E002F1170323F087
:208A40000F0B5A4500F2B280A1F10805FBF7C0FB56F8089CCB450CD804D25A46294640469C
:208A600000F0A6F834464046FBF7D6FB2046BDE8F88F56F8041C05EB090A21F00101DAF8BD
:208A80000430691ADA0748684CBF002755F80970C30707EB090354BF0868002003445B4544
:208AA00071D3B842ABEB090308D2984252D2A3EB000B034633B95B46344623E09F42FBD264
:208AC000DB1BBB46D1E9024294600CB1CA68E2609842A5EB030540D90A68D21A4B440A609A
:208AE0002B600C6844F001046C60DAF8040000F001001843CAF804004046FBF795FB05F18C
:208B000008045B46D3B10AEB0700DAE90212916011B1DAF80C20CA602A689F421A442A601B
:208B20002BD9FB1AA918AB502A684A60476807F001073B4343604046FBF776FB4046FBF7F4
:208B40006BFBB44292D0A9F1080231462046F7F777FF8BE74FF0000BACE72B6809EB030297
:208B60006B6843F001032A606B60DAF8043003F001031343CAF80430C1E7436803F0010303
:208B80001A434260DAE74046FBF746FB21464046FBF7CEFB044600283FF468AF3146A9F1E7
:208BA0000802F7F74DFF3146404643E700245DE7F0B40C680B4606460D196968C90719D479
:208BC0001859D5E902172844B96009B1ED68CD601D6899181C59AD1A25449D504A601A60A0
:208BE00044689B5804F001041C4344603046F0BCFBF71ABB02F110018C4209D39918A41AD4
:208C00009C504A601A609B5843F001036B60EEE7F0BC704708B500F039FA406B08BD0B6854
:208C2000036003B9486008607047034608461146126812B14A689A4201D1FBF7EDBB1A68A7
:208C4000026018607047FFEC4FF47A7290FBF2F302FB13000B60024B584348600020704717
:208C600040420F0038B543680C460568084AD917E5FB02311846074B074AC0184FF000039C
:208C800041F1000100F0DCFA2060002038BD00BF00CA9A3B3F420F0040420F00084631B197
:208CA0000139022934BF6FF085006FF0150070470EB403B503AA52F8041B019200F01DF825
:208CC00002B05DF804EB03B070470CB40A4600B589B071B1014602A800F022F90BAA0A99C0
:208CE00002A80192FBF758FE09B05DF804EB02B0704702A800F02CF9F0E770B58EB0144636
:208D00000D46064604A8039200F022F92246294604A8FBF741FE079A013210460192FBF705
:208D2000E7F9044660B10146019A08A800F0F8F8039A294608A8FBF72FFE34600EB070BD2C
:208D40004FF0FF30FAE70A22002100F000B837B50C460190009290B301A800F02BF9019BD2
:208D6000009A1D782D2D01D02B2D12D1013301932146019800F025F82D2D0FD1B0F1004F5F
:208D800009D9FBF73FFB222303604FF000407CB915E00025ECE7FAD04042F8E7002805DA4A
:208DA000FBF730FB222303606FF000403CB135B1236813F8012CAA4201D1013B236003B089
:208DC00030BD2DE9F04385B00E4614460190002850D001A800F0EEF8019B1F782D2F01D0C2
:208DE0002B2F18D10133019301A9204600F046F8051E12DAFBF706FB0024162303606EB347
:208E000037B1019B13F8012CBA4201D1013B0193019B336022E00027E6E74FF0FF38002439
:208E2000B8FBF5F805FB08F96FEA0909019B03AA2946187800F098F858B1444503D8039B53
:208E400010D199450EDAFBF7DDFA4FF0FF34222303602D2FD3D16442002ED2D1204605B0F6
:208E6000BDE8F08304FB0534019B01330193DDE70446CDE70029FBD10C46EFE770B50D46E7
:208E80000C6890B92378302B21D16378661C03F0DF03582B1DD102461021A07800F064F8AD
:208EA000B8B1023410202C6070BD102809D12378302BF8D1637803F0DF03582BF3D102342C
:208EC000F1E7831E182BEED94FF0FF30ECE70A20E9E734460820E6E738B50546C0686B6931
:208EE0001B1A934228BF1346002B1C460ADD2B6922461844F7F7A4FDEB682A69002123445F
:208F0000EB60D154204638BD07B501228DF807100DF10701FFF7E0FF03B05DF804FBFFEC3E
:208F2000064B013A0360064B42614360054B83600023C0E903310B70704700BF098F0008E7
:208F4000D98E0008DB530008C3680133C3607047034B0360034B83600023C360704700BF95
:208F6000498F0008DB5300080A290ADC2F281EDD2F3181421BDBA0F13003012002B113604C
:208F80007047242913DCA0F13003092BF3D9602805DD563181420ADBA0F15703EDE740285A
:208FA00005DD3631814202DBA0F13703E5E700231846E3E770B5044605682E4601353078B8
:208FC00000F069F80028F8D1266070BD13B50190FBF778FC0130FBF78BF8044610B1019992
:208FE000FBF74CFC204602B010BDFFEC014A00F003B800BFE81400242DE9F0418846164621
:20900000044610B9CAB11468BCB125462C4615F8011BA9B1404600F015F80028F6D1297866
:209020002F46013539B1404600F00CF80028F6D000233B702F4606B137602046BDE8F08126
:209040000C46FAE703461A78184601338A4202D0002AF8D1104670470A4640F2011100F04E
:209060008FB870B5044616460D4639B100F022F8022D03D10021204600F017F83246204630
:209080004FF48171BDE8704000F07AB808B5FBF755FC006808BD202805D0093804288CBF22
:2090A000002001207047012070470A464FF48A7100F066B8002240F2151100F061B8F0B51C
:2090C000876885B004460D461668002F55D03B69C3B940F20D339D420DDCB5F5417F0EDB50
:2090E000A5F54175092D0AD8DFE805F02A09090909090916222640F20F539D422CD06FF0C0
:20910000180007E05B69002BE3D03246984710F1190FDED005B0F0BD236836B1326822B13F
:2091200043F0400300202360F4E723F04003F9E7236843F48063F5E7236823F48063F1E727
:20914000FB8903F00F03032BD9D03146384605B0BDE8F04000F032B83B69002BCFD05B6924
:20916000002BCCD001AA40F20C51204698470028D0DBBDF90C303380CCE76FF00800C9E767
:209180000EB477B507AD01A955F8046B0095FEF75EFB041E06DB2A4631460198FFF78FFFDD
:2091A000041E05DA6442FBF72DF904604FF0FF34204603B0BDE8704003B0704738B504460B
:2091C0000D46C9B110B90870002038BD0068FFF7F5FF0028F9DB04F11801284600F020F89A
:2091E000A06820B9E28902F00F02032AEDD10449284600F015F8E7E76FF01500E5E700BFB0
:2092000068A5000808B5054B0BB1FFF777F8FFF7DFFABDE80840F7F778BD00BFFD820008E6
:2092200038B505460C46FBF74DFB611E2B1811F8012F12B928461A7038BD03F8012BF6E7B3
:209240007BB972B90029BEBF00204FF0004106E008BF00281CBF6FF000414FF0FF3000F0BB
:20926000DFB9ADF1080C6DE904CE002909DB002B1ADB00F06DF8DDF804E0DDE9022304B0A2
:209280007047404261EB4101002B1BDB00F060F8DDF804E0DDE9022304B0404261EB410136
:2092A000524263EB43037047524263EB430300F04FF8DDF804E0DDE9022304B0404261EB4A
:2092C00041017047524263EB430300F041F8DDF804E0DDE9022304B0524263EB430370470D
:2092E00053B94AB9002908BF00281CBF4FF0FF314FF0FF3000F094B9ADF1080C6DE904CE78
:2093000000F026F8DDF804E0DDE9022304B070479FED0B6B41EC170B9FED0B5B27EE066B67
:20932000BCEEC66BB8EE464BA4EE457BFCEEC77B16EE101A17EE900A704700BFAFF3008038
:20934000000000000000F03D000000000000F0412DE9F047089D04468E46002B4DD18A428A
:20936000944669D9B2FA82F252B101FA02F3C2F1200120FA01F10CFA02FC41EA030E9440CA
:209380004FEA1C48210CBEFBF8F61FFA8CF708FB16E341EA034306FB07F199420AD91CEB95
:2093A000030306F1FF3080F01F81994240F21C81023E63445B1AA4B2B3FBF8F008FB103339
:2093C00044EA034400FB07F7A7420AD91CEB040400F1FF3380F00A81A74240F207816444DB
:2093E000023840EA0640E41B00261DB1D4400023C5E900433146BDE8F0878B4209D9002D39
:2094000000F0EF800026C5E9000130463146BDE8F087B3FA83F6002E4AD18B4202D382423A
:2094200000F2F980841A61EB030301209E46002DE0D0C5E9004EDDE702B9FFDEB2FA82F277
:20944000002A40F09280A1EB0C014FEA1C471FFA8CFE0126200CB1FBF7F307FB131140EA8F
:2094600001410EFB03F0884208D91CEB010103F1FF3802D2884200F2CB804346091AA4B2F2
:20948000B1FBF7F007FB101144EA01440EFB00FEA64508D91CEB040400F1FF3102D2A645E1
:2094A00000F2BB800846A4EB0E0440EA03409CE7C6F12007B34022FA07FC4CEA030C20FA51
:2094C00007F401FA06F31C43F9404FEA1C4900FA06F3B1FBF9F8200C1FFA8CFE09FB1811DB
:2094E00040EA014108FB0EF0884202FA06F20BD91CEB010108F1FF3A80F08880884240F2AE
:209500008580A8F102086144091AA4B2B1FBF9F009FB101144EA014100FB0EFE8E4508D9A0
:209520001CEB010100F1FF346CD28E456AD90238614440EA0840A0FB0294A1EB0E01A142AA
:20954000C846A64656D353D05DB1B3EB080261EB0E0101FA07F722FA06F3F1401F43C5E965
:20956000007100263146BDE8F087C2F12003D8400CFA02FC21FA03F3914001434FEA1C470D
:209580001FFA8CFEB3FBF7F007FB10360B0C43EA064300FB0EF69E4204FA02F408D91CEB03
:2095A000030300F1FF382FD29E422DD9023863449B1B89B2B3FBF7F607FB163341EA03416F
:2095C00006FB0EF38B4208D91CEB010106F1FF3816D28B4214D9023E6144C91A46EA0046C4
:2095E00038E72E46284605E70646E3E61846F8E64B45A9D2B9EB020864EB0C0E0138A3E748
:209600004646EAE7204694E74046D1E7D0467BE7023B614432E7304609E76444023842E7EA
:20962000704700BF0720704710B54220094CFAF749FC4FF000634320C4F88034FAF742FC80
:209640004420FAF73FFC0023C4F88034C4F8D83410BD00BF0040025808B5042000F0BCF973
:20966000064B4FF47A70DB68584300F0A9F900F0D9F9BDE8084000F0BFB900BFAC00002456
:2096800008B500F0D7F900F0BFF9002000F0A4F90020BDE8084000F093B9FFEC0F4BD3F89F
:2096A000002442F00102C3F80024D3F800245207FBD50022C3F81024D3F8002422F0A8524E
:2096C00022F41022C3F80024054AC3F82C24D3F8002422F48022C3F8002470470040025832
:2096E0000000FF0108B54FF0006000F03CFA4FF00160BDE8084000F036BA08B500F0C4FB0F
:209700004FF0006000F01CFA4FF00160BDE8084000F016BA00F0D4BA4FF0E023C3F8080DC7
:2097200070470F2894BF4FF4003000207047431E0E2B10B5044609D821B12046BDE81040E7
:2097400000F04DBA00F036FA0028F6D110BD00F1006000F5003000F0B3BB830705D100F111
:20976000006000F5003000F0EBBB0020704700207047FFEC014B1868704700BF0010005C87
:20978000234BF0B51A680446224BC2F30B06120C1F885868BE421D7A2BD09F89BE4205D1A2
:2097A00001200C2505FB003358681D7A41F203039A4220D042F201039A421ED042F203038C
:2097C0009A421CD041F201039A4208BF5A25621E0B46441E0A44934217D214F8016F581C39
:2097E0007EB92C2482421C7001D9981C5D70401AF0BD0020D5E75925E9E75825E7E7562540
:20980000E5E7034600F8016CE5E71846EFE700BF0010005CBC00002400F1FF5000F58F10EF
:20982000D0F800087047FFEC012802D0022804D0704700210248FAF72FBB00210148FAE775
:2098400043090400440904000128014602D0022803D070470248FAF71FBB01210148FAE710
:209860004309040044090400012808B502D002280BD008BD0948FAF70BFC80F00100C1B298
:209880000648BDE80840FAF707BB0548FAF700FC80F00100C1B20248F3E700BF4309040089
:2098A00044090400D0E9003283F308881047FEE74FF0E0224FF4003070B5D2F8883D344D41
:2098C00043F47003C2F8883D324B334AD3F8803803F57F1303F57E539B029360FAF7F2FA22
:2098E0002E48FAF7EFFA2E48FAF7ECFA0120F6F7E1FE00202C6DF6F7DDFE2A4B9C4242D1F7
:2099000000240120F6F7D6FE264620462C65F6F7D1FE254800F014FB0546244800F010FB04
:20992000234B98420ED125F0FF02224B9A4209D1EDB21E2D06D84FF47A7000264543AC4236
:2099400038BF2C464220FAF7A3FB054660B95EB1FBF79EFE0120F6F7ADFE0D4B114A2C46CE
:2099600028461A65F6F7A6FE01211348FBF713FE02211248FBF70FFE20460024FBF7D8FE1B
:20998000FBF786FEF8E741F288340126C1E700BF0040005800E0F11FAC000024430904004D
:2099A0004409040007B007B0A0010208A40102085D7D05C500ECC2926AA500087BA500086B
:2099C000044B1B6858434FF0E02320F07F405861704700BFD4000024021E054B05480CBF5A
:2099E0000821012102F0040219600421F6F780BED400002410E000E0012200210148F6F719
:209A000077BE00BF10E000E000220121044808B5F6F76EFE4FF0E02300229A6108BD00BFF9
:209A200010E000E0022200210148F6F761BE00BF10E000E0002202210148F6F759BE00BFDC
:209A400010E000E0042838B505460C4613D80120F6F7F0FD032D094B4FF000000CBF24F0F8
:209A6000FF01002153F825301943054B1965F6F7E1FD002038BD4FF0FF30FBE7A4A500087A
:209A8000004000580128044608B502D10021FFF7D9FF2046F7F730F900F0E2F9436803F155
:209AA00010010A68D207FCD4DA68D20705D5034A5A6002F1883243685A60704723016745E5
:209AC00002460A488168914203D801F5801191420AD807488168914205D801F580119142D7
:209AE00098BF002070470020704700BFD8000024EC00002420B40D46406811461A462844A4
:209B00005DF8045BF6F7F4BD012300220C21FFF7F1BFFFEC38B50546BFF34F8F074C6B6801
:209B20001B6913F0070307D00120F6F7F6FD013CF5D16FF00F0038BD1846FCE7404B4C003E
:209B400038B5FFF7BDFF054650B1FEF7B7FC041E04DB2846FFF7A2FFFEF7C6FC204638BD5A
:209B60006FF01204FAE738B5FFF7AAFF054658B1FEF7A4FC041E05DB2846FFF7C5FF284682
:209B8000FEF7B2FC204638BD6FF01204FAE7B0F5803F08B503460AD200F580004001FFF77F
:209BA0008FFF026980689B1A00EB431008BD4FF0FF30FBE7B0F5803F08B50DD2FFF7E7FFE0
:209BC000002300F1200201780130FF2918BF01338242F8D1184608BD6FF00D00FBE7F8B5C7
:209BE000044600F580600F2C4FEA404562D82846FFF766FF0646FEF761FC00284DDB3046E6
:209C0000FFF788FF074600284BD13046FFF746FF04233A460C21FFF76DFFF3684FF47062DF
:209C20000C21E31A30461B0203F4E063FFF762FF80233A460C213046FFF75CFF3046FFF753
:209C400069FF044650BB034604220C213046FFF751FF23464FF470620C213046FFF74AFF8F
:209C60003046FFF751FF3046FEF73EFC2CBB2846FFF726FF08B305F5FF3000F2FF10FFF738
:209C80001FFFD0B1284605F5003383420CD1002C14BF6FF004004FF40030F8BD6FF00404F7
:209CA000DEE76FF00404DEE702680430013218BF0134EAE76FF00D00EFE76FF00400ECE78D
:209CC0002DE9F84F06460F461546FFF7F9FE0446002800F0C2808368B34200F2BE80AA19C7
:209CE00003F580139A4200F2B880FEF7E7FB002865DB2046FFF70EFF8046002840F0AA80E3
:209D000020462037FFF7CAFE302325F01F0B0C211A46B946FFF7EEFEB3444246B04602232E
:209D20000C212046FFF7E6FED84532D0BFF34F8FBFF36F8F59F8203CC8F8003059F81C3C11
:209D4000C8F8043059F8183CC8F8083059F8143CC8F80C3059F8103CC8F8103059F80C3C9F
:209D6000C8F8143059F8083CC8F8183059F8043CC8F81C30BFF34F8FBFF36F8F2046FFF709
:209D8000C9FE08BB636809F120091B6913F0C06F17D0002302220C212046FFF7ABFE4FF0F6
:209DA000FF33002214212046FFF7A4FE2046FFF7ABFE002D41D12046FEF796FB2846BDE8D9
:209DC000F88F08F12008AFE76FF00405EEE74FF0FF33002214212046FFF78CFE326857F871
:209DE000203C9A4233D1726857F81C3C9A422ED1B26857F8183C9A4229D1F26857F8143C3F
:209E00009A4224D1326957F8103C9A421FD1726957F80C3C9A421AD1B26957F8083C9A42AC
:209E200015D1F26957F8043C9A4210D1636820371B6913F0C06F0AD120365E45C7D14FF012
:209E4000FF33002214212046FFF754FEB3E76FF00405F4E76FF00405ADE76FF00D00AEE7F1
:209E60004FF0E021054BD1F80C2D02F4E0621343C1F80C3DBFF34F8FFEE700BF0400FA0589
:209E80002822FF21F6F7F1BE10B5054C2046FFF7F7FF04F12800FFF7F3FF024B636010BD72
:209EA000EC1400240000020800F10801202208B54068FFF72FFC202808BF002008BDFFECD3
:209EC0001D4A20F01F0310B554689C4225D0D46AA34224D10123282404FB0323C0F38204AF
:209EE00013B93CBB154BD062A01C934243F820101FD1F4B91A68072A1BD19A6A013210D0BE
:209F000003F128042046FFF7CFFF50B120464FF0FF34FFF7B5FF204610BD0023DBE7002339
:209F2000DCE70548FFF7C0FF04460348FFF7A8FFF1E71C600024EEE7EC140024141500246C
:209F4000144A38B520F01F035168056899421AD0D16A8B4215D101232824C0F382000A21DB
:209F600004FB032401FB0303944203F1020352F8235006D0072804D12046FFF795FF20B192
:209F8000ED43284638BD0023E6E72046FFF778FFF7E700BFEC1400242A18002461726D768E
:209FA000372D6D2F61726D5F686172646661756C742E630049646C65205461736B00FFEC9A
:209FC0000000000000000000B004002401000000BC04002405000000BC04002405000000D6
:209FE0009C04002400000000D004002401000000D804002400000000C804002400000000B4
:20A00000626F6F746C6F616465725F6D61696E004170704272696E675570006972712F6955
:20A0200072715F756E65787065637465646973722E63003C6E6F6E616D653E0001000000D1
:20A04000B919000802000000B919000803000000B9190008060100009D19000807000000A1
:20A060009D19000808010000991900080A000000B919000809010000B91900080B0000008C
:20A08000B91900080C000000B91900080D000000B9190008736572636F6E3A3A2045525212
:20A0A0004F523A20416C726561647920636F6E6E65637465640A00736572636F6E3A2052D0
:20A0C00065676973746572696E67204344432F41434D2073657269616C2064726976657219
:20A0E0000A00736572636F6E3A204552524F523A204661696C656420746F20637265617417
:20A100006520746865204344432F41434D2073657269616C206465766963653A2025640A72
:20A1200000736572636F6E3A205375636365737366756C6C792072656769737465726564E8
:20A1400020746865204344432F41434D2073657269616C206472697665720A002F646576F0
:20A160002F747479537800FF00000024000000000000000000000000000000000000000061
:20A18000000000000000000061280008ED280008F5270008D9270008392700088D260008C2
:20A1A000A7260008E1260008ED260008F52600082D2700082D2700081D2B00088D2B0008B5
:20A1C000C52B00083D2C0008D52B0008E12B000800000000CD2A0008212E0008232C00084D
:20A1E0001D2C0008CD300008F72D0008A5320008000002580004025800080258000C02587E
:20A20000001002580000000000000000001C0258556D656D00FFECC200000000000000001D
:20A2200032000000010000004B000000020000006E000000030000008600000004000000A3
:20A240009600000005000000C8000000060000002C010000070000005802000008000000FF
:20A26000B004000009000000080700000A000000600900000B000000C01200000C000000B6
:20A28000802500000D000000004B00000E000000009600000F00000000E10000011000001C
:20A2A00000C20100021000000084030003100000000807000410000020A10700051000002F
:20A2C00000CA08000610000000100E000710000040420F00081000000094110009100000FA
:20A2E00060E316000A10000080841E000B100000A02526000C100000C0C62D000D100000D7
:20A30000E06735000E10000000093D000F100000696E66006E616E00286E756C6C2900FFB9
:20A320000080E03779C3314300003426F56BFC420000901EC4BCC642000040E59C309242E3
:20A34000000000A2941A5D42000000E876482742000000205FA0F2410000000065CDBD417D
:20A360000000000084D7874100000000D01253410000000080841E4100000000006AE8404F
:20A38000000000000088B3400000000000407F400000000000004940000000000000144066
:20A3A0009A9999999999B93F7B14AE47E17A843F2D431CEBE2361A3F3A8C30E28E79453E22
:20A3C000BC89D897B2D29C3C33A7A8D523F649393DA7F444FD0FA5329D978CCF08BA5B25AB
:20A3E000436FAC642806C80A00000000000024400000000000005940000000000088C34013
:20A400000000000084D797410080E03779C34143176E05B5B5B89346F5F93FE9034F384D40
:20A42000321D30F94877825A3CBF737FDD4F1575505834424C76312E31372E3067653561FF
:20A440006366363300FFECC2050000002C002F6465762F7474795330002F6465762F6E75EB
:20A460006C6C00FF0000000000000000B15E0008B55E00080000000000000000B95E0008B4
:20A4800000000000FF600008A1670008BF5F00089D6200080000000059650008D361000816
:20A4A000000000002F6465762F74747941434D256400FFECD16C00080F6C0008CD6E00084E
:20A4C000C76B0008CD690008BD69000867690008796900087B69000861730008D569000806
:20A4E0000000000079710008000000000000000003730008000000007F69000842756C6B6E
:20A50000004D6174656B004D6174656B20483734332D736C696D00120100020200004062B6
:20A52000314B00010101020301FFECC2AB760008AB760008000000009B760008000000007E
:20A5400025732F257300FFECA5800008417F00087F7E000800000000877F0008637E0008C0
:20A5600000000000000000002F002F6465762F74747953302C3537363030002F6465762F60
:20A5800074747941434D300053544D33323F3F3F3F3F3F3F0053544D333248375B347C352F
:20A5A0005D7800FF0000000007B007B0020007B0000008B0263A09B098EDFF7F01000000CB
:20A5C00000000000000000000000000000000000000000000000000000000000000000007B
:20A5E0000000000000002C019C0C00240000000000005802440A002488A100080000002441
:20A600000000000000000000000000000000000000000000000300080000000000C201006C
:20A6200035000000000E270700100140097C09000A7C0900FFFFFFFFFFFFFFFF2CA500086A
:20A640007C00002401000000FFFFFFFF00000000000000000000000000000000010000005C
:20A6600048A500080000000000000000D95900000000000000000000E001000000000000D2
:20A6800088A500083F0000005004000095A500083F000000010000000100000000200052FD
:20A6A00000000008000000000000000001000000002100520000100808000000008000007E
:020000040802F0
:200000003AC5002405030208A9020208A9020208A9020208A9020208A9020208A90202086D
:20002000A9020208A9020208A9020208A9020208A9020208A9020208A9020208A902020818
:20004000A9020208A9020208A9020208A9020208A9020208A9020208A9020208A9020208F8
:20006000A9020208A9020208A9020208A9020208A9020208A9020208A9020208A9020208D8
:20008000A9020208A9020208A9020208A9020208A9020208A9020208A9020208A9020208B8
:2000A000A9020208A9020208A9020208A9020208A9020208A9020208A9020208A902020898
:2000C000A9020208A9020208A9020208A9020208A9020208A9020208A9020208A902020878
:2000E000A9020208A9020208A9020208A9020208A9020208A9020208A9020208A902020858
:20010000A9020208A9020208A9020208A9020208A9020208A9020208A9020208A902020837
:20012000A9020208A9020208A9020208A9020208A9020208A9020208A9020208A902020817
:20014000A9020208A9020208A9020208A9020208A9020208A9020208A9020208A9020208F7
:20016000A9020208A9020208A9020208A9020208A9020208A9020208A9020208A9020208D7
:20018000A9020208A9020208A9020208A9020208A9020208A9020208A9020208A9020208B7
:2001A000A9020208A9020208A9020208A9020208A9020208A9020208A9020208A902020897
:2001C000A9020208A9020208A9020208A9020208A9020208A9020208A9020208A902020877
:2001E000A9020208A9020208A9020208A9020208A9020208A9020208A9020208A902020857
:20020000A9020208A9020208A9020208A9020208A9020208A9020208A9020208A902020836
:20022000A9020208A9020208A9020208A9020208A9020208A9020208A9020208A902020816
:20024000A9020208A9020208A9020208A9020208A9020208A9020208A9020208A9020208F6
:20026000A9020208A9020208A9020208A9020208A9020208A9020208A9020208A9020208D6
:20028000A9020208A9020208A9020208A9020208A9020208A9020208000000000000000020
:2002A000FFECC2925D7D05C5EFF305801EF0040F02D0EFF309818D466A4602F16802EFF3D3
:2002C00011831EF0100F0CBF2DED108A90B02DE9FC4F6946DFF828D000F076FFB0E8FC4F77
:2002E0001EF0100F0CBFB0EC108A40301EF0040F0CBF80F3088880F3098883F311887047A7
:200300000012002408B501F00CF81E4B1E48DA1CC11E121A22F00302994288BF00220021A9
:2003200001F0A3FC194B1A48DA1CC11E121A22F00302994288BF0022164901F029FB00F0A7
:2003400023F900F059FF00F08FF9BFF34F8FBFF36F8F4FF0E023D3F8902F22F00102C3F8E5
:20036000902F0522C3F8942FBFF34F8FBFF36F8F36F1B4FF00F06CFE00F07EFE00F036FD16
:2003800002F0D8FC4CC20024000F0024D90E00240000002424651C08744A82B0D2F8003468
:2003A00023F4802343F48033C2F80034704B0193019B002B00F3D180019B002B40F3CB800C
:2003C0006A4BD3F8182422F4706222F00F0242F00802C3F81824D3F81C2422F4E06242F08E
:2003E0004002C3F81C24D3F81C2422F4E06242F48062C3F81C24D3F8182422F0700242F08D
:200400004002C3F81824D3F8202422F0700242F04002C3F82024D3F8102422F47C5242F484
:200420000062C3F81024534AC3F82824524AC3F83024524AC3F8382402F50032C3F8402421
:200440004F4AC3F82C24D3F8002442F0A852C3F80024D3F800249001FBD5D3F800241101AD
:20046000FBD5424BD3F800249200FBD5D3F80C2842F00602C3F80C28D3F8182842F44042E3
:20048000C3F81828D3F818289004FBD5374BD3F804289104FBD5D3F8F4244FF0B04142F0CF
:2004A0000202C3F8F424D1F82C2442F00102C1F82C24D3F818289204FBD5324A222111606D
:2004C000D3F8102422F0070242F00302C3F81024264BD3F8102402F03802182AF9D1D3F869
:2004E000542422F4405242F40052C3F85424D3F8582422F4407242F40072C3F85824D3F868
:20050000502422F4E04242F48052C3F85024D3F8502422F4E02242F48032C3F85024D3F8BF
:20052000582422F0E04242F08052C3F85824D3F8542422F4401242F40012C3F85424D3F8DF
:20054000582422F44032C3F85824D3F8502422F04052C3F8502402B07047D2F800349B0349
:200560003FF52AAF019B013B21E700BF00400258F82F910012202000770203072F02010175
:200580008808BF000020005210B52F4C00200122D4F8003443F00103C4F800342B4BC3F8BF
:2005A0000821C4F810042A4BD4F80024134043F01003C4F80034274BC4F82C34D4F80034C6
:2005C00023F48023C4F80034C4F8600400F0A2FCFFF7E2FED4F8D83443F0006343F0230326
:2005E000C4F8D834D4F8DC34C4F8DC34D4F8D43443F48033C4F8D434D4F8E03443F089531A
:2006000043F09F03C4F8E034D4F8E83443F4C10343F48043C4F8E834D4F8EC34C4F8EC34B8
:20062000D4F8F03443F4405343F03003C4F8F034D4F8E434C4F8E434D4F8F43443F00203D6
:20064000C4F8F43410BD00BF004002580080005167EFFEEA0000FF01024BDA691206FCD508
:20066000986270470010014010220021144808B500F09AFC134800F07FFE134800F07CFEF9
:20068000124B5A6822F4FE4222F070021204120C5A601A6822F04F4222F47F0222F47F42E0
:2006A00022F0FC021A600A4A99680A409A6040F62302DA601A6842F00D021A6008BD00BFC1
:2006C000F0440258097C09000A7C0900001001400000F1FF10B5D0F88C4001F4D873A0F8FD
:2006E000741001F00101226822F4D87213432360D0F88C20936823F001031943916010BD20
:2007000010B5EFF3118400238022EFF3108372B682F3118883F31088FFF7DCFFE4B284F341
:20072000118810BD10B5EFF3118400238022EFF3108372B682F3118883F3108849B1D0F8D7
:200740008C201368926803F4D87302F0010213430B800021E4B2FFF7BDFF84F3118810BD1A
:20076000F0B5036EEFF3118400228021EFF3108272B681F3118882F31088D3F88C100A689A
:2007800022F0010002F001050860D3F88060D3F88870710801EB4701B1FBF6F1642941D991
:2007A000013122F40040490820F00100D3F88C201060D3F88C20D16093F87A10254A012912
:2007C00002EA000238D142F4C06293F87B00092802D0082835D1A1B342F48052D3F88C10C8
:2007E0000A60D3F88C0093F87C60416821F440510EB141F400514160D3F88C0093F87E60DC
:20080000816821F4407126B1D3F89C600EB141F4007181602A43D3F88C30E4B21A6084F3CA
:200820001188F0BDC1F3420221F00F0140F400400904090C1143B9E7022908BF42F48062C5
:20084000C3E7B3F87A10B1F5E06F08BF42F08052C4E700BFFEE9FFEF036ED3F88C20506A18
:20086000B3F8762040EA0242C0B20A600022A3F87620704710B5006EEFF311840023802274
:20088000EFF3108372B682F3118883F31088B0F8743039B143F02001E4B2FFF731FF84F3E2
:2008A000118810BD23F4907121F00101F4E7036ED3F88C30D869C0F340107047036ED3F89D
:2008C0008C309962704710B5006EEFF3118400238022EFF3108372B682F3118883F3108882
:2008E000B0F8743041B143EA020189B2E4B2FFF707FF84F3118810BD23F08001F5E7036EFF
:20090000D3F88C30D869C0F3C010704708B5036E114693F87D2022B1D3F8980008B100F049
:2009200015FD002008BDF8B58368B1F5887F5D692C6E00F0368110DCB1F5817F00F0D8809A
:2009400040F20F13994200F00A8140F20113994200F09E806FF018007EE040F23313994296
:2009600052D040F23513994277D0B1F5987FF1D1EFF3118600238021EFF3108372B681F3EC
:20098000118883F31088D4F88C3012F0010F1F6827F001011960D4F88C309D68D4F89030E4
:2009A00029D012F0080F02F0060214BF00214FF40071022A19D0042A4FF0000218D00020F7
:2009C00023F4403345F0080523F400730B431343184300F0D1FCD4F88C309D60D4F88C30F8
:2009E0001F60F6B286F3118835E04FF48032E6E74FF40030E4E723F4403025F0080520F4EC
:200A0000007000F0B9FCE6E7EFF3118100238020EFF3108372B680F3118883F31088D4F83A
:200A20008C30D707186820F001051D60D4F88C506B684CBF43F4803323F4803396074CBF27
:200A400043F4003323F400336B60C9B2D4F88C30186081F311880020F8BDEFF31181002323
:200A60008020EFF3108372B680F3118883F31088D4F88C30012A186820F001051D60D4F88D
:200A80008C506B680CBF43F4004323F40043DBE7002A00F0A08094F87A303BB3012B4FF479
:200AA00080710CBF4FF4007300230B4394F87C101046002914BF402100210B4394F87E10FF
:200AC000002914BF4FF0005100210B4394F87D10002914BF4FF0004100210B4343F03003B1
:200AE0009360D4F8801001F02DF9B4E71946DCE7002A70D0936803F0300130296BD199001C
:200B000003D5D4F89C10002965D0002B03DAD4F8981000295FD013F480711DD013F4007FE8
:200B200014BF0123022384F87A3093681046C3F3801384F87C309368C3F3407384F87E3023
:200B40009368DB0F84F87D3001F01CF9C4F880002846FFF705FE7EE784F87A10E5E7EFF3C5
:200B6000118600238022EFF3108372B682F3118883F31088B4F87430284600216FEA4343A2
:200B80006FEA5343A4F87430FFF79DFED4F8900020F4402020F4807040F4802000F0ECFB16
:200BA0001FE7EFF3118600238022EFF3108372B682F3118883F31088D4F8900000F0DCFB15
:200BC000B4F8743001212846C3F30E03A4F87430FFF779FE05E76FF015003DE710B5046E06
:200BE00094F8840000F022FD002294F884001146BDE8104002F056B938B5056E06492A4638
:200C000095F8840002F04EF9044618B995F8840000F020FD204638BD1D0C020810B51446A4
:200C2000D2F88C20D3699BB29806A4F8763013D5B4F8741089060FD5204601F0DBFDB4F86F
:200C400076301A0606D5B4F874301B0602D5204601F09AFD002010BD13F00E0FEFD00E23C0
:200C60001362ECE7036E0A461E49D3F88C308B4220D00CD8A1F540518B421FD001F5806122
:200C80008B421FD0A1F500618B421FD0704716498B421FD001F580618B421ED0A1F5184192
:200CA0008B421DD111484FF000410AB10A46002100F07AB90D484FF08041F6E70B484FF489
:200CC0008021F2E709484FF40021EEE707484FF40031EAE706481021E7E705482021E4E7D6
:200CE000704700BF0078004000100140E8440258F044025870B50026046E0546314620467C
:200D000084F87860FFF70EFD31462846FFF7AAFFD4F88C20136823F00D031360D4F8900015
:200D200000F00CFCD4F8940000F008FCD4F89C0008B100F003FCD4F8980018B1BDE87040D5
:200D400000F0FCBB70BDFFEC38B5046E002201210546D4F88C301A60FFF784FFD4F890000F
:200D600000F00AFBD4F8940000F006FBD4F89C0008B100F001FBD4F8980028B120F440206F
:200D800040F4802000F0F8FAD4F88C2094F87C10536823F47D5309B143F400535360284606
:200DA000D4F88C20104B11680B401360D4F88C2094F87910936823F4E06323F0010343EA03
:200DC00041639360FFF7CCFCD4F88C200020136843F0005343F00D0313600123A4F874003B
:200DE00084F8783038BD00BF03BEFF3338B5084D002455F8040B10B10021FFF793FC0134CA
:200E0000082CF6D10348BDE83840FFF79DBF00BF04851608E00100247FB50D490D4801F0E2
:200E2000F3FA0D4968460D4D00F066FF00231C4655F8041B39B15E1C303368468DF80930EE
:200E400001F0E2FA33460134082CF1D104B070BDE0010024EC841608F9841608048516086B
:200E600013B504460DF106010948FFF75BFC0A2C02D10D20FFF7F0FBE0B2FFF7EDFBBDF881
:200E800006100348FFF73CFC204602B010BD00BFE001002430B4EFF3118400238022EFF318
:200EA000108372B682F3118883F31088BFF34F8F164B174AD3F80038118803F4807578B158
:200EC00001311180128875B1C2B10023BFF34F8FE4B284F31188BBB1042030BC00F07AB825
:200EE00051B10139EDE7002AEFD043F48073074AC2F800380123E9E7002DE6D023F48073AB
:200F0000024AC2F80038E0E730BC7047004002586C4B0024EFF3118200238021EFF3108306
:200F200072B681F3118883F310880749D1F8003823F48073C1F800380021044B1980D3B294
:200F400083F31188FFF7A6BF004002586C4B002470B5EFF3118500238022EFF3108372B6B3
:200F600082F3118883F310880E4AD2F8083880B143F001034FF47A740A4EC2F80838013CCB
:200F800003D3D6F80838DB0707D5EDB285F3118870BD23F001030446EEE7012000F01AF879
:200FA000EDE700BF0040025830B5EFF3118400238025EFF3108372B685F3118883F3108824
:200FC000036823EA0101E3B20A43026083F3118830BDFFEC82B000221C49B0F57A7F0BD832
:200FE000002242F22A51642811D800220A2818D8002208BB02B070470192019B8B4202DD3E
:20100000A0F57A70E9E7019B01330193F5E70192019B8B4201DD6438E5E7019B013301939B
:20102000F6E70192019BB3F56E7F01DB0A38DDE7019B01330193F5E70192019B5E2B01DD57
:201040000138D6E7019B01330193F6E7AD730100BFF34F8FBFF36F8F4FF0E0230022C3F8D9
:20106000502FD3F8142D42F40032C3F8142DBFF34F8FBFF36F8F70474FF0E022F0B5D2F8DA
:20108000803D03F00704C3F34E31C3F3C9030434B3FA83F505F01F05BFF34F8F184601FA7F
:2010A00004F700FA05F6013846EA0706C2F8606FF7D20139F2D2BFF34F8FD2F8143D43F498
:2010C0008033C2F8143DBFF34F8FBFF36F8FF0BD4FF0E02210B5D2F8844D44F00103C2F8D2
:2010E000843DD2F8803DC2F8844D03F007031C1D0123A340BFF34F8F5C1E044204D05C421E
:201100002040C2F8700F18444FF0E024C2188A420AD9884203D24FF0E023C3F8700FBFF341
:201120004F8FBFF36F8F10BDC4F85C0F1046EDE7F0B54FF0E026D6F8803D03F00700C3F3DE
:201140004E32C3F3C9030430B3FA83F404F01F04BFF34F8F194602FA00F701FA04F501390E
:2011600045EA0705C6F86C5FF7D2013AF2D2BFF34F8FBFF36F8FF0BDF0B44FF0E0260F1AE4
:201180000124D6F8802D02F007031D1DC2F34E33C2F3C9020133AC40AB4002FB03339F42A4
:2011A00002D3F0BCFFF7C4BF63421840BFF34F8FC6F8680F20448142FAD8BFF34F8FBFF338
:2011C0006F8FF0BC7047FFEC37B50A4D0C462B680BB91C462960019000F0AAFA296801989D
:2011E00001F088FE14B900232C682B60204603B030BD00BF704B0024EFF3148343F0040312
:2012000083F314884FF0E023D3F8342F22F04042C3F8342FD3F8882D42F47002C3F8882D02
:201220007047FFEC024B1878421C1A70704700BF6E4B002410B50523012404FA03F1DAB264
:20124000814201D3104610BD0133202BF5D11A46F8E7FFEC072A1BD901231F2A03FA02F3E1
:20126000A2F1030203F1FF3300EA030094BFDB106FF060430144194421EA030120EA0303C2
:20128000D140D340034A505C034AD35C1843704700207047618516085885160830B10029C3
:2012A0000CBF012003200AB140F004004FF0E023C3F8940D70472DE9F04780461446FFF778
:2012C000B1FF054608EB010628F01F0A89464FF0E027A6EB0A00FFF7ADFF4FF0FF3303FA18
:2012E00000F000EA0A0AA6EB0A00FFF7A3FFC7F8985D45EA0A0506460246494645F010056E
:201300004046013EC7F89C5DFFF7A4FF000244EA460480B2044344F00104C7F8A04DBDE83A
:20132000F0874FF0E0230022D3F8900D1146C0F30720904202D1C3F8941D7047C3F8982DF1
:201340000132C3F8A01DC3F89C1DF2E702064FEA10130CD403F00F03064A52F8232032B18C
:2013600000F00F00012319B103FA00F0906170471030F9E76C8516082DE9F0470509044617
:20138000C0F3031715F0080540F0D2806A4B53F82760002E00F0CC8000F4402300F00F089D
:2013A000B3F5002F00F0B180B3F5402F00F0AF80B3F5802F40F0AD80C0F30021FFF7C6FFBC
:2013C0000121EFF3118200238020EFF3108372B680F3118883F31088022940F09C8014F47D
:2013E000704FC4F3033017D023074FF00F094BBFA8F1080343464FF0240C4FF0200C9B0030
:201400005CF806E009FA03F900FA03F32EEA090E43EA0E034CF806304FEA48090323D6F83E
:2014200000E0032903FA09F32EEA030E6FEA030C01FA09F343EA0E0333606ED004F44033A5
:20144000B3F5803F6BD0B3F5003F0CBF02230023D6F80CE003FA09F30CEA0E0E43EA0E03ED
:20146000F36080B923074FF00F0A4BBFA8F108034346242020209B0050F806E00AFA03F3E0
:201480002EEA0303835101F1FF3EBEF1010F0DD804F44065B5F5006F43D0B5F5406F42D053
:2014A000A5F5806ADAF1000545EB0A05B36805FA09F50120BEF1010F0CEA030C00FA08F0AA
:2014C00045EA0C05B56073682FD8A5052DD503430129736013D0E30511D504F00C044FEAF8
:2014E00088030F2004F1B04403F00C03D4F8081498409F4021EA00010F43C4F80874D2B28E
:2015000082F311880020BDE8F087022159E7032157E7294655E700207EE7002398E70123C6
:2015200096E70225C2E70325C0E723EA0003CFE76FF01500E7E700BF6C851608C0B2FFF751
:201540001BBFFFEC02064FEA101310D403F00F03084A52F8233053B11A6900F00F000123E0
:2015600003FA00F0104214BF1846002070470020704700BF6C8516080F2810B531DDA0F1E4
:2015800010041F2C0ADC03F1604303F561430B60012303FA04F4146000201CE03F2C08D874
:2015A0001C4C30381C440C60012303FA00F01060F2E75F2C04D8184C50381C440C60F3E73C
:2015C0007F2C04D8154C70381C440C60ECE7952C02D94FF0FF3010BD114C90381C440C6014
:2015E000E2E7104B04280B6003D14FF480331360D2E7052802D14FF40033F8E7062802D1E4
:201600004FF48023F3E70F28E3D1074B0B600123EDE700BF04E100E008E100E00CE100E050
:2016200010E100E024ED00E010E000E013B5802301AA69460446FFF79FFF20B90F2CDDE99B
:20164000003102DD196002B010BD1A6822EA01021A60F8E713B5002301AA69460446FFF713
:201660008BFF20B90F2CDDE9003102DD196002B010BD1A680A431A60F9E7FFEC08B54FF0EE
:20168000E02324494FF0FF305B6803F00F035A1C03F1382361339B0041F8040B8B42FBD1CF
:2016A0004FF0E0231C49C3F8081D4FF08031C3F8181DC3F81C1DC3F8201D5301174A03F12E
:2016C000604303F5644342F8041B9342FBD1144B002214490B201A6001F0E4FB00221249FE
:2016E000032001F0DFFB4FF0E02100220420D1F81C3D23F07F4343F0E043C1F81C3D0B49C3
:2017000001F0D0FB0420FFF7A5FFF02383F3118862B608BD80E100E00000020800E400E041
:20172000704B00243919020835170208391802087047FFEC2DE9FF414FF0E02305460E46E4
:201740001746D3F82C4DD3F8288D63000FD5304A0020304900F0E8FA5FFA88F33BB13A46FC
:201760003146284604B0BDE8F04100F065B8284A0020294900F0D8FA2B46254A00202749B7
:20178000009600F0D1FAEFF31183EFF31082EFF30581EFF31480D2B2DBB200921C4ACDE971
:2017A00001101F49002000F0BFFA4FF0E0230020D3F8302DD3F8381DD3F83C3DCDE9004201
:2017C000CDE90213124A4346164900F0ADFA00200F4A154900F0A8FA14F0020013D00C4ABB
:2017E0000020124900F0A0FAEFF3118300238022EFF3108372B682F3118883F31088AD2122
:201800000B4800F0CDF9002CEEDA014A0949E9E7B98616088C851608A8851608C285160822
:20182000D9851608148616085186160869861608A18616088F86160870B586B04FF0E0255B
:201840000E46314A059000203049D5F8284D00F06BFA059B00202C4A2D49009600F064FA64
:20186000D5F8283DD5F8342D00202A490092264A00F05AFAEFF31183EFF31082EFF30581DD
:20188000EFF31480D2B2DBB200921F4ACDE901102149002000F048FA1B4A2049002000F065
:2018A00043FAE50704D5184A00201D4900F03CFAA00704D5144A00201A4900F035FA210770
:2018C00004D5114A0020184900F02EFAE20604D50D4A0020154900F027FAA30604D50A4ABE
:2018E0000020134900F020FAEFF3118300238022EFF3108372B682F3118883F310886521E8
:201900000C4800F04DF900BF19881608C7861608EE86160808871608D985160825871608CF
:201920004A8716086D87160889871608AD871608CF87160802881608CA6E012A08B508D012
:20194000022A0AD01AB9D422086F00F021F8002008BD0A6F034B1A60F9E70A6F11604A6F8F
:20196000F8E700BF704B0024FFECC2925D7D05C518DF88DFCD06CD767CD30CD3D982D9121F
:201980002C00050A0F14191E232800BFAFF3008000B501B400F004F801BC00BDAFF3008094
:2019A00000B5042A60DB00F0030E61F3830E7A4BD3E80EF0AFF30080AFF30080AFF300803F
:2019C00011F8013B00F8013BA2F1010211F8013B00F8013BA2F1010211F8013B00F8013B70
:2019E000A2F101022DE9F01F282A07DBB1E8F81FA0E8F81FA2F12802282AF7DADFF89CE175
:201A00004FEA920BDEE80BF051F8043B40F8043B26E0B1E81800A0E8180021E0B1E8380007
:201A2000A0E838001CE0B1E87800A0E8780017E0B1E8F800A0E8F80012E0B1E8F801A0E8C5
:201A4000F8010DE0B1E8F803A0E8F80308E0B1E8F807A0E8F80703E0B1E8F80FA0E8F80F70
:201A6000BDE8F01F02F00302002A08BF00BD11F8013B00F8013B013A08BF00BD11F8013B90
:201A800000F8013B013A08BF00BD11F8013B00F8013B00BDAFF30080AFF30080AFF30080B7
:201AA00011F8013B00F8013BA2F1010211F8013B00F8013BA2F1010211F8013B00F8013B8F
:201AC000A2F10102282A35DB2DE9F01FB1E8F81F20F8023B4FEA134364F31F434FEA14440B
:201AE00065F31F444FEA154566F31F454FEA164667F31F464FEA174768F31F474FEA184896
:201B000069F31F484FEA19496AF31F494FEA1A4A6BF31F4A4FEA1B4B6CF31F4BA0E8F80F47
:201B20004FEA1C4C20F802CBA2F12802282ACDDABDE8F01F042A97DB51F8043B20F8023B38
:201B40004FEA134320F8023BA2F10402BAE711F8013B00F8013BA2F1010211F8013B00F81B
:201B6000013BA2F1010211F8013B00F8013BA2F10102042AFFF678AF51F8043B00F8013B7E
:201B80004FEA132320F8023B4FEA134300F8013BA2F10402EDE7000070190208801902081B
:201BA00008B508F053FB012000F004F8002008B500F006F9044608B500F033F8204602F0CF
:201BC0003BFA2DE9F0410E468046174600F0DCF804461EB300F0D8F801F01AFB002809DB61
:201BE000E36B002B10DD4FF0FF3500F0CDF801F06BFB06E000F0DAF80368002BC3F1000509
:201C0000EEDD2846BDE8F0810C2505FB03450133C5E91086AF640025E363E6E74FF0FF35C6
:201C2000EFE7F8B5064600F0AFF80C230446C06B0027451E03FB0044002D00DAF8BDD4E955
:201C40000D23E16BC4E90E7713B1012A03D19847013D0C3CF0E7022A02D130469847F7E7A5
:201C6000032AF5D108469847F2E7002A43D010F0010F034639D0013A03F8011B012A38D93E
:201C8000F0B541EA01259E07ADB22BD0023A23F8025B032A18D95C0745EA054616BF141F98
:201CA000144643F8046B224603EB040C072A13D8E2086FF0070707FB02423C40032A2344F1
:201CC00084BF043A43F8046B012A02D9023A23F8025B02B11970F0BDACEB0207083AC7E9A4
:201CE0000066E3E7032AD6D8F0E7012AC8D1197001E0002AFBD17047421E11F8013B02F888
:201D0000013F002BF9D17047064B07B51B780341DB0703D5019201AA00F0D0FD03B05DF836
:201D200004FB00BF640400240EB403B503AA52F8041B0192FFF7E8FF02B05DF804EB03B0B0
:201D40007047FFEC0E4B002230B5D3E900548C4209D1C561836823F4805323F00F0319434D
:201D60008160002030BDA94202D1C1612146F1E7013208331F2AE8D1C1614FF48051E9E7E0
:201D800028881608C069704708B500F002F8006808BD1FB5002001A901F0BAF90028ACBFEC
:201DA0000298002005B05DF804FBFFEC08B5FFF7F0FF08B1143008BD0048FCE7744B002403
:201DC00007B5019000F003F8019801F0C3F82DE9F041FFF7D9FF05460024FFF7DAFF4FF0F4
:201DE00001082F7B061D103508FA04F31F4206D056F8240018B155F8243003B198470134F4
:201E0000042CF1D1BDE8F08113B50446E36D20460191DB6A984701990028F7D0E36D2046FD
:201E20005B6A02B0BDE8104018472DE9F74F858F0446B0F9403088462DB24FF0800B0192FA
:201E40000135AB42D8BF0025E38F1BB2AB420AD0A38F2DB2626C00201BB202F80380A58728
:201E600003B0BDE8F08F019B002B30D0EFF3118AEFF3108772B68BF3118887F31088E38F0B
:201E80001BB2AB421ED1E27802F0FF09E2B90121E26D20466170926A904704F11C0001F02D
:201EA00075F9E26D06464946926A204690475FFA8AFA8AF31188E37863B9002EC4DA6FF0BC
:201EC0000300CDE70026F2E76FF07F06EFE76FF00A00C5E76FF07F00C2E72DE9F74F8368AF
:201EE00080460E4601925C6904F14809484601F04DF9051E2FDB00254FF0010B019B9D424D
:201F000004D2E3785BB30DB96FF07F05E36D012120469B699847B4F85020B4F8523012B210
:201F20001BB29A42B4F95420C0F29D80B4F85010B4F8523009B21BB2C91A0A2392FBF3F2C4
:201F4000914205D8E36D1B6A13B1002220469847484601F06BF9284603B0BDE8F08FB4F8FD
:201F60005230B4F8502019B212B28A421FD0A26D0133525C1BB2B4F954109942D8BF002315
:201F8000A4F85230A36813F4E07F05D00A2A07D113F0400F18BF0D22013506F8012BADE785
:201FA0000D2AF9D113F4807F18BF0A22F4E7002DACD1D8F80830002B4FD0D8F8005015F01B
:201FC00040054DD1EFF3118A8023EFF3108772B683F3118887F31088E26D294620465FFA3F
:201FE0008AFA92699047B4F85010B4F8522009B212B2914229D1E26D01212046926990476C
:20200000B4F85010B4F8522009B212B2914202D08AF3118872E7E278A2B904F1240084F8B9
:2020200002B001F0B3F88AF31188002803DBE378002B3FF463AFE378002B7FF465AF6FF0FF
:20204000030563E76FF07F00EDE78AF31188E36D012120469B69984750E76FF0500555E784
:202060006FF00A0552E7B4F85230B4F850101BB2D31A03FA81F160E72DE9F04183685E6916
:2020800006F11405284601F081F8041E23DBF378002B36D13378013313F0FF0734D0012F7F
:2020A0002DD1EFF3118800238022EFF3108372B682F3118883F3108833795FFA88F86BB980
:2020C000F36D30461B689847041E07DA88F31188284601F0ABF82046BDE8F081F36D30465D
:2020E0009B689847041EF36D03DA5B6830469847ECE79B6901213046984788F3118837707E
:20210000E6E76FF07F04E3E76FF01704E0E7F7B50E4600F1640700F1740557F8044B8CB164
:202120006368A26843F0180333401343A3604BB101A920690AF05CFB019B002B02DC206902
:2021400001F074F8AF42E8D103B0F0BD2DE9F84383680E4615465C6904F12C08404601F0C8
:2021600015F8071E51DB002D52D004F16402002352F8045B002D37D104EB8302193304F1A1
:20218000340904EB830356664846736101F038F8A38FB4F940201BB201339A42D8BF002378
:2021A000E28F12B29A4227D1484604F1480901F03DF8484601F024F8B4F85020B4F8523037
:2021C000484612B21BB29A421EBF736803F001031D4301F02BF8E37893B145F01805294681
:2021E0002046FFF794FF0DE00133042BC0D100236FF00F07736105E0756805F00405D3E729
:20220000002DECD1404601F011F83846BDE8F8837369002BF6D01D607561F3E72DE9F0476F
:20222000836880460F4616465D69464B1B6823B1EB78ABB16FF07F0425E000F05DFF002874
:20224000F6D105F1340A504600F0A0FF041E1ADBEB7803F0FF018BB3504600F0E7FFE9E777
:20226000EFF3118400238022EFF3108372B682F3118883F3108807EB0608B84506D1E4B2FF
:2022800084F3118834462046BDE8F087EB6817F8011BD80703D50D2905D11A0705D4284689
:2022A000FFF7B2FDE9E70A29F9D113F0240F03D00D212846FFF7A8FD0A21F0E7D8F800207A
:2022C000B146EB6D284682F040089B6AC8F380189847B9F1000F01D1344623E0EB6817F8E6
:2022E000011BD80703D50D290AD11A070AD442462846FFF79AFD041E10DB09F1FF39E8E76A
:202300000A29F4D113F0240F01D10A21EFE742460D212846FFF789FD041EF6DAB14501D261
:20232000A6EB0904AA8FEB8F12B21BB29A4204D0EB6D012128469B6A9847504600F076FF44
:20234000A1E700BF704B00242DE9F04700F1340804460E46404600F019FF051E1DDBEFF3B4
:20236000118700238022EFF3108372B682F3118883F31088E37803F0FF0553B3A38F6FF05E
:202380007F05E387FFB287F311881E4F002DD7F800902CDA404600F049FF2846BDE8F08744
:2023A000E36D0121204684F801A09B6A9847484600F0ECFEE36D054600219B6A20469847D6
:2023C000002DDFDBA28FE38F12B21BB29A42E7D1D8E74FF0010A04F11C09F3E74FF47A7024
:2023E00001F0A4FB3B68A3EB0903B34206D2E36D20461B6B98470028F0D0CBE76FF07305B7
:20240000CBE700BF844B00242DE9F0410B7905460C462BB10B6943F001030B610523CB60AA
:202420000122002104F1340004F11C070AF0C5F90122002104F148000AF0BFF901220021E8
:2024400004F114000AF0B9F90022384604F1240611460AF0B2F90022304611460AF0ADF97D
:202460000122002104F12C000AF0A7F90021384601F0E3F80021304601F0DFF823462846BC
:202480004FF4DB720249BDE8F04100F068BA00BF2089160810B504460121FFF738FEA3787B
:2024A0003BB1002304F12400A370BDE8104000F0BDBE10BD10B504460421FFF728FE637889
:2024C0003BB1002304F11C006370BDE8104000F0ADBE10BD70B583680E4615465C69E36D18
:2024E0001B695BBB40F207339E422ED0B6F5427F1CDAB6F58A7F00F08E8040F215139E42AA
:2025000000F0AD806FF0180040F201139E4200F0AC80B6F5817F10D1002D00F0AE802B687B
:20252000A3606B68E360EB6823612CE037D040F209339E424FD06FF0180070BD984710F1A7
:20254000190FCFD00028DFD0F7E7EFF3118100238022EFF3108372B682F3118883F310880D
:20256000B4F85220B4F8503012B21BB29A420CDCB4F85030B4F852201BB212B29B1ACAB2B0
:2025800082F311882B600020D7E7B4F85220B4F8500012B2B4F9543000B2121AEEE7EFF320
:2025A000118100238022EFF3108372B682F3118883F31088E28FA38F12B21BB29A4203DC1C
:2025C000A38FE28F1BB2D8E7E28FA08F12B2B4F9403000B2E1E7EFF3118100238022EFF3B6
:2025E000108372B682F3118883F31088A28FE38F12B21BB29A4206DAE38FA28F1BB212B2E0
:202600009B1A013BBBE7A28FE08F12B2B4F9403000B2121AF4E7EFF3118600238022EFF3CD
:20262000108372B682F3118883F3108835F0020209D1B4F85030A4F85230E36D1B6A13B1DD
:20264000114620469847013D012D04D8A38F2046E387FFF72FFFF6B286F3118893E742F208
:2026600010712046FFF770FE67E735B1A3682B60E3686B602369EB6085E76FF015005CE735
:2026800070B504460D46EFF3118600238022EFF3108372B682F3118883F3108881F001030C
:2026A000C37089B91821FFF732FD637823B104F11C00657000F0BAFDA3782BB1002304F1FC
:2026C0002400A37000F0B2FDF6B286F3118870BD10B5044600211C3000F003FE002104F1BA
:2026E000240000F0FEFD012104F1340000F0F9FD012104F1480000F0F4FD04F12C00012117
:20270000BDE8104000F0EDBD70B5836805465C6904F11406304600F073FD2378012B06D97F
:20272000013B2370304600F081FD002070BD0021E36D204621709B6998472B685B0604D482
:202740004FF47A612046FFF7FFFDEFF3118500238022EFF3108372B682F3118883F310880D
:20276000E36D2046DB68984723791BB9E36D20465B689847EDB285F311882046FFF78AFE25
:202780002046FFF7A5FFCDE7F8B5002504462F46A28FAEB2E38F12B21BB29A4210D1A28F72
:2027A000E38F12B21BB29A4204D1E36D002120469B6A9847EEB12046BDE8F840FFF77ABE9A
:2027C000E36D2046DB6A98470028E8D0E38F2046616C1BB2E26DC95C526A9047E38FB4F9A7
:2027E000402001331BB29A42E38700DCE7870135CEE7F8BD2DE9F743B0F850505A23B0F98A
:20280000546004462DB200270135AE42D8BF002516FB03F6642396FBF3F61FFA87F9E36DDE
:202820002046DB69984700283FD0B4F85280B4F85020B4F852300FFA88F812B21BB29A421A
:202840001FDBB4F85010B4F8523009B21BB2C91AB14221D2E36D01A920465B699847454566
:20286000DDD0B4F850300137A26D1BB2D0542BB20135A4F85030B4F95430AB42D8BF00253E
:20288000CBE7B4F85230B4F850101AB2B4F954309B1A03FA81F1DBE7E36D1B6A002BD9D0C0
:2028A0000122204698470028D4D0B9F1000F02D02046FFF7EFFD03B0BDE8F08310B586B04B
:2028C000144602A8019100F019F82268019902A80AF088F806B010BD0D2938B504460D46D6
:2028E00007D0284600F016F8031E03DBE3680133E36038BD0433F4D0FBE7FFEC034B036066
:20290000034B83600023C360704700BFD9280208FDDD020838B50A4B04460A4D1B683BB981
:2029200000F0EAFB20B9286840B103681B6803E0286818B103685B6821469847204638BD6F
:20294000704B00246C04002410B514460846114607F020FE204610BD0846FEF781BAF0B5D5
:2029600085B007460E461D46019200F01BF8041E12DB03AA0199384600F07AF8041E09DB4C
:20298000039B0024DA8922F00F0242F00102C3E90465DA8100F028F8204605B0F0BD00F082
:2029A0005BB8FFEC38B50F4C01F038FB0546A368984204D1A38900200133A38138BD2046A9
:2029C00000F026FC002807DAFFF7F0F900680428F5D08C28F3D040420028EFD10123A5609A
:2029E000A381EBE77004002408B501F017FB0A488389012B0CD1002383814FF0FF338360A7
:202A000000F062FC002805DABDE80840FFF7CEB9013B838108BD00BF7004002410B503468D
:202A20000446184613F8012B2AB9001B1C3009F063FA18B910BD2F2AF3D1F6E700F1180373
:202A4000013C14F8012F12B900221A70F2E72F2AFAD003F8012BF4E708B50348FFF7DEFFAD
:202A6000024B186008BD00BF61C71B08784B002400232DE9F04116461360027888B0002AC6
:202A800045D08DF81C30CDE9010301A8CDE90333CDE9053300F04CF8002835DA019FDDE942
:202AA0000354384600F036F8037880463846D3B1FFF7B4FF48B96FF00B04069808B109F078
:202AC00003FA204608B0BDE8F0813DB16B68C0E900436860474604460025E2E7A368C0E9D7
:202AE0000043A060F6E7FFF799FF0028E3D035B16B68C0E90043686000243060DDE7A3685D
:202B0000C0E90043A060F7E76FF01004D5E76FF01504D6E7017803460246013031B12F2912
:202B2000F8D11346013219782F29FAD018467047F8B5036805461B782F2B11D004462C4889
:202B400000F0CCF82B4A54F8143B002818BF02462949204609F0FBFE6B69002B41D02B6005
:202B6000264B28681C6803782F2B3DD1002637464CB922466FF001032A61C5E90004C5E98F
:202B800002761846F8BD04F11701431E11F801CF13F8012FBCF1000F0FD10AB12F2A17D190
:202BA000FFF7B8FF0378BBB1E38903F00F03032B14D0A368264600240BE022B12F2A02D07A
:202BC000944505D3E2D900246FF001032246D3E7636827461C46CBE70246CDE7024600232D
:202BE000CAE76FF00B03CCE76FF01503C9E700BFADAC1608E648180854891608784B002477
:202C000030B58DB000230546694601A8009307F0D1F9041E05DB01A80BF076FB009B28603E
:202C20006B6020460DB030BD37B50346114CC8B122460068596803C268460F4D00F030F836
:202C40002268009B0199D21A63685B1A002122606360002B02F1FF3008DB09B1C4E9002369
:202C600003B030BD2046FFF7CBFFE5E72B4402460121EEE77C4B002400CA9A3B08B507F0D6
:202C800039F807F0A1F80020BDE80840FFF7CCBF024A136801331360704700BF844B00240E
:202CA0000C4B4FF47A7270B500251E68044600233046294614F0AAFE294620604FF47A72A2
:202CC0003046002314F0A2FE034B28465A43626070BD00BF844B002440420F0038B50446F5
:202CE00018B300F0CBF9124B1B689D688DB12146284601F0C7FA041E0CDB2B6C3D2153F862
:202D000024000BF09DF968B1441C00F0C7F9204638BD2C4600F0C2F96442FFF747F804601E
:202D20000024F4E76FF01504F4E76FF01504F3E7584C00243F4C01233F4DA82204F18C069B
:202D40002B7083B500212046FEF78FFF032318223A49237730463A4B3A4FC4E90533062387
:202D6000A3860BF081F9384920463E6009F0B5FC364B374E1C6002232B7000F0D9FA01A9D7
:202D8000684606F08DFFDDE9000109F087F8042333603368012B49DD3068800009F0ACF868
:202DA0002C4B186033680460224894F8341001F013FBA3681F489B6A9F6007F039FD1D48E4
:202DC00001F048F91B4801F035FBA36805221A720022214B1A6003232B7000F04FF90CF082
:202DE000DAFE1E4B0BB101F085FB1D4B0BB1FFF745FF1C4B0BB101F06DFD02F035FB07F070
:202E0000AFFB0BF012FF04230A482B7034F1CAFE084801F03FFB05232B7000F025F8062387
:202E20002B7000F03BF907F001FDFCE733685B00AEE700BF904B0024484C00245A891608F9
:202E4000352D0208884B0024584C0024604C0024444C0024544C0024404C0024F54402080C
:202E60007D2C0208D548020813B5002401220949094801F01FFA01F099F901F0A3F9074B5A
:202E800040F67A4264210094054800F08EFE204602B010BDE6481808ADAC1608D154020885
:202EA000A4891608A52870B505460C461AD8EFF3118600238021EFF3108372B681F311885F
:202EC00083F310881CB9FEF7B1FB2246074C0848F6B240F8354000EBC500426086F31188AA
:202EE000002070BD6FF01500FBE700BF312F0208004F0024A52808B50CD8094A52F8303028
:202F00005BB102EBC00252689847064B1A68064B1A6008BD0022054BF6E71A46FBE700BFAA
:202F2000004F0024584C0024604C0024312F020808B5EFF3118300238022EFF3108372B687
:202F400082F3118883F3108836210148FEF728FEAD8916080E4B37B504461D684FF0FF33C1
:202F6000002201A90320019300F090FB01F03CF8214600F033F8044610B10120FEF71AFE73
:202F800002460146284600F0F1FF204607F0C8FA584C002470B500230C468E68016A39B188
:202FA0008D680A68AE4210D1A3B98AB9C0E9083304F1140000F0CEF804F10C0000F0CAF8E4
:202FC0002046BDE8704008F07FBF0B461146E6E70262EDE702B943621A60E9E7F7B50446B3
:202FE0000F4600F0FAFF00F118060546304600F007F92146284600F038F8044630B9304635
:2030000001F097FA4FF0FF3003B0F0BDC761012300F10C0701A98371384609F0E9FB0146D0
:2030200030B16379E3B121462846FFF7B3FF17E0019A002AF5DA14340132204609F0BDFBA5
:20304000384601F076FA18B901A9384609F0D0FB019B002B01DA0028F2D0204600F0D0F82A
:20306000304601F066FA0020CEE7006A10B183688B4200D170470068F8E7FFEC054B1B6844
:203080002BB1054A126812B9DA8E0132DA860020704700BF584C0024704B0024134B10B565
:2030A0001A68C2B1124B1B68ABB9EFF311848021EFF3108372B681F3118883F31088B2F95C
:2030C0003630002B09DC0023D3860A4B1B6853B9E4B284F31188002010BD013B9BB2D386A5
:2030E000002BF5D1EFE707F061FAF1E7584C0024704B00244C4C0024044B1B6823B1186856
:20310000B0FA80F04009704701207047584C002438B50F4B0C461D6870B101F055FAA0B125
:20312000AB8E03F00303022B07D0AA6883689A4203D06FF00C0007E02846C36C2360036DCB
:203140006360436D0020A36038BD6FF00100FBE7584C002408B540B103881B0401D4012389
:20316000038000F0C9F9002008BD6FF01500FBE710B5FFF7EFFF041E05DA6442FEF716FE86
:2031800004604FF0FF34204610BDFFEC1B4B70B504461D68EFF3118600238022EFF310832E
:2031A00072B682F3118883F3108820B303881BB2002B038803F1FF331BB2038008DD00246B
:2031C00000F0D8F9AC65F6B286F31188204670BDA865FFF753FF204600F0D4F9002305210F
:2031E00028462B8707F03EF9B5F9384004B16442FFF754FFE7E76FF01504E4E7584C0024DE
:2032000010B504462046FFF7C1FF031DFAD010BD10B5FFF7BBFF041E06DA6442FEF7C6FDF7
:2032200004604FF0FF3010BD0020FCE770B50546002844D0EFF3118600238022EFF310838D
:2032400072B682F3118883F31088038847F6FF721BB2934205D1F6B286F311886FF08A00D6
:2032600070BD00F099F92B8801331BB22B80FFF705FF2B881BB2002B15DC124B1C689CB17C
:20328000A36DAB420DD12946204600F04BF904F13C0000F0EDFE00232046A36507F024FA98
:2032A00002E02468EBE700242946204600F098F9F6B2FFF7F3FE86F311880020D0E76FF07D
:2032C0001500CDE76C4C002410B5FFF7AFFF041E05DA6442FEF76AFD04604FF0FF342046A1
:2032E00010BD70B505460C46FFF7C8FEEFF3118600238022EFF3108372B682F3118883F324
:2033000010882B881A0409D42B881B040ED5F6B286F31188FFF7C2FE002070BD002CF3DDF9
:20332000013C2846FFF782FF24B2EAE72C80EEE700F0CEB8CB6803F130021B6B1BB18B4255
:2033400012D14B6813600023021DC1E90133CB600B8243681BB18B4209D10B681360054B38
:203360001A6819600A6070471A1D5B68E6E71A461B68EFE77C4C002408B503460846B3F9C5
:203380001020002A04DC1946FFF7D4FF012008BD0020FCE708B50B4601461846FFF7CAFF70
:2033A000002008BD10B5C068117C90F82E3099420ED9047CA1420DD9A34206D2437F0F2B04
:2033C0009FBFC11801338C774377117C01F050F9002010BD437F0F2B9FBFC21801339177A1
:2033E0004377F5E70346084670B51546B3F91020DC68002A02DC1946FFF79CFF227C94F8DE
:203400002E108A4204D0637F23B9204601F07AF9002070BD297C8A4210D904F11E0000226A
:203420009342F5DD10F8015BA94220D1013B1FBFE1181219897F91776377E9E704F11F0693
:203440000020012225189342A97F09DC013B20461EBFE218927FAA77637701F009F9D7E7D4
:2034600016F8015B8D4288BF10460132EAE70132D6E7FFEC054B10B51B68C4689C4203D121
:20348000FFF7B0FF012010BD0020FCE7584C0024064B10B41B68C4689C4203D05DF8044BB5
:2034A000FFF7A0BF00205DF8044B7047584C0024F8B504460D4617464068002300B103B19D
:2034C000F8BD06683A462146A84703463046F5E7074A0021074B1A6002F11403013143F8A3
:2034E000143C14331F29F9D10023C2F86C327047804C00247C4C002410B5EFF311840023B6
:203500008022EFF3108372B682F3118883F3108800220349E4B2FFF7CBFF84F3118810BDAF
:2035200095330208036830B5DBB18B78DB0718D44C682346B3B90E4A136893B11D681C606B
:20354000156000224B601A82C3E90210026B5A600363B3F9102047F6FF718A4201D00132E9
:203560001A8230BDDA689042F3D01B68E2E700BF7C4C0024024B01461868FFF7D3BF00BF99
:20358000584C0024024B03491A68FFF791BF00BF584C0024A53302080C4B002210B5114604
:2035A0001C68436833B9012A02BF0B8A03F1FF330B8205E0D968A14203D11A8A013A1A8264
:2035C00010BD194601321B68ECE700BF584C0024024608460149FFF76BBF00BFE5330208CE
:2035E00013B502460C46A0B10B4B1B6823B102B0BDE81040FFF7ECBF084901902046FFF7E5
:2036000057FF019A0649204602B0BDE81040FFF74FBF0449F7E700BF704B002491340208C1
:20362000753402087933020810B50446216B01B910BD8868FFF77EFEF8E7012910B50C467D
:203640000AD002290ED081B9827842F001028270FFF752FF204610BD8278002422F001027F
:203660008270F7E76FF08504F4E76FF01504F1E710B5FFF7E2FF041E05DA6442FEF796FB9E
:2036800004604FF0FF34204610BDFFECF8B51746194B06460C461D68FFF7F0FC0FB1EB6DAB
:2036A0003B60D4B1EFF3118300228021EFF3108272B681F3118882F31088022E11D0032EB9
:2036C00014D0012E14D1EA6D21680A430024EA65DBB283F3118800F011F8FFF7DFFC204686
:2036E000F8BD2168EA6D22EA0102EFE72268EDE76FF01504ECE700BF584C0024184B30B5D8
:203700001D6885B0FFF7BAFCEC6D284601F040F9E4430440039424B9FFF7C0FC204605B0A6
:2037200030BD03A800F070F8431C014610D0019003A809F081F80199284600F013F8044618
:2037400030B1011D284600F06FF8204600F02EF8039B002BE5D1FFF7A1FC0120DFE700BF71
:20376000584C002438B58368EFF3118500228020EFF3108272B680F3118882F3108800209A
:203780005C6B74B122798A4206D103F1340130B9084608F07DFF04E020462468F1E708F085
:2037A00081FFEDB285F31188204638BD10B5037B83B9EFF311848022EFF3108372B682F3D4
:2037C000118883F310880E4908F02EFFE4B284F3118810BD022B0CD1EFF31184002380220D
:2037E000EFF3108372B682F3118883F310880549EAE7012BEDD1BDE8104008F065BB00BF3B
:20380000505400244854002438B5054601242146284609F022F820B90134202CF7D14FF07A
:20382000FF34204638BDFFEC2DE9F0410D460978044629B35C3009F010F8012807467ED17C
:20384000EFF3118600238022EFF3108372B682F3118883F31088237FF6B2062B12D1297872
:2038600004F1600008F0F9FF60B12B68204663676B68A3670023236606F036FF86F3118869
:203880000026B4E086F31188A4682978EFF3118200238020EFF3108372B680F3118883F358
:2038A0001088636B13B11879884208D1D2B282F3118833B12A685A606A689A60E0E71B68D2
:2038C000F0E7564B1B68FBB1554808F0E1FE20B9544808F0DDFE0028D2D02B6843606B68B2
:2038E0008360EFF3118500238022EFF3108372B682F3118883F3108804F13401EDB208F02E
:2039000093FE85F31188BBE7EFF3118600238022EFF3108372B682F3118883F310884048E4
:20392000F6B208F0B5FE86F311880028D5D1102008F0D2FA0028A3D001230373CDE7FFF781
:203940009DFB2978A06801F03FF8064600282CD0406848B301F04AF800284BD073684360F7
:20396000B2688260F3689B0604D4297801238B40134383602B68C3606B680361EFF3118648
:2039800000238022EFF3108372B682F3118883F3108804F16401F6B208F046FE224920469A
:2039A00006F08CFF86F311880026FFF777FBEFF3118800238022EFF3108372B682F31188FB
:2039C00083F31088237F062B08D12B68204663676B68A3670023236606F086FE5FFA88F88E
:2039E00088F31188002F08D001DA6FF015063046BDE8F0816FF00B06D7E7237F052B03D1F7
:203A00000421204600F043FF237F072BEFD12B78082BECD1204600F07FFEE8E7704B002441
:203A200050540024485400244D3A020807B5019100F0CAFD28B1019903B05DF804EBFFF708
:203A4000F3BE6FF0020003B05DF804FB2DE9F04F87B00446FEF7AAF903684FF0800904F1B7
:203A6000640A019304F16C08B4F938300293EFF31183039FEFF3108772B689F3118887F3E9
:203A80001088A28E0397DFB212F400720AD087F31188FEF78BF9019B0360029B238707B058
:203AA000BDE8F08F5046059208F0F2FD059A06460028ECD0A18E059241F40071A1864146E5
:203AC00008F0B2FDD4F85CB0B5684BEA0505E56587F31188736806F10C01059A307B9847A6
:203AE000EFF31183049A0593EFF3108272B689F3118882F3108804924146A28E304622F483
:203B00000072A286E26D554082EA0B02154085EA0B05E56508F0A6FD059BDBB283F31188B9
:203B2000FFF7ECFD304600F08DFFA0E707B568B1084A0021B0FBF2F302FB130000934FF46F
:203B40007A7358430190684600F0D8FF03B05DF804FB00BF40420F0070B586B00546A82012
:203B60000E46CDE9043208F0C7F90446D0B10021868603910C9902910B9901910A99DDE9EA
:203B800004320091294600F043F8051E05DA204608F09AF9284606B070BD2046E56800F0DD
:203BA0009FF9F7E76FF00B05F4E71FB5069C00920A46CDE9013400231946FFF7CDFF04B00A
:203BC00010BD13B5049C0094FFF7EFFF041E05DA6442FEF7EBF804604FF0FF34204602B0CB
:203BE00010BD1FB5079C0294069CCDE9003413460A460221FFF7B0FF04B010BD13B5049C05
:203C0000CDE9003413460022FFF7EBFF02B010BD2DE9F34790F8346088460546914631460D
:203C20001F46DDF828A000F0D7FB041E40DB0D9906F00306A86800F0D1FA041E11DB284697
:203C400000F044FC041E0CDB87B152463946284606F074FD041E05DB284600F0FBF9041E91
:203C600013DA57B1284600F0EBFB21E032465146284606F02FFC041EEEDA2B6D002BF1D0FE
:203C80003146284606F0B8FCECE70B9B49460A4A2846009600F0A8F8041EE2DB0C9A414699
:203CA000284600F0B1F8041EDBDB284600F0C2FB204602B0BDE8F087193F02082DE9F74F18
:203CC00004460E4601929946EFF3118700238022EFF3108372B682F3118883F31088DFF805
:203CE00000A1DFF80081DAF800500020D8F800300135394A116888420DDB1068C00008F075
:203D0000FBF8354A0546002847D1FFB287F311886FF00B003BE0012D1168B8BF01250139DF
:203D2000294053F821B003EB810EBBF1000F31D1CEF80040FFB2E560CAF8005087F31188A3
:203D4000019BF6B29DF8302059460320267402F00302667484F82E60C4E90539A38E23F0D4
:203D60006303134304F15C02A386FFF78FFC204684F81CB006F05CFDFFF780F91749204658
:203D800008F0ABFC04232377FFF788F9584603B0BDE8F08F01350130ACE711684FF0000C19
:203DA0000D4B490011601A68D8F8000002EBD272BCEB620F04DB08F087F8C8F8005092E777
:203DC00050F82C000CF1010C1A68C168013A0A4045F82200E7E700BF444C0024384C0024ED
:203DE000404C0024544C002410B49DF8044001945DF8044BFFF762BF13B501240094FFF7EB
:203E00005DFF02B010BDFFEC344B2DE9F74F002914BF8946994607460024154649461822C2
:203E20008C300AF045F9484687F8A4400AF038F9461C4DBB2C460234384606EB840106F076
:203E40002FFC06464FEA8408002844D000EB080AA8F10808B346043DC0F800A048460AF02A
:203E60001FF90446B044494601345046FDF744FF5444D8451BD100204AF8040CBA68926A2A
:203E8000966003B0BDE8F08F40F2011855F824000028D0D00AF004F90130FB6C06449E4218
:203EA00016D201344445F1D16FF00600E9E74BF8044F55F8041F084601910AF0F1F88146D5
:203EC0000199204609F10109FDF716FF4C44D0E76FF05A00D5E76FF00B00D2E7C58916088A
:203EE00038B50446EFF3118500238022EFF3108372B682F3118883F31088037F042B01D013
:203F000033F170FE2046EDB233F14CFE204606F0EBFB85F3118838BD38B5134B1C68A38E54
:203F200003F00303022B02D0204600F0F5FEA368012040F201119B6A9A6852F820304BB92B
:203F4000A38EA56903F00303022B08D11146A847FDF730FE01308842EFD10120F8E70146B9
:203F6000284608F01FFCF8E7584C002470B5838E0E460446190517D43AB9806828B1437ACB
:203F8000012B02D1543009F087FC204600F03AF8A56855B9204600F053FA204600F080FD09
:203FA000A38E43F40063A38670BDA38E03F00303012B03D06B690BB136021E606B7A012B60
:203FC000E8D1002305F10C066B61EB72AB891B04E0D53046FFF72AF9F8E708B500F0F4FAC3
:203FE00000B1806808BDFFEC054B186830B1037F032B01D1C06870476FF00200704700BF8F
:20400000584C002410B5044600F0B7FA204600F063F82046BDE8104000F018BC054B186888
:2040200030B1037F032B01D1C06870476FF00200704700BF584C00240446002208B5E4B2E0
:20404000034B21461868FFF791FF204606F068FA584C002410B51821044606F021FB20B1F4
:20406000A3689B6A0360002010BD6FF00B00FBE738B50446EFF3118500238022EFF31083AB
:2040800072B682F3118883F31088F0B14368E3B1104B00201B68DBB1A3420FD123681BB156
:2040A0009A68A1680A449A6058B10A4908F0FAFA00206060EDB285F3118838BD18461B68FF
:2040C000E9E7044808F0E4FAF2E76FF01500F1E71B68FFDE585400243C30FFF7C9BF2DE999
:2040E000F84300220B461146586809F0B4FD0546EFF311848026E4B20023EFF3108372B693
:2041000086F3118883F31088002700F108084046FFF776F8284608F0BBFA03460028F6D01B
:204120000269002AF3D040691F6184F311889047EFF31184E4B24B46EFF3108372B686F363
:20414000118883F310889946E1E7FFEC2DE9F0418CB004460E4617460DF11008114A2021F6
:204160001D46404608F000FCCDF808804FF00008CDF80C80FEF782FF02AB20463A463146FD
:204180000093094BFFF73AFD041E07DB2C614446FEF784FF20460CB0BDE8F081FEF77EFFCE
:2041A000F8E700BFCE891608DF400208034B4FF4A062F9210248FFF7C9BF00BF80040024E7
:2041C000D3891608034B4FF4CC6232210248FFF7BDBF00BF94040024DA8916082DE9F8434A
:2041E0000C46274B07461D68FEF748FF24BBAB681C6C0CBBFEF752FF2046BDE8F8830135AA
:2042000054F825604FEA8509002EF8D18DB105F101084FEA8808404607F05EFE064610B321
:20422000A8F104080023444440F8093005F1FF3825B900243E64DDE70025E1E754F8040CDF
:2042400009F02EFF013007F047FE46F8280080B905F18045013D06EB850555F8040F28B977
:20426000304607F031FE6FF00B04E3E707F02CFEF3E754F8041D4546FDF73EFDD6E700BFCC
:20428000584C002470B5046C84B1002054F8203063B14A1E013B12F8016F13F8015FAE4243
:2042A000F9D00EB93D2D03D00130EFE76FF0010070BDFFEC2DE9F8430E4614460546002840
:2042C0005DD009B10B782BB9A4B12846BDE8F84300F05CB8FEF7D2FE2A4B1B689F683B6C7E
:2042E00073B129463846FFF7CDFF011E08DB24B9FEF7D4FE2046BDE8F883384600F068FEEB
:20430000284609F0CDFE0446304609F0C9FE2044023007F0E1FD804630B3D7F84090B9F18E
:20432000000F2AD1082007F0D7FDD0B14C4640F8248000EB840300242A4613495C603346FA
:204340003864404608F0ECFAD2E7013459F82430002BFAD1A11C4846890007F0C5FD00281F
:20436000E5D1404607F0B0FD0C24FEF797FEFDF71DFD04604FF0FF34BCE70024E6E71624F1
:20438000F5E700BF584C0024E189160838B5114B04461B689D6828B103781BB13D2109F0A0
:2043A0004FFE30B1FDF702FD162303604FF0FF3038BDFEF763FE45B121462846FFF762FF65
:2043C000011E02DB284600F003FEFEF767FE0020EEE700BF584C002470B506464FF47D700B
:2043E00007F08AFD044610B300F0BEFC051E04DA204607F069FD284670BD04F14400B460DC
:204400000BF0FAFB204609F052FB0122002104F1180008F0D2F90C340022002520461146A8
:2044200008F0CBF900212046FFF707F9E3E76FF00B05E0E7D0E902321A6001225A72704736
:2044400038B58468054634B1637A012B04D9013B63720023AB6038BD204600F096FC2046EB
:2044600000F037FB204600F070F804F144000BF0C7FB204609F03AFB204600F095FDA37ACD
:2044800023B1237A43F008032372E2E7204607F01BFDDEE738B5032105460B480BF08CFFA0
:2044A000041E0BD101210BF0A5FC204602210BF0A1FC2846BDE8384000F0AABD01DD0BF064
:2044C000E8FC6FF0160038BDEC841608084B10B51B68044681689868443144300BF02AFC28
:2044E000002804DB2046BDE8104000F091BD10BD584C00240023044A044942F83310013318
:20450000A62BFAD1FDF7BAB8004F0024312F020808B53AB119B9FEF739FE404208BD00F0DF
:204520000DF9FAE711B9FEF76BFEF6E700F00AF9F3E708B528B1FEF779FE002803DA404239
:2045400008BD1620FCE70020FAE738B50446256A2DB904F11800BDE83840FEF7FBBD28468B
:2045600050F8143B2362FEF7F5FD05F10C00FEF7F1FD284607F0A8FCE9E7F8B58026002700
:204580000446FEF77BFDE36F1BB9BDE8F840FEF785BDEFF311832A46EFF3108272B686F32F
:2045A000118882F31088E06F1546DBB20268E267076083F31188037C043043F00203037394
:2045C000FFF7B7FFDFE7FFEC0346EFF3118100228020EFF3108272B680F3118882F310884A
:2045E0000A4A106860B1002B0EDB094A1268013A1A4050F8220018B1C2689A4218BF002038
:20460000CBB283F3118870470020F9E7544C0024444C002438B5044618B3C068B0B1EFF372
:20462000118200238025EFF3108372B685F3118883F310880C4B00251B68013B03400B4892
:20464000006840F82350D3B283F31188236D13B1204605F0D1FF2046FFF7F2FE204607F08B
:2046600033FC002038BD00BF444C0024544C00244B1EFE2B73B504463CD8EFF3118600230B
:204680008022EFF3108372B682F3118883F31088037FCDB2022B0ED0032B18D103681B7C9A
:2046A000994225DC294605F0B9FFF6B286F31188002002B070BD114B1B681B7C9942F1DC2B
:2046C00000F0E2FC2046257400F0BAFCEDE70C4A02EBC3010979C9070AD552F8331001913C
:2046E00008F006F801992046257400F0E1FCDCE72574DAE76FF01500DBE700BF584C002484
:204700006489160838B504460D46FFF7B1FF10B984F82E50607738BD10B5EFF31184002370
:204720008022EFF3108372B682F3118883F3108805F0DAFFE4B284F3118810BD0A4600216C
:2047400000F008B80A46002100F04EB80A46002100F056B8214B2DE9F74307468946904625
:204760001D68EFF3118600238022EFF3108372B682F3118883F3108800F0E0FC044688B16E
:20478000D8F80420164B9A4224D801AA4146484600F0DCFB28B9019C002C0ADC6FF07304FF
:2047A00000E04442F6B286F31188204603B0BDE8F0833C35FFF718FC21460346094A2846BC
:2047C00000F0EEFA3846FEF7E1FC04462846FFF74FFCE7E76FF01504E4E700BF584C002420
:2047E000FFC99A3B1B48020870B504460D461646324629462046FFF7ADFF031DF8D070BD8D
:2048000010B5FFF7A7FF041E05DA6442FDF7CEFA04604FF0FF34204610BD10B5EFF311848F
:2048200000238022EFF3108372B682F3118883F31088FFF7C9FE28B1037F052B02D174214A
:2048400000F025F8E4B284F3118810BD70B50446EFF3118500238022EFF3108372B682F31A
:20486000118883F31088037F052B09D1866D3146FEF7AEFE338801331BB233800023A36560
:204880002046EDB2FEF7D0FE85F3118870BDF8B504460E46EFF3118500238022EFF3108315
:2048A00072B682F3118883F31088037F052B0DD1876D3946FEF78CFE3B88204601331BB208
:2048C0003B8000232687A36505F00EFFEDB285F31188F8BDF8B50024284B294E6020C3E9F7
:2048E0000044284BC3E90044274BC3E90044274BC6E90044C3E9004407F0EEFA054648B137
:2049000000F160072C7528461835314607F08CFEAF42F7D1602007F0DFFA044658B100F19E
:2049200060050227174E277520461834314607F07BFEA542F7D1402007F0CEFA044658B12E
:2049400000F140050027104E277320461034314607F06AFEA542F7D1402007F0BDFA04467B
:2049600058B100F140050227084E277320461034314607F059FEA542F7D1F8BD3054002464
:2049800038540024405400245054002448540024002337B582680193EFF311858021EFF39F
:2049A000108372B681F3118883F31088546B2CB9EDB285F31188019803B030BD217901A851
:2049C00007F02DFF2468F2E738B50D46044640B1FEF754FBE46A14B1237CAB4203D1FEF728
:2049E0005DFB204638BD2468F5E7FFEC124B10B51B6843B1114807F04BFEE0B91048BDE8E9
:204A0000104007F045BEEFF3118400238022EFF3108372B682F3118883F310880748E4B272
:204A200007F036FE84F3118828B9182007F054FA08B10123037510BD704B0024385400242C
:204A40004054002410B5037D83B9EFF311848022EFF3108372B682F3118883F310880E49F4
:204A600007F0E2FDE4B284F3118810BD022B0CD1EFF3118400238022EFF3108372B682F395
:204A8000118883F310880549EAE7012BEDD1BDE8104007F019BA00BF385400244054002480
:204AA00038B5044600F16405284607F0F1FD50B904F16C05284607F0EBFD38B94FF0FF32F5
:204AC000C4E9172038BDFFF7BDFFEDE7FFF7BAFFF0E738B5044600F12C05284607F0D8FD5E
:204AE00028B93434204607F0D3FD18B938BD00F04DFBF2E7FEF75AFEF4E7FFEC2DE9F74306
:204B00000F46054600283BD042681F4B9A4237D8EFF3118600238022EFF3108372B682F373
:204B2000118883F31088DFF864906846F6B2D9F8008007F08EFE2A460021684600F0F4FBBB
:204B400010F10B0F044606D186F311880024204603B0BDE8F08387B101A9284607F0E8FD86
:204B6000D9F8003001983946A3EB080290428ABFC01A0020404407F0CDFD86F31188E6E74B
:204B80006FF01504E3E700BFFFC99A3B844B00247FB51D46CB0714462AD5EFF31186002326
:204BA0008022EFF3108372B682F3118883F3108802A9F6B200F06EF9002806DA86F31188D6
:204BC0004FF0FF34204604B070BD6A4602A9204607F0CAFD29466846FFF790FF044686F338
:204BE0001188002CEEDA6442FDF7E0F80460E7E729461046FFF782FF0446F2E77047FFEC83
:204C00000F4B70B51D68AC68FEF738FAE37A5A0706D4284600F070FABDE87040FEF73EBAB3
:204C2000626900230AB11360636104F10C06E372A3891B04EDD53046FEF7F8FAF8E700BF30
:204C4000584C002408B5064B1B689B8E03F00303012B02D10020FDF7B3F80120FCF7AAFF5E
:204C6000584C002408B580683C3007F0F6FD0028D4BF0020012008BD0023084A12F83310EE
:204C8000814206D102EBC3035878C04300F00100704701330B2BF1D101207047E8891608B9
:204CA00038B585685AB100231A4A12F83300814219D102EBC30305F13C005C68BCB9EFF39E
:204CC000118400238022EFF3108372B682F3118883F3108805F13C00E4B207F0ADFD84F3E1
:204CE0001188002413E001330B2BDED1E7E7EFF3118500238022EFF3108372B682F3118835
:204D000083F3108807F08BFDEDB285F31188204638BD00BFE88916082DE9F0438668002452
:204D2000104D4FF002093C36A04685B0304607F090FD6B6873B12F7801A90022CDF80C907A
:204D40003846CDE90138012300F036FA3946304607F065FD013408350B2CEAD1002005B01B
:204D6000BDE8F083E889160838B505464C2007F0C3F8044630B10122002107F01EFD002095
:204D8000AC6238BD6FF00B00FBE710B5846A2046FEF7E0F92046BDE8104007F095B8FFEC53
:204DA0002DE9F0410C46164698460546002839D0002A37D0002935DBEFF3118700238022FB
:204DC000EFF3108372B682F3118883F3108843680BB1FFF74DF91F4901346E600E68C5F8D9
:204DE0000C801EB9284607F01FFC2CE03046334600229968521801D5196831B9A24214DC33
:204E0000196829B9A41A1349ECE718460B46F0E78868024418460B46F0E70E4A294607F042
:204E200013FC10E06FF0150012E099689E42A2EB0102A4EB0204A1EB04019960EDD1054971
:204E4000284607F0FBFBAC60FFB287F311880020BDE8F0815854002438B50D4C236843B15C
:204E60009A680025013A9A60236813B19B68002B00DD38BD204607F00BFC23681BB19A68CA
:204E800081680A449A6043684560C0689847EBE758540024431E012B37B50D460CD80846EA
:204EA000FDF7FEFE0446002C36DA6442FCF77EFF04604FF0FF342FE0002830D16846FDF7B6
:204EC000EFFE04460028EED1EFF3118300228021EFF3108272B681F3118882F3108811496B
:204EE000DBB2009A0868496802440092019A0A44019283F311880C4A019B934208DD0B4808
:204F0000009A93FBF0F10A4400FB113300920193009B2B60019B6B60204603B030BD6FF0E3
:204F20001504C2E77C4B0024FFC99A3B00CA9A3B02680B689A4204D306D840684B68C01AE5
:204F400070474FF0FF307047012070477FB50E4669461546FFF79EFF044608BB6946304646
:204F6000FFF7E6FF002805DA4FF0FF332B60204604B070BD019B7468009AE41A3368002C35
:204F8000A3EB02030394029304DA064A013B224402930392294602A807F0CAFB0446E6E76C
:204FA0001624E4E700CA9A3B38B5036C04466BB90023236438BD06F087FF236C58590435EF
:204FC0000028F8D1184606F07FFFF1E70025F4E770B5036C05460C4653F8210006F074FF30
:204FE000A3002A6C0433D15842F824102146286C0134C658002EF3D1012C03D106F064FF10
:205000002E6470BD0231890006F06EFF2864F8E7002307B502460190012118460BF02CFEEA
:20502000019A0023062101200BF026FE0023019A062102200BF020FE002003B05DF804FB04
:205040000F4B10B51B680446B3F93620002A0ADD1A7C037C9A4206D20A4900F029F8012300
:205060000020237710BD0649204600F021F8022320B10322227722681377F3E72377F1E7D7
:20508000584C00244C4C002438B5436804465BB90368032201251A772046044907F028FB82
:2050A00000232846237738BD0025F5E7584C002410B50B68027CB3B11C7C944206D25A68E5
:2050C00062B9C0E900325860086013E01B68F2E7C0E900321060486000200CE0C0E9003291
:2050E00010605860F8E74A68002AF1D1C0E90033C1E90000012010BD38B50446EFF31185E8
:2051000000238022EFF3108372B682F3118883F31088037F043B032B0BD800F097F9042398
:2051200007212046238700F07DF9EDB285F3118838BD072105F096F9F7E7FFEC38B5124B6D
:205140001D68E8B1EFF3118400228021EFF3108272B681F3118882F31088028812B2002AC9
:205160000BDD0288013A12B20280FEF703FA0020A865E4B284F3118838BD6FF00A00F8E73A
:205180006FF01500F8E700BF584C002410B5EFF3118400238022EFF3108372B682F3118889
:2051A00083F310880349E4B207F03EFA84F3118810BD00BF305400242DE9F74F1546504A3B
:2051C0001F280746D2F800B00E46DBF808A004D96FF0150003B0BDE8F08F41B939465046BB
:2051E000FFF7F2FB044665B916BB0020F2E7002BF4D10B68012BF1D0FFF73EFD0028EDD133
:20520000E6E739465846FFF72DFD30B100230122C5E900230223AB60E6E72CB163682B605C
:20522000A3686B60E368F6E7C5E90044AC60DBE73568012D11D12A4639465846FFF730FD53
:20524000054685B9002CD0D020460AF12C0107F009FA2046FFF79AFFC7E70022394658468F
:20526000FFF71EFDEDE7D4B9EFF311834FF0800B00930022EFF3108272B68BF3118882F39F
:205280001088204807F004FA009B0446DBB283F3118850B10AF12C01077407F0C5F965607A
:2052A0007368A360B368E3609FE7502006F014FE14490446C0B1EFF31183EFF3108972B683
:2052C0008BF3118889F3108800F1500220461434CDE9002307F0A8F9009A0A499442019BE2
:2052E000F4D1DBB283F31188EFF311830093EFF3108872B68BF3118888F310880846C1E782
:20530000584C002430540024027F062A0AD140F2FF22A0F87420742280F876200022826763
:2053200005F0E2B97047FFEC394B2DE9F34707460D4692461C68EFF3118800238022EFF349
:20534000108372B682F3118883F3108806682046FFF71EFB30405FFA88F80190A0B101A8BF
:20536000FEF752FA01462046FEF7FCF91DB143682B6083686B600679FEF718FA88F3118801
:20538000304602B0BDE8F0873B682366BAF1000F33D0DAF8043004F13C091E4ED917DAF872
:2053A00000C09E191C481D4A4FF0000341F10001ECFB0061304612F029FB23460146184A40
:2053C0004846FFF7EDFC2046062105F04BF84846FEF74EFE94F8741000231F29236611D8DF
:2053E000384607F03AFA80B194F87460002DC5D0636F2B60A36F6B60C0E70621204605F04E
:2054000031F8E7E76FF00A06F0E76FF00306EDE7584C00243F420F0000CA9A3B40420F008B
:205420000953020838B50C46074B054653F8311003EBC4031B79DB0703D5FFF739FE2C77CB
:2054400038BD07F03FF9FAE764891608054B027F10B553F83210044607F04AF900232377D8
:2054600010BD00BF6489160800F01AB838B50D4604462F21284608F09AFD00B1451C28467C
:2054800006F0C8FF031E08DB06F0D6FFC368236083682362436823770023184638BDFFECBC
:2054A000014800F003B800BFA804002410B5044648B1FDF7E3FD054B1A6822601C60FDF7C9
:2054C000EDFD002010BD6FF01500FBE76054002430B585B004460D46002003A911F036F914
:2054E000039B642B05D0642303A90020039311F0FBF800F013F82946204600F02DF8019057
:2055000011F0CAF8019A044900F51A7008F0A0FA012005B030BD00BF408A160808B500F0B8
:2055200007F800214FF60170BDE8084009F035BB002307B5054A00930123054905480BF044
:2055400031FDC01703B05DF804FB00BF678A16086E8A1608738A160870B5054601200E465B
:2055600000F0ECF8044670B100F0C4F9204600F0C9F9334601212A46204600F0A1FC636A5C
:205580000146204698476FF00B0070BD00F52970704770B504460E461546B2B1D0F8943294
:2055A0003BB1D0F8980208F061F9D4F8940208F05DF9D4F890322B60D4F88C326B60D4F861
:2055C0009832AB60D4F89432EB600023C4F88C62C4F8943270BD38B50446D0F8945211F0B7
:2055E0005BF800F59C70854209D111F055F800F59C7008F03BF90123C4F88C3238BDD4F8DC
:20560000940268B108F032F9D4F8940207F094FF4FF0FF33C4E9A3330023C4E9A533EDE75C
:20562000D4F88C020028F3DB0128F1D00AF06BFCEEE738B50D460446FFF7CDFF2B68C4F85F
:2056400090326B68C4F88C32AB68C4F89832EB68C4F8943238BD10B50446FFF7BCFFD4F84C
:205660009C0208B106F030FC2046BDE8104006F02BBC0C4608B5FFF7EEFF2046FCF79AFA9A
:2056800038B5D0F8945204466DB90949D0F88C0207F016FFC4F8940238B1D4F88C32C4F8CA
:2056A0009802C4F89032002038BD4FF0FF30FBE7669616080EB417B50446FFF7E1FF58B994
:2056C00006AA0599D4F89802019208F0CEF903B0BDE8104003B070474FF0FF30F7E70EB4A4
:2056E00017B50446FFF7CCFF58B906AA0599D4F89402019208F0B9F903B0BDE8104003B07A
:2057000070474FF0FF30F7E737B505460C460192FFF7B6FF70B92046D5F89432019A0121E0
:2057200008F01EF80446D5F8940208F09FF8204603B030BD4FF0FF34F9E7FFEC38B50546A4
:205740004FF4497006F0D8FB044638B3144B154A0360154BC2618360144B154AC360154B87
:2057600002624361144B80F888520361134B8361134B4362022380F82B32C0F8903210F053
:205780008BFF012300F51A70C4F88C32C4F8980210F082FF00F59C70C4F89402204638BDDD
:2057A000C557020893550208575602080957020833560208DF560208B55602088D550208DD
:2057C0007356020808B590F88802FFF7B7FF08BD2DE9F04F0D46114604462DED028B83B093
:2057E00000F0C2F808EE100A08B3A36920469847074600286FD0394918EE100AD4F830820F
:2058000007F075FEC4F83002A0B92769FCF7CEFA006808F087FB324B2A463249009020464C
:20582000B84718EE100A00F0C3F8C4F830824FF0FF354AE04FF0FF35DFF8B0B0DFF8B090D2
:20584000DFF8A0A010F028FF00F59C7008F00EF8D4F8300207F0F9FE0023C4F83402984230
:20586000A4F838320CDA23691E46FCF79FFA006808F058FB5B4600904A4651462046B04758
:20588000D4F830228021384607F008FF98B194F82B329A0704D463693A4613492046984735
:2058A0003946204601F004FE05460028CAD094F82B32DB07C6D4D4F8300207F03DFEC4F8B2
:2058C000308218EE100A00F073F8284603B0BDEC028BBDE8F08F4FF0FF35F2E70994160819
:2058E0007D8A1608728C1608EA131708838A1608898A1608014A0249FFF76ABF8E8A160804
:205900009D8A160838B50446FDF7B8FB084B01221D781A70FDF7C2FB45B9064A204606491B
:20592000FFF756FF022384F82B3238BD0020FCE764540024A58A1608DF1F180808B50249D7
:2059400043699847002008BD3CC41B0808B50448FDF7C4F9034B002808BF184608BD00BFDB
:20596000EB8A1608E28A160870B506460C4609B10B7823B90C48BDE8704008F0C3BA2F2BB6
:2059800001D10846F7E7FFF7E1FF08490546204608F060FB08B92846EDE72246294630468E
:2059A000BDE8704000F080BCE28A160840C8180808B106F089BA704701292DE9FF4106463F
:2059C00017464EDD55682A49284608F043FB00284BD02849284608F03DFB044658BB26484E
:2059E000FDF77CF9254B002808BF184608F08AFA804608F077FD054678B13A68356903928A
:205A0000FCF7D4F9006808F08DFA1D4B00903046039A1C49A8474FF0FF35B8F1000F02D083
:205A2000404606F051FA14B12046FFF7C1FF284604B0BDE8F0811449284608F00BFB044673
:205A400038B9FFF783FF08F05DFA804606F08EFDCFE729463046FFF787FF4FF0000804469F
:205A6000C7E70024A0460548C3E70446FAE700BFB58A1608E5931608E48A1608E28A160884
:205A8000B78A1608728C160860F01A082DE9F04F834685B017464FF0000A4FF00108634C29
:205AA000009122463946009808F0D6FC431C13D108F0DFFCD0F8009007EB8907009B9945A3
:205AC00025DBB8F1000F15D0DBF81430584658494FF0000898470DE065280FD06E2810D0DE
:205AE000452811D04FF0FF38DBF810303A68584650499847404605B0BDE8F08F4FF0010A6E
:205B0000CFE74FF00008CCE74FF0000AC9E708F0B0FC03684B4504D0DBF814305846464925
:205B20009847BAF1000F64D03D682C462B780BB923705EE05C2B04D02E4604F8013B751CB1
:205B4000F4E76B786E1C0D2B0AD80D2B0ED8DFE803F04B0D0D0D0D0D0D5A5D0D636960661C
:205B60005C2B37D0782B0AD0302B18D023464FF05C0203F8022B6A7862701C46DFE7033595
:205B80000023029616F8012F03931046019206F074FC039BDDE90121A0B90E461AE00435C1
:205BA0000021737832460136303BD8B2082803D9164604F8011BC2E7B54203EBC101F0D1A4
:205BC0002A46F5E7A2F130001B01092805D8AE420344D6D104F8013BB1E71046019306F0FE
:205BE0005AFC019B5738F2E74FF05C03237000236370DBF81430584657F8042B09F10109ED
:205C00000E4998475AE74FF00703E3E74FF00803E0E74FF00C03DDE74FF00A03DAE74FF08B
:205C20000D03D7E74FF00B03D4E700BFBD8A1608A2A51A08138C16083B971608EA13170838
:205C400038B504464569FFF781FE034902462046A847002038BD00BF3CC41B082DE9F047BD
:205C6000514B86B0164601291A880DF114099B7805460C46ADF8142089F802300DD10022D3
:205C80004A4900F0E5FB04466B692846E41748499847204606B0BDE8F087022901D0042949
:205CA0006DD17768384608F0FBF9012810D832682C690392FCF77AF8006808F033F93D4B0F
:205CC000039A3D4900902846A0476FF01504E0E797F80080B8F12D0F0FD0B8F12B0F0CD0EB
:205CE00032682C690392FCF761F8006808F01AF9304B039A31490090E5E74FF0010A17F8DA
:205D0000011F11F0DF0F24D10223033C012C49D801339C0056F8230000F0A8FA0390043C27
:205D20003059FCF7DBFF039958BB0A462846315900F030FB041EACDA326860422F690392EA
:205D400008F0F0F81E4B0090039A28461D49B8479FE7484608F074F90028C1D0A0EB090331
:205D600095F92B22B8F12B0F0AFA03F35BB20CBF134322EA0303DBB285F82B32BFE70123FA
:205D8000C3E730590122FEF795FA041E81DA32682F690392FCF70AF8006808F0C3F80A4B80
:205DA0000090D1E7002474E7C2CD18083D590208A2A51A08DBCA18084B8C1608138C1608ED
:205DC000C18A1608728C1608DB8A16087FB551680446154600F018FB002827DA831C25D069
:205DE0002A6840422669039208F09CF8104B00902046039A0F49B0474FF0FF366868FEF769
:205E0000C5FA00280FDA2A6826690392FBF7CEFF006808F087F8084B00902046039A05492A
:205E2000B0474FF0FF36304604B070BD0026E5E7CC8A1608728C1608D98A160803297FB53D
:205E40000546144618D1916801226068FEF732FA002819DA22682E690392FBF7A7FF0068DE
:205E600008F060F8124B0090039A28461149B0474FF0FF3004B070BD516800F07FFA0E49C1
:205E8000002818BF0146DFE76168284600F0BCFA00280ADA831C08D0226840422E6903925E
:205EA00008F040F8054B0090DEE70020E2E700BFD98A1608728C160861C71B08CC8A160809
:205EC0002DE9F341044690461E4641B1D0F89412394807F08EFDD4F8940207F0C7FCB8F1CC
:205EE000010F2ADC354F04F52976D4F89412384607F07FFDD4F8940207F0B8FC10F0CCFB39
:205F0000054610F0C9FB802100F59C7305F10802304600F0B6FA013044D1D4F89842FBF7D9
:205F200045FF0068002507F0FDFF254B00902046244A254907F08CFD0BE077682349384627
:205F400008F088F8054640B963692046326820499847284602B0BDE8F0811E49384608F05E
:205F600079F880B9B8F1020F06D0B168204602B0BDE8F04101F09CBA2369326816492046AE
:205F800001259847E5E73B7831682D2B03D10A4623691249F3E73A46204602B0BDE8F04139
:205FA000FFF716BC3146204601F082FAD4F8940207F05CFC99E700BFA18D1608C08D160828
:205FC0001D8B1608268B1608728C1608EF8A1608F28A16081A8B16084B8C1608688D160814
:205FE0002DE9F74F04460D461046012116460AF0F0F9B0F100081DDA05223E49304607F036
:20600000C6FF28B9276933462A463B492046B8472669FBF7CBFE006807F084FF374B00903A
:206020002A4637492046B0474FF0FF36304603B0BDE8F08F4FF4007005F04EFF074658B9FF
:20604000404609F060FF2669FBF7B0FE006807F069FF2C4B0090E3E70026DFF8B0A020E04E
:2060600007F060FF284B00902A4625492046B0472AE02BD04FF00009E368ABEB090207EB61
:20608000090120469847002830DAFBF78FFE00682669042821D12A4651462046B0474FF048
:2060A000FF364FF40072394640460AF0CCF9B0F1000BDEDAFBF77AFE006826690428CFD1A1
:2060C0002A4612492046B0474FF0FF36404609F01AFF384605F0F8FEA8E707F023FF0C4B24
:2060E00000902A4606492046B047D8E78144CB45C2DCD6E7328B1608388B16087E8A160823
:20610000728C1608698B16087BC41608488D1608966C17082DE9F74F0646894610460121F1
:2061200098460AF056F9071E11DA3469FBF73EFE006807F0F7FE1F4B00904A461E493046A2
:20614000A0474FF0FF34204603B0BDE8F08F0C9B0025C24603F1FF3B88F800505A465146A0
:2061600038460AF070F9041E16DAFBF71FFE0368042B1AD03469FBF719FE006807F0D2FEC4
:206180000E4B00904A460C493046A0474FF0FF34384609F0B8FED6E7FAD025444FF0000303
:2061A000A244ABEB040B08F805300C9B002BD5D1ECE700BF7E8A1608728C16087BC4160876
:2061C0002DE9F341054610460C461646984606F068F90746E8B905221749304607F0D7FE3A
:2061E00028B92F693346224614492846B8472E69FBF7DCFD006807F095FE22464FF0FF344D
:2062000000900F4B28460F49B047204602B0BDE8F081384606F073F9044640B10246089BA3
:2062200031462846C0470028F3DA4FF0FF34384606F052F9E9E700BF328B1608388B160801
:20624000708B1608728C160810B5044607F028FF00212318E443E218002A03DD13F8012C1D
:206260002F2A00D010BD03F8011DF4E7F8B50446207825462646013468B92846002707F0EC
:206280000FFF2C18B44204D014F8010C06F0EBF830B92846F8BD06F0E6F80028E8D1ECE75C
:2062A00004F8017DEEE7FFEC7FB50B460446114915461846039304F1280607F0CBFE039BAB
:2062C00078B92B460C4A4FF40071304606F04CFB0023304684F8283104B0BDE8704007F0F1
:2062E00011BE064A4FF400713046009506F03CFBEEE700BFE64818085689160854891608B9
:2063000070B5D0E9A7450E462544AC4212D2701E611E10F8012F11F8013F9A42F9D01AB91E
:206320003D2B01D1204670BD204607F0B9FE01300444EAE70024F5E770B5D0E9A73605462C
:206340000C468B421E4416D88E4214D9084607F0A7FE0130631E0444321B002A06DCD5F807
:20636000A032181AC5F8A002002070BD14F8012B03F8012FF0E74FF0FF30F6E708B5FFF735
:20638000BFFF034618B13D2107F05AFE431C184608BDFFECF8B5D0F89C3205460E461746D4
:2063A00033B1FFF7ADFF014610B12846FFF7C4FF304607F075FE0446384607F071FE0444D2
:2063C000D5F89C020234B0B1D5F8A0120C44214605F08AFD024610B96FF00B00F8BDD5F80C
:2063E000A03218443B460749C5E9A724324606F097FA0020F2E7204605F06EFD0028EBD084
:206400000246EFE7E189160810B5044698B1FFF777FF014678B12046FFF78EFFD4E9A70154
:2064200000290CDC20B105F04FFD0023C4F89C320023C4F8A032FCF731FE002010BD05F0D7
:2064400053FD10B1C4F89C02F5E76FF00B00F5E72DE9F041D0E9A74605460F4690462644E2
:20646000B44202D30020BDE8F081224641462846B8470028F7D1204607F012FE01300444E9
:20648000EEE75B68526800F02FB800690AF0C2BA13B504468DF8071001220DF10701206994
:2064A0000AF0B8FA002803DAFBF780FC0368042BF2D002B010BD13B5044601220DF10701A7
:2064C000E06809F0C0FF002803D14FF0FF3002B010BD05DAFBF76AFC0368042BEDD0F4E76A
:2064E0009DF80700F3E7FFEC10B586B0074C0492074A01940292074A059303920A460146C8
:2065000001A800F009F806B010BD00BFB7640208916402088B640208012A2DE9F84F0646AE
:206520000F46904604DC00240C702046BDE8F88F0025DFF8B49083680322AA462A4998478C
:20654000336830469847431C04460DD1002DECD000232C467B55E8E74FF0000AF0E74FF048
:20656000010AEDE75D46EBE7BAF1000F09D05B28F2D1BAF1020F0CBF4FF0000A4FF0020AD3
:20658000DEE7082801D07F280CD1002DE4D0736830460821013D9847B368032249463046F4
:2065A0009847CDE71B28DAD00A2808D16C1C0A210023304679553B5573689847B5E70D281B
:2065C000F4D0C0B205F046FF0028B9D17C5505F1010B023573682146304698474545C1DBD2
:2065E0005C4607F80BA0A0E7788B160810B50022044610F8013B5C2B00D13AB18B4200D151
:2066000012B1002BF3D11C46204610BD0122EFE70023027802B970475C2A00F101010AD1D7
:206620004BB903465A7803F8012B002AFAD1014601230846EDE70023FBE790F83B3200EBAD
:20664000C30393F848329A09032A02D113F0010313D090F83C32184490F83D0283070CD45F
:206660008309022B05D0032B04D0012000F001007047C04300F00100F8E70020F6E770B5CC
:206680000568044695F8293213B1406809F03BFCAB68284604F10C0600259847A368AB423B
:2066A00004DC2046BDE8704005F00EBC56F8040B013505F009FCF1E72DE9F04180461746B1
:2066C0000C46B9B1084607F0EBFC0646384607F0E7FC01308119204605F006FC054658B9AA
:2066E0002546D8F81030074A4046074998472846BDE8F0810E46E9E700233946835507F000
:20670000E3FBF4E77B8B1608A68C160838B500F10C0281680446006801F0CAF80546204661
:20672000FFF7ADFF284638BD10B590F83B42043400EBC40494F828329B09012B0CD10023E9
:2067400080F82A3281F0010094F8282260F3000284F82822184610BD022B07D1002380F837
:206760002A3294F8282261F30002F1E790F83C42044494F83D329B09012B0CD1002380F828
:206780002A3294F83D22C2F38000484060F3000284F83D22DEE74B4280F82A12DAE7FFEC13
:2067A0002DE9F04F8BB0884604461646149F1D460097116802F050FA002808DB14BF012173
:2067C000002120460BB0BDE8F04FFFF7ADBF94F82932BBB139464FF4DB72284609F0F9FD72
:2067E000071E11DA326825690392FBF7DFFA006807F098FB584B00902046039A5749A8474A
:206800000121DEE74FF0FF3794F82832002B7DD02368204698478346002800F093805C207E
:2068200005F06AFB0546002800F0888000F10C0A4FF00009C0F80880C0E900B7C8451FDC9C
:2068400094F829322BB1DBF81C30002239465846984704A900200FF079FFD0B13268276949
:206860000392FBF7A3FA006807F05CFB3C4B0090039A20463949B8472846FFF700FFBFE79A
:2068800056F8290009F1010907F03CFB4AF8040BD4E7D4F82C32002B0BD0049F4FF0010030
:2068A000A7EB03071FDA05F031FFB842A8BF3846049006A805F086FE012106A805F090FE31
:2068C00004A906A805F094FE2B46264A06A905A805F09CFE68B132682769039207F022FB1E
:2068E000214B0090C4E705F013FFB842B8BF3846DEE705980FF076FE049B656920460093C0
:206900003268059B1949A84700215AE794F8293223B1E36906AA3946204698473246414610
:20692000204600F0C5FF94F8293205461BB1236A06A920469847002DE6DA61E7DBF808307E
:206940005846984794F82932002B3FF459AF384609F0D9FA54E700BF7E8A1608728C1608E7
:206960007D8B16080D6702088B8B16089A8B1608F8B500250446061D2F4623689D4202DB01
:2069800000232360F8BD3068013505F09DFA46F8047BF2E72DE9F04F0446BFB00E46D1F881
:2069A0000080DFF8DC920592039398F80070454608F10108002F00F043823946484607F070
:2069C0003FFB0028F1D13E2F0DD16B783E2B0DBF0235A94DC6F80080356008BFA74D284607
:2069E0003FB0BDE8F08F232F02D135600546F6E7222F039BA24A824606BF002345469146B5
:206A00000393A8469F4B08BF99460346474618F8011B61BB37600026AB46B0469A4958461F
:206A200007F062FA03460BEB030707F1010A97F80090002B4DD0B9F1000F33D1002E65D030
:206A400031465A462046FFF737FE0546FFF7E0FD2E46002EC3D0059B1B681D2BBFDC059A96
:206A600002EB830201335660059A1360B7E718B102785C2A00D193B15C2903D0602903D177
:206A80008AF0010A00230BE0BAF1000FFAD14846FFF7ACFD0028F5D007F801ABBAE7012354
:206AA0003846B3E75A1E00215A44A2EB030C12F801095C2803D1944581F00101F7D10493D4
:206AC00051B17149781C07F00FFA049B01300344A9E7B9F1000FB1D0B9F1600F40F0598162
:206AE00031465A4607F8018B2046FFF7E5FD494606463846FFF77AFD049058B9634B25690F
:206B00001A4663492046A847624DA2E72846FFF77FFD64E7049B83F8008000230993FDF764
:206B200063FA5D4A03465D4909A805F010FF002802DB099B0693B3B923692046584A5949C9
:206B400098470027DFF84C9131464A462046FFF7B3FD049B064603F1010A17B1384605F043
:206B6000B3F9D3465AE70DF17C0A502200210BA8FBF77BF87C2200215046FBF776F8B4F87F
:206B800028320DF1280B524607934FF4807359462046A4F8283200230A97FFF7FBFE81468D
:206BA000002841D02046FFF748FD074628B301275946CDF82C90002352462046FFF7EAFE8C
:206BC0000BAB43F8270018B101370AA9132FF2D13EAB0F2F03EB870343F8CC8C04DD236945
:206BE0004A46314920469847262339460BAA20460093069BFFF7D4FD0746079B1FA8A4F816
:206C00002832FFF7B5FE8FB12769FBF7CFF8006807F088F9254B00902046214A2449B847CB
:206C2000099805F051F98CE70746E6E7DDF824A01FA9504609F03AFE814678B1D4F8109063
:206C4000FBF7B4F8006807F06DF91A4B00902046134A1749C847DFF83C9081E0DDF894B08D
:206C60000BF1010005F038F9074628BB236920460B4A0C499847EEE7C78D1608C98D16088B
:206C8000CE8D1608489116080C8C1608B98B1608168D1608C68D1608A68B1608AB8B160897
:206CA000B88B1608A68C16087F8D1608BB8B1608728C1608C08B16085046012109F089FBDB
:206CC000B0F1000A34DAD4F81090FBF76FF8006807F028F95B4B009020465B4A5B49C847C2
:206CE0003846002705F0F0F8B5E74FF40072504609F0A9FB00281ADAFBF758F80368D4F8F9
:206D00001090042B07D1504A20465149C847504609F0F9F8E4E7FBF749F8006807F002F94B
:206D20004C4B00902046484A4849C847EFE78144CB4507EB0901D8D88946474BB945A9EB4A
:206D4000070B23D0184619F8011D07F079F9424B0028F3D1B946504607F80B8009F0D3F8DC
:206D6000099809F021FE00280CDAD4F810A0FBF71DF8006807F0D6F8384B00902046324AA7
:206D80003249D047099805F09FF8DDE64FF0000BE0E7B9F1240F7FF4E4AEB94631465A4668
:206DA000204609F8018BFFF787FC7B7806467B2B30D107F102097D214846FFF717FC18B978
:206DC0002569274B274A9CE682460AF8018B039B13B10123039A13602349484607F03AF9B0
:206DE000F0B994F82A222148214F002A14BF8346BB4694F82B329B0705D45B464A461D4977
:206E000020466769B84731465A462046FFF754FC0646A6E6484607F043F909EB000AD6E726
:206E200049462046FFF7AAFA83460028E1D1124F4846FBF753FF002814BF8346BB46D8E769
:206E40003D46CCE57E8A1608B88B1608728C1608488D16087BC41608CE8D1608C58B160824
:206E600009C61A08CC8B16080F8C1608118C1608CC8D1608CF8B1608C68D16082DE9F04F83
:206E8000B9B004460D465022002105A8FAF7EDFE7C22002119A8FAF7E8FE002319AA03A9E7
:206EA0002046A4F828320395FFF774FD0546002800F0BF80A74907F0CDF8804630B1A64993
:206EC000284607F0C7F8002840F08F80002319AA03A92046FFF75EFD064608B103781BB98A
:206EE00023692A469D4924E094F83C72E31993F83D329B09012B14D094F83B1204EBC1033C
:206F000093F84832C3F38113033303F00303012B07D9D4F8303223B1D4F83492B9F1000F9A
:206F200002DA23692A467CE006291DD923692A468B492046984794F84832002203F03E0387
:206F4000A4F83A2243F00103C4F84C2284F8483219A8FFF70DFD01212046FFF7E5FB054678
:206F6000284639B0BDE8F08F0131B8F1000F2046C9B20CBF4FF001084FF00208FFF75DFB21
:206F80000A1D002384F83B1204EBC10104EBC20284F83A3240EA8813B4F8385292F82802E3
:206FA00023F03E034D4400F03E00034382F82832C1F84C52354681F849726A49284607F086
:206FC00049F80646002840F03681034619AA03A92046FFF7DFFC054618B10378002B40F03C
:206FE0008B8023695F4A5D49AAE05F49284607F031F8034608BB19AA03A92046FFF7CAFC4E
:2070000094F83B320546043304EBC30393F82812C1F38112033202F00302012A03D9236975
:20702000514A524985E741F0C00183F828120028C3D10023C4F82C3259E14D49284607F0D9
:2070400009F80346002848D119AA03A92046FFF7A1FC10B12369464A44E794F83B22131D1C
:2070600004EBC30393F828128D09032D02D023693F4AD6E71AB923693D4A3E4959E7CA07AE
:2070800026D50246D3F82C12D4F8300206F0BDFA00280BDA2569FAF789FE006806F042FF47
:2070A000354B00902046324A3449A847012384F83A3294F83B321A1D013B04EBC20292F8BD
:2070C00028126FF3871182F8281284F83B32B0E741F0010183F82812EBE794F83B3204EBA6
:2070E000C30393F84832C3F38113033303F00303012B3FF662AF14E7214906F0ABFF03468C
:2071000068B919AA03A92046FFF744FC054600283FF467AF0378002B3FF463AF012694F8E9
:207120003C12631893F83D329B09012B03D123690C4A0E4904E0062924D92369094A08496F
:2071400020469847B4F83C3203F46053A4F83C32FEE600BFD88B1608DE8B1608138C1608B4
:20716000E28C1608F28B1608E48B1608BE8C1608E78B1608FD8C1608EC8B1608728C16080B
:207180001DFF1A0820460131FFF757FA80F00103C9B25B0084F83C12214443F0400391F85A
:2071A0003D2243EA860302F0380223F03803134381F83D320023C4F82C32002D00F0978091
:2071C000AE49284606F046FF002840F0A9800A2319AA03A9C4F82C3203462046FFF7DAFB5E
:2071E0000546002800F08380A54906F033FF0646002840F09580034619AA03A92046FFF746
:20720000C9FB0746002800F08B80324604A906F0E8FC00F11403C4F82C02272B05D8049B7B
:207220009F4202D01B78002B72D023692046934A944998478CE69449284606F00BFF03460A
:20724000B0B919AA03A92046FFF7A4FB94F83C220546224492F83D329909012902D023699D
:20726000894A66E7022161F3871382F83D32A1E78649284606F0EEFE0346A8B919AA03A934
:207280002046FFF787FB94F83C320546234493F83D229109022902D023697C4A49E742F02F
:2072A000C00283F83D2285E77949284606F0D2FE034608BB19AA03A92046FFF76BFB10B1D2
:2072C0002369734A8FE694F83C32E21892F83D227F2A02D823696E4A2BE71BB923696D4A23
:2072E0006D492DE7013BC4F82C0284F83C3219A80025FFF73DFB33E694F83C32234493F89B
:207300003D329B09012B7FF455AF23692A4610E719AA03A92046FFF73DFB05460028E6D098
:207320002046FFF78AF90028E1D001264FF00009DFF878A1059504AB19AA03A92046CDF853
:207340001090FFF727FB38AB07464FEA860803EB860343F8CC0C00286ED0049BE3B105ABAB
:20736000984458F8047BBB4617F8011BA1B1504606F066FE0028F6D001368BF80090BB46BB
:2073800017F8011B21B1504606F05AFE0028F6D1132EC8F800B0E4D10136122ECBDD771E03
:2073A00038AB3E4903EB870353F8CC0C06F052FE18B901233E4684F82832022E58DDA6F137
:2073C000020938AB364903EB890353F8CC7C384606F040FEA8BB012394F82982204684F8E1
:2073E000293238AB03EB860656F8D01C4E46FEF7BBFA4FF02609074638AB00220F2E03EB72
:20740000860343F8CC2C04DD23692A462549204698473B4605AA31462046CDF80090FFF7C8
:20742000BFF9054627B13846FEF7C2FA84F8298219A8FFF79DFA93E5012EB0D18046814618
:20744000DAE71949384606F005FE88B9012394F82982204684F8293238AB03EB860656F80E
:20746000D01C4E46FEF780FA4FF016090746C3E74FF00008C1464746BEE700BF028C1608DD
:20748000078C1608138C1608F58B1608FA8B1608FF8B1608F28B1608FD8C16080A8C16089F
:2074A000C78D16087F8D1608C98D1608CE8D16082DE9F843002705460E460C468946DFF834
:2074C0007C8080F83A72A31B41462046A5F8383206F00AFD235C22181BB10A2B01D0232B04
:2074E00005D149462846BDE8F843FFF7C7BC3B2B02F101040CD1494628461770FFF7BEFCF1
:2075000098B9A14695F83A32002BDCD000200CE022212046FFF76AF848B9064B28462C6901
:207520001A460549A0474FF0FF30BDE8F883441CE8E700BF48911608168D16089C8D16083B
:2075400090F83B32043300EBC30393F828229209032A09D193F8292280F83C2293F8282256
:207560006FF3000283F828220020704708B503490369126898474FF0FF3008BD8A8C1608D6
:20758000002070474FF0FF30704708B50021436A9847FFEC10B4CB680A68446923B1A446C6
:2075A00004495DF8044B6047234603495DF8044B184700BFD28D160834C41B0837B50446EE
:2075C0000A460E4D286830B9236920460C4903B0BDE8304018471146019206F03BFD019A66
:2075E00050B963692046074998472946204603B0BDE83040FFF7CEBF1035E3E774911608CF
:207600008A8C1608DB8D160801292DE9F74F04460D46164640F3D1809049506806F01AFD0F
:20762000002800F016810122002356F82250002B00F0C180636920468949984763698949B8
:207640002046984763698849204698476369874920469847636986492046984763698549A8
:207660002046984763698449204698476369814920469847636981492046984763697A49A2
:207680002046984763697E492046984763697D4920469847636977492046984763697A4996
:2076A0002046984763697049204698476369774920469847636973492046984763696D499B
:2076C00020469847636970492046984755B129462046FFF773FF002003B0BDE8F08F02223D
:2076E0000123A2E76A4D204663696A49984729462046FFF74FFF55F8103F002BF7D1002793
:207700003E463D46384604F097FE002834D1002DE1D00236013D4FF000086369502E5E49A2
:20772000204696BF50270127B7FBF6F73D449847B5FBF7F54545CED0C1464FF0000A636910
:20774000204656499847484604F076FE834638B1DBF80C30DBB90AF1010AA9445745F2D1A8
:20776000636920464E4908F101089847E2E74D492046013790475DE0C36833B100680135A1
:2077800006F08EFC864238BF06460137BAE7DBF800202046636944499847DBF8000006F02B
:2077A0007FFC83465E45D6D9636920463D490BF1010B9847F6E7002D89D100263B49204620
:2077C0003546FFF7FBFE6369204635499847304B53F82600043606F063FC854238BF05462C
:2077E000942EF4D102354FF00008502D96BF50260126B6FBF5F606F12409B9FBF6F9C145AC
:207800003FF47DAFC2464FF0000B6369204623499847BAF1240F676914D81D4B4FEA0A12E3
:20782000214920469A580192B847019A104606F037FC0746BD42626999D80BF1010BCA443C
:207840005E45E6D163692046154908F101089847D5E7022D7FF443AF0546EBE6E58D160861
:20786000E88D1608FC8D1608378E16083B8E1608478E16084F8E1608688E1608708E1608E6
:20788000778E1608868E16088C8E1608958E160874911608A48E1608C18E16083A9716084B
:2078A000A2A51A083B971608EA131708BC8E1608F7B5174604460E461268134D286808B919
:2078C000124B17E01146019206F0C4FB019AC0B92B7AB34207DD23690D49204698474FF0BD
:2078E000FF3003B0F0BD6B7AB34202DA23690949F3E76B683A463146204603B0BDE8F040D3
:2079000018471035DAE700BF749116086D7502084B8C16087F8D16082DE9F04F91B0054634
:2079200001A908F0D1FF041E4EDB039B284603F47043B3F5804F03D009F036F8044643E0F6
:2079400004F0AFFD0746002842D0284606F0A8FB064630B1431EEA5C2F2A02D100221E4673
:20796000EA54DFF87480DFF87490DFF874A0384604F0C5FD834650B9384604F0ADFD041EF4
:2079800022DB284605F806B008F0B8FED6E70BF1010B4146584606F05DFB0028E7D0494675
:2079A000584606F057FB0028E1D05B465246C6F58071A81904F0D8FF2846FFF7ADFF041E65
:2079C000D5DA384604F088FD204611B0BDE8F08F4FF0FF34F8E700BF40C8180860F01A080C
:2079E0005689160810B50749044606F033FB38B10549204606F02EFBB0FA80F0400910BD1B
:207A00000120FCE740C8180860F01A082DE9F0439E0795B00546884614461F4671D0EAB1E1
:207A20000132FEF741FC814605A908F03FFF0646484604F049FABEB12C69FAF7B7F9006818
:207A400006F070FA454B00902846454A4549A0474FF0FF34204615B0BDE8F08305A940464B
:207A600008F024FF0646E6E7B90743D53E4B02AE186859681A899B7A03C6B3703280079E85
:207A800006F47043B3F5C04F4FD162238DF80830F20544BF72238DF80930330644BF7723FD
:207AA0008DF80A30700644BF78238DF80B30B10644BF72238DF80C30F20644BF77238DF809
:207AC0000D30330744BF78238DF80E307007284644BF72238DF80F30B107244944BF7723CB
:207AE0008DF81030F20702AA44BF78238DF811306B699847FB0704D56B6928460B9A1C49DE
:207B000098476B692CB3671C184928463A46984723786E69042B17D13846FFF763FF044679
:207B200090B914492846B04794E7B3F5005F01D16323ABE7B3F5804F01D16423A6E7B3F5C9
:207B4000004FA5D03F23A1E70B4928460024B04780E742460949284698477BE7C08B160841
:207B600055B71608728C1608DC93160856DF1608D4931608D9931608A2A51A083BC41B0845
:207B8000F0B51F46137885B00546042B28D10132039110460292FFF725FFDDE90221F8B943
:207BA0002846FEF781FB064602466B690D49284698470D4B32460D4928460097FEF700FBC0
:207BC000044638B90A4B3246084928460097FEF7F7FA0446304604F077F9204605B0F0BD75
:207BE0000024FAE7E79316080D7A020855B71608817B02082DE9F74305468846164600243E
:207C00000127DFF84890474500DA1CB1204603B0BDE8F08356F827102846FDF7A5FE024657
:207C200040B94FF0FF342B6932684946284698470137E8E7019028463168FEF7D1F9019AD6
:207C400004461046FDF7B4FEF2E700BFA68C16081346024A1968FEF7C3B900BFEC93160803
:207C60002DE9F04F2DED028B95B0516804461546FDF77AFE804660B94FF0FF3723692A6887
:207C800020466F499847384615B0BDEC028BBDE8F08F012108F09DFB031E08EE103A13DA4A
:207CA0002A684FF0FF3726690392FAF77FF8006806F038F9634B00902046039A6249B047BF
:207CC0004046FDF775FEDEE7A9682046FDF74CFE064658B94FF0FF3723692A682046584946
:207CE000984718EE100A08F00EF9E9E705A908F0DDFD074600283CD1079B03F47043B3F5C0
:207D0000804F2CD13046FEF79FFA686804F00AFC314602462046FEF7C7FA814640B92369A2
:207D200020462A68464998473046FDF741FED8E730464FF0260A4E46FDF73AFE41463046D3
:207D400006F088F9C0B9236920462A683F499847B9F1000FE8D0484604F0B6F8C1E7B3F557
:207D6000004F0CBF4FF0260A4FF0020A4FF00009E4E74FF0260AF9E751464FF4DB72304630
:207D800008F027FBB0F1000A2ADA2A68D4F810A00392FAF70BF8006806F0C4F8294B009065
:207DA0002046039A2849D047D2E70392F9F7FEFF006806F0B7F8264B0090039A2046224981
:207DC000D84726E05A465046039108F023FE002823DBABEB000B0399BBF1000F0144F1DC6B
:207DE00004F128014FF4007218EE100A039108F02AFBB0F1000B21D00399E3DAF9F7D6FF24
:207E00000368D4F810B0042B2A68CED111492046D847504608F077F89AE7F9F7C7FF03688D
:207E2000D4F810B0042B2A68F0D00392F9F7BEFF006806F077F8084B0090BEE75F46E8E72A
:207E4000A68C16087E8A1608728C1608688D16087BC41608488D1608966C17082DE9F04FB7
:207E60004FF0000995B005460E4690464F46DFF85CA1DFF85CB152464146304606F0ECFA42
:207E8000421C044612D1B9F1000F0BD106F0F1FA03680133B34221DA2B69D8F80020434942
:207EA00028469847204615B0BDE8F08F6C2C06D0732C07D0522C08D147F00407DBE747F0B0
:207EC0000307D8E747F00107D5E72B695946D8F8002028464FF001099847CCE706F0C9FAB9
:207EE0000368B3420CDBFDF731FD01462846FDF73BFD064650B92B69D8F800202C49CFE734
:207F000006F0B7FA036858F82310EFE706F0C8F8F243304400211318002B03DD10F8013CFB
:207F20002F2B18D005A9304608F0C0FC002815DAD8F800202F690392F9F738FF006805F06F
:207F4000F1FF1C4B00902846039A1B49B8473046FDF72EFDA6E700F8011DDCE7079B03F438
:207F60007043B3F5804F07D03B46002231462846FFF74CFD0446EAE76B6932460F4928460C
:207F800098470F4B32460F4928460097FEF718F904460028DBD17B07D9D50B4B324609495F
:207FA00028460097FEF70CF9E4E700BF7F8D1608A68C1608C08B1608728C1608E7931608A1
:207FC0000D7A020855B71608817B0208F7931608138C16082DE9F34706460D46144600270B
:207FE000DFF8B48042462146284606F035FAB0F1FF3F82463ED106F03CFA0368AB4235DAAB
:2080000006F037FA0368304654F82310FDF7ACFC054658B31D484FF02F084FF00009002F95
:2080200018BF28462F2106F00BF8044608B180F8009040F2FF11284608F099F8B0F1000AC3
:208040001DDAF9F7B3FE0368112B00D1BFB93469F9F7ACFE006805F065FF0D4B00902A4648
:208060000C493046A0472846FDF7A2FC504602B0BDE8F087BAF1700F08BF0127B2E7002C0C
:20808000F1D0204600F8018BCCE700BF61C71B080D901608728C1608F89716082DE9F04F9F
:2080A000414F8DB004468846164604ADDFF81091DFF810A1DFF810B10FCF0FC597E80F00F6
:2080C000002785E80F004A463146404606F0C4F9431C05461BD1B7B906F0CBF908F1FF33D2
:2080E00002689A423ED106F0C4F90368204656F82310FDF739FC074600283DD12369326854
:208100002A492046984728460DB0BDE8F08F462D07D0722D1BD03A2D236920D13268244999
:2081200011E006F0A2F9006805F057FDC0B210F0EF0F8DF81100C6D00C28C4D02028C2D0CE
:20814000236951463268204601279847BBE706F08CF9006805F041FDADF82000B3E7326844
:208160005946F0E706F085F90368326843452369B4BF10490E49C4E704A901F059F9051E1B
:208180000EDA3268D4F810800392F9F70FFE006805F0C8FE084B00902046039A0749C0470F
:2081A0003846FDF705FCAEE70C941608A68C16084B8C16087F8D16081F901608728C1608A1
:2081C000FB9316082E8C1608138C16082DE9F04385B0516804461546FDF7C6FB074650B977
:2081E0004FF0FF3623692A68204618499847304605B0BDE8F083A9682046FDF7B5FB804623
:2082000050B94FF0FF3623692A6820460F4998473846FDF7CDFBEAE70146384608F020F945
:20822000061E0EDA2A68D4F810900392F9F7BEFD006805F077FE064B00902046039A0549F0
:20824000C8474046FDF7B4FBE2E700BFA68C160801941608728C16082DE9F0415568C4B0C7
:2082600006461B492846174605F0F4FE044600B9BD6829463046FDF777FB054628B30CBB3C
:2082800001464FF4807204A805F0EEFE04A8FFF743FB002804460EDA3A68D6F81080039206
:2082A000F9F784FD006805F03DFE0A4B00903046039A0949C0472846FDF77AFB204644B033
:2082C000BDE8F08108F070FBE3E74FF0FF34F5E708941608C58B1608728C16082DE9FF4173
:2082E000516806461746FDF73FFB0546C8B108F005FA041E0EDA3A68D6F810800392F9F7A4
:2083000055FD006805F00EFE074B00903046039A0649C0472846FDF74BFB204604B0BDE8F0
:20832000F0814FF0FF34F8E7FA901608728C1608D2E90012FDF74CBA2DE9F04F2DED028BF4
:2083400013788DB0044608EE101A042B40F0C881511C2932884611F8013B2BB1303B092BED
:2083600000F2BE818A42F6D1002318EE102AB2490BA80B93434604F0EAFA002803DB0B9A7E
:20838000002A40F09480AD4E2569F9F70FFDB14600683746B24605F0C5FDA94B0090204675
:2083A000A84AA949A84708960796CDE9056663694246A6492046984763695246A349204650
:2083C0009847059B65693A4603932046089BA0490293069B0193079B00934B46A8476369FD
:2083E00032469C49002520469847434618EE102A99490BA80B9504F0AAFAA84203DB0B9AB3
:20840000002A40F0E6802569F9F7D0FC006805F089FD8B4B009020468A4A8B49A8470025E7
:208420002E4684F82850636932468C492046984763692A468949204698473EB1002D00F017
:2084400034814FF47A704543B5FBF6F60A23B6F5487F656920462CBF21212021B6FBF3F23F
:20846000009103FB12637E49A8470025434618EE102A7C490BA80B9504F069FAA84203DB1D
:208480000B9A002A40F013812569F9F78FFC006805F048FD6A4B009020466A4A6A49A8479D
:2084A0004FF0FF300DB0BDEC028BBDE8F08F4FF4007104F1280B2046604E5B46009161496B
:2084C000B146FDF727FE05460B98374603F0FCFC002DB24608960796CDE90566FFF667AFAA
:2084E0000BF101010D4611F8012B0A2A00F0FF80002AF7D1154605225B49584605F047FD64
:2085000048B90BF10C00FDF7B1FE0790002D3FF44EAFAB46E4E706225449584605F037FD73
:2085200028B90BF10C00FDF7A1FE8246EEE706224F49584605F02BFD88B909900BF10C00C5
:20854000FDF794FE2C21089005F07AFD0028DDD0099A00F8012BFDF789FE0590D6E70622B3
:208560004449584605F013FD28B90BF10C00FDF77DFE0690CAE709223F49584605F007FDE2
:2085800070B90BF10C00FDF771FE07460246114601320B78303B092BF9D900230B70B5E7FA
:2085A0000A223649584605F0F2FC28B90BF11200FDF75CFE8146A9E708223149584605F0C4
:2085C000E6FC0028A2D10BF10C00FDF74FFE06469CE74FF4007104F1280920464B460091A4
:2085E0001849FDF797FD06460B9803F06DFC002E2E46FFF618AFDFF88CA0DFF88CB009F1D9
:2086000001010F4611F8012B0A2A6BD0002AF8D117460A225146484605F0B9FC0246A8BB69
:20862000014609F10C0005F016FB0646002F3FF4FAAEB946E3E700BF2C94160861C71B08E0
:20864000399416086CE91B08728C16084294160847941608649416086A9416087694160854
:208660007D9416088B9416082E951608EC94160827951608E5941608F3941608FD9416084A
:2086800008951608119516081C9516080A225946484605F07CFC02460028C7D1014609F17D
:2086A0000C0005F0D8FA0546C0E72E46CEE64FF4007304F128071049204600933B46FDF72C
:2086C00029FD06460B9803F0FFFB002EFFF6E8AE38466669FDF7CAFD084902462046B047E1
:2086E0000020DFE64FF0000307F8013B91E7002205F8012BFFE600BF6CE91B083CC41B0816
:2087000073B516460446002201A9706805F069FA054628B1019B72689A4201D01B7843B1C1
:20872000236920463268064998474FF0FF3002B070BD02466369034920469847A847F6E7C1
:20874000138C16089994160830B5044685B01D4943691D4A984763691C4A2046194998477C
:208760001B4B6569204603931A4B1B4A02931B4B1B4901931B4B00931B4BA84763691B4A8D
:2087800020461B49984763691A4920461A4A984763691A4A2046174998476369184A2046EF
:2087A000184998476369184A2046184998470023174A204600931749174BFDF701FD05B0BF
:2087C00030BD00BF42941608A5941608A9941608BA941608C13F1808B6941608C0941608E1
:2087E000479416089B131708AF941608C494160864941608CC9416089EB71B08C853170896
:20880000D1941608D8941608DD9416083CC41B08328B16086CE91B0839830208032970B52F
:20882000054686B0144618D1506803782D2B0ED14378303B092B0AD8002205A9013005F0D8
:20884000D0F90646A0680378303B092B0DD92B6928462268184998472AE00229F7D150687A
:208860000378303B092BF2D80C2605A9002205F0B8F931460EF041F8E0B1F9F797FA036841
:208880002E69032B0DD0162BE1D022680392F9F78DFA006805F046FB084B039A084900903F
:2088A00004E0A368226800930649074B2846B0474FF0FF3006B070BD138C1608E48F160807
:2088C000728C16082F8D1608B179170873B515460646002201A9686805F083F928B1019B08
:2088E0006A689A4201D01C7844B1336930462A68044998474FF0FF3002B070BD05F0BEFDA3
:208900002046F9E7138C160873B515460646002201A9686805F065F928B1019B6A689A4273
:2089200001D01C7844B1336930462A68044998474FF0FF3002B070BD05F0BCFD2046F9E7CC
:20894000138C16081346024A1968FDF749BB00BF34951608F0B589B004460120164604A944
:20896000FCF798FA002812DA326825690392F9F71DFA006805F0D6FA204B00902046039A6F
:208980001F49A8474FF0FF35284609B0F0BD71682046B4F82872FEF78BFD051E15DB06A975
:2089A0000120FCF777FA051E12DA326825690392F9F7FCF9006805F0B5FA104B0090204624
:2089C000039A0F49A8474FF0FF35A4F82872DBE7049B069A0598D21A079B66699842C1BFB5
:2089E000084902F1FF32C9180791079B06491B1A2046B3FBF1F30549B047E6E74295160864
:208A0000728C160800CA9A3BA0860100509516082DE9F0474FF00008A4B004468946164614
:208A20004746DFF82CA252463146484605F014FD431C054640F08F8005F01BFD03684B4570
:208A4000C0F2EC803668002F00F09C802C22002110A8F9F70AF903AA7149384605F0B3FA7E
:208A60008146002800F08580DFF8E8A10027032249465AF8040B05F06FFA20B101370C2FD4
:208A8000F5D14FF0FF371497013772D003AA6449002005F098FA00286BD00A22002105F0D0
:208AA000A0F8431E1E2B64D8139003AA5D49002005F089FA00285CD00A22002105F091F88B
:208AC000172856D8129003AA5649002005F07BFA00284ED00A22002105F083F83B2848D82B
:208AE000119003AA4F49002005F06DFA002840D00A22002105F075F83D283AD8109003AA69
:208B00004749002005F05FFA002832D00A22002105F067F8A0F26C70C8282AD8159010A8CF
:208B2000B8F1000F22D005F0EFFB0027059005A9384606970DF022FCB84265DA2769F9F753
:208B400035F9006805F0EEF9374B0090324637492046B84712E0732D03D105F086FC0768E8
:208B600061E7752D52D14FF001085CE705F0E1FBDBE7236932462E4920469847284624B0C8
:208B8000BDE8F08703A93846FCF784F9002808DA2769F9F70BF9006805F0C4F9254B009077
:208BA000D4E705A903A8B8F1000F0BD005F0C4FBA0B92769F9F7FAF8006805F0B3F91E4B1D
:208BC0000090C3E705F046FC40B92769F9F7EEF8006805F0A7F9194B0090B7E705AB184A24
:208BE000502110A805F082FA002808DA2769F9F7DDF8006805F096F9124B0090A6E763694A
:208C000010AA1149204698470025B7E708492369204632684FF0FF359847AFE70B49F6E742
:208C200047B61A086495160868951608728C1608138C160842951608769516087F951608BA
:208C40008B951608A19516083CC41B087F8D160860951608DC9516082DE9F0410F4686B0C1
:208C6000054603920293FAF709FA0C9B3846DDE9022100F07FFB041E33DB95F82832002BD1
:208C80003BD195F8886205934EB10DF005FD22464FF48C71D0F83C0107F00FFA064620465C
:208CA000042205A90DF0EBFD041E1FDAF9F77EF800680A281FD0D5F8108005F033F9174B11
:208CC0003A46009028461649C04795F8883243B13EB90DF0E1FC40F21911D0F83C0107F04C
:208CE000ECF9FAF7DBF944EAE47014E0059C003C18BF0124E9E70024E7E705A90DF026FDEB
:208D0000059B3A4607490093284623466E69B047FAF7C4F9002006B0BDE8F0810C96160851
:208D2000728C16089A8B1608012938B5044615680BDD0749506805F08DF930B9054A2946E4
:208D40002046BDE83840FDF74BB9034AF7E700BFEF8A1608149616082396160801292DE938
:208D6000F04F044685B08846164634DC514A316805B0BDE8F04FFDF733B96F2F23D0742F1A
:208D800009D03A2F236923D13268294620464FF00109984703E005F068FBD0F800A0464A47
:208DA0003146404605F058FB431C0746E5D1B9F1000F3CD105F05DFB0368434514DB23698B
:208DC00032683E4931E005F050FB03680393E6E732685946DAE74FF00009DFF8F0B0374D16
:208DE000CA46CDF80C90DAE705F043FB036856F8235005F03EFB03680133036005F039FB89
:208E0000036843454FDA05F034FB036856F823B005F02FFB03680133036005F02AFB0368E0
:208E2000434508DA23693268254920469847384605B0BDE8F08FBAF1000FC0D035B12946F9
:208E40002046FCF791FD05460028F0D059462046FCF78AFD8046D0B1039B01465246284647
:208E60000093002308F09EF8071E0EDA3268D4F810900392F8F79AFF006805F053F8114B7A
:208E800000902046039A1049C84715B907E0002DCDD02846FCF78CFDB8F1000FC7D0404699
:208EA000FCF786FDC3E7BAF1000F88D0AB464D46CCE700BF33961608429616084B8C1608B8
:208EC0007F8D16083C961608728C1608138C16082DE9FF41516806461746FCF745FD054667
:208EE000D0B1002108F0CDF8041E0EDA3A68D6F810800392F8F75AFF006805F013F8084B71
:208F000000903046039A0749C0472846FCF750FD204604B0BDE8F0814FF0FF34F8E700BF69
:208F20004F911608728C16082DE9F04F044685B08B4616460125DFF8C080DFF8C090DFF8DB
:208F4000C0A05D4503DB002005B0BDE8F08F56F8252013785C2B44D153786E3B0A2B21D8DC
:208F6000DFE803F03420202039203C2020200600971C00211022384604F06DFE0A21039007
:208F8000384605F0A6F80628039A0DDD130E6769154920460193C2F307430093C2F3072351
:208FA000D2B2B8470135CCE7022807DDC2F307236769D2B20D492046B847F3E70028F1DD79
:208FC0006369D2B20A4920469847EBE76369094920469847E6E763695146F9E76369494609
:208FE000F6E763694146EEE7489616084C96160813C21B08A2A51A08EA131708345418084B
:20900000519616082DE9F04F074693B00E461546DFF8F892DFF8F8A22C68A849204605F005
:2090200019F878B9012E40F375812A1D711E3846FFF7E8FFB0FA80F040094442204613B053
:20904000BDE8F08F23782D2B40F0A780012E40F361819B49204604F0FDFFD5F804B030B9BA
:209060009BF80040B4FA84F46409644212E09549204604F0EFFF28B99BF80040003C18BF05
:209080000124F2E759463846FCF76EFC0446F8B94FF0FF344FF00208012C00F03B81B045D4
:2090A000CCDA55F828204FEA880B87491046019204F0D0FF019A002840F0F780002C40F067
:2090C0002E8108F101030BF1040BF61A5D44A3E703A907F0EBFB83462046FCF769FCBBF1E2
:2090E000000FD5D1D5F800B07849584604F0B2FF40B9059C04F47044B4F5C04418BF4FF031
:20910000FF34C7E77249584604F0A4FF28B9059C04F47044B4F50054F0E76E49584604F033
:2091200099FF28B9059C04F47044B4F58044E5E76949584604F08EFF04460028AAD06749C3
:20914000584604F087FF28B9059C04F47044B4F50044D3E76249584604F07CFF38B9059BD9
:2091600013F4927F0CBF4FF0FF34002492E75D49584604F06FFF28B9099C002CCCBF0024F6
:20918000012472E75849584604F064FF18B9059B13F0920FE6E701247CE7022E40F3BA80B4
:2091A000D5F804B04946584604F054FF20B15146584604F04FFF50B9A968204604F04AFFB5
:2091C000003818BF012044424FF0030864E74749584604F03FFF38B9A968204604F03AFF4F
:2091E000B0FA80F04009EEE7002203A9204604F0F8FC2B6883461B780BB90124E4E7039BDA
:209200001A78002AF9D103A9A86804F0EAFCAB6804461B78002BF0D0039B1B78002BECD13E
:20922000D5F804803249404604F014FF28B9BBEB040418BF4FF0FF34C6E72E49404604F05F
:2092400009FF28B9A3454FF0FF34A8BF0024BBE72949404604F0FEFE28B9A3454FF0FF347B
:20926000C8BF0024B0E72549404604F0F3FE28B9A3454FF0FF34D8BF0024A5E72049404662
:2092800004F0E8FE28B9A3454FF0FF34B8BF00249AE71C49404604F0DDFE0028ADD1A34555
:2092A0004FF0FF3418BF00248EE71749104604F0D1FE78BB002C7FF404AFBFE61DFF1A08EB
:2092C000539616085696160886961608599616081A8B1608078C16085C9616085F9616089F
:2092E0000894160862961608659616086B9616086E96160872961608769616087A961608C6
:209300007E96160882961608899616086C961608689616083B693846024A034998474FF094
:20932000FF348BE664031708688D160804320139FFF768BE01F18043013B70B504460E46B0
:2093400052F823001546094904F084FE30B92A1DB11E2046BDE87040FFF754BE23692046C9
:209360002A68034998474FF0FF3070BDD4581808688D16082DE9F04188B00E461746984628
:2093800003F048F8002806DA0224F8F70FFD04604FF0FF3448E003F04FF805460028F3D003
:2093A00004A803F096FA04460028EED102A803F08CFA04460028E8D16B6803A904A803933E
:2093C00003F0A7FA044630BBA96804A803F0A5FA044600BB042104A803F098FA0446D0B947
:2093E0006FB92868E968D6B9002302AACDE9006304AB0DF029FB041E13DA64420BE04FF43A
:20940000D2733A46012102A80093434603F02EFA04460028E5D002A803F04CFAB5E70436A4
:20942000E2E702A803F046FA204608B0BDE8F08130B599B004460D462822002103A8F8F782
:2094400014FC01A90020FBF725FD00B30023069303216B7820468DF8153006F0BAFF0028A1
:20946000039038DAF8F7A2FC046864420A9820B107992EF11FFA00230A93002C76DA64427B
:20948000F8F794FC04604FF0FF3019B030BD0DA901A804F051FF0028D8D012994F29D5DD7D
:2094A0000E9A503953010F9A03F4FC6343EAC2230D9AC2F344021343109A02F01F029BB214
:2094C00042EA412211990131490101F4F0710A4343EA0243BBE70DAA40F20C5106F0EDFDFA
:2094E000041E04DB9DF834302BB96FF01204039806F009FDBAE79DF83630002BF5D0EA69A3
:209500000E9B22B1934203D26FF01504EFE7EB61BDF93C30B3F5006F079325D008DCB3F537
:20952000007F0AD0B3F5806F1CD04FF0FF34DEE7B3F5805FF9D10C2300E0092303A9284672
:209540008DF8133000F014F8041ED0DB07982EF1AFF90A900028CAD003A9284600F0B8FAFC
:209560000446C4E70A23E9E70B23E7E700208CE72DE9F04F038A95B004460D4613B94FF497
:20958000007303823022002108A8F8F76EFB638A002B00F0EC80012B0B930F9300D1022382
:2095A00013936B7A202B0ED02A69218A531EEA7903EB41130B99D3402B72DBB2E269521A0B
:2095C000D31A0C93089394F80290B9F1FF0F08D1E369B3F5006F80F0CF8000234FF0070921
:2095E000A370089B4FF00008059303EB4303C34606930C9B039302330793139BCDE9018807
:20960000049395F809A0BAF1000F03D0BAF10C0F40F0C980A77826787B1C296906EB460292
:20962000B81C99400A44012101FA03F301FA00F000211844069B1844531E41F1FF31C0180C
:209640004FF0000341F100010EF0E0F90190002800F0A780059B42F6D27200FB1636EB7927
:209660000133FE4000FA03F3934296BF03224FF47F63B3FBF2F3B21C9A4201D90026019640
:2096800001230293BAF1000F03D0BAF1100F40F0168194F802B02A692778BBF1000F40F098
:2096A000848007EB5202079810184FF0000343F10001013861F100010EF0A8F9002800F0DF
:2096C000FC80039B4FF6F07207FB1037EB79013B27FA0BF700FA03F3934228BF1346BA1CE2
:2096E000934203D3B7F57F6F00F2DF804FF00108002E40F08280C346BAF1200FA67840F0FB
:20970000AE800122E069049B02FA06F794F800A0C31A2A69DF1B002E40F092800AEB920288
:20972000F81C10184FF0000343F10001013861F100010EF06BF998B1EB790AFB1077624AA3
:20974000023BF74000FA03F3934228BF1346FA1C9342C0F084804FF6F3739F427FD9129764
:2097600020236B72129BC5E90503049B53E001230B930F93202313E7B3F5805F01D2012375
:209780002CE7B3F5005F01D2022327E7B3F5804F01D2032322E7B3F5004F34BF04230523F7
:2097A0001CE7019E6CE700266FE70BF1FF330BF101009A40012303FA00F0039B3A441844AA
:2097C00072E74FF00108C346029B0BB1019B0993BBF1000F00D00D90B8F1000F00D00E97F9
:2097E000BAF1000F0DD10E9BB3420DD80C23AE616B72099B6B610B9B0DE00020C3460746BA
:20980000E2E7BAF1100FF1D110236B720E9BAB610D9B6B610F9B6382EB232B719023AB71B2
:209820002A4B6B6281236B816B7A202B22D03C236B715B2385F820306B7A0020637016E0E0
:20984000012E03D10AEB5202B81D6AE7B11E701C8A40012101FA00F05244184461E70136F3
:20986000F6B24E45A6707FF6CCAE6FF0160015B0BDE8F08F58236B71772385F82030012368
:20988000A278934000222B72E189638A0129228201D98B42D0D8012BE281CDD9013B9BB2EA
:2098A000062B88BF0623E381C6E7002E89D1029B0BB1019B09930D9091E74FF0010B002E4F
:2098C0003FF41AAF00209AE7F0FFFF0F8C96160838B50C4605460A690021E069F8F7C5F99A
:2098E000E369A28860491A80A2799A70E0690330F8F702FAE3692269DA722369E2691B0A04
:2099000013730123A978E2698B405373E3696A8ADA81E3692A781A74E3692A8A5A742B8A06
:20992000E2691B0A9374EB69E269B3F5803F3FBFD374AB8BE2691B0A2CBF13621375F822BD
:20994000E3695A753F22E3691A83FF22E3695A83E3696A69DA61EB1C6A786169202AE269B6
:2099600040D0D1822921E26982F82610E269A96982F82710AA69E169120A81F82820E269AC
:20998000698B82F82910E269E97E82F82A10E269D5F80310C2F82B105968C2F82F1019893E
:2099A000A2F833109B7A82F835306B780C2BE3690CBF2E492E490A68C3F836204A68C3F8C7
:2099C0003A20E06962893E30616AF7F7E1FFE36994F8202083F84120E3694AF65522A3F860
:2099E000FE2138BD51620221E269D1620121E2691186E269E98951862921E26982F8421006
:209A0000E269A96982F84310AA69E169120A81F84420E269698B82F84510E269E97E82F88C
:209A20004610E269D5F80310C2F847105968C2F84B101989A2F84F100E499B7A82F85130BC
:209A4000E2690B68C2F852304B68C2F85630E0696289616A5A30F7F79BFFE36994F82020F0
:209A600083F85D20B8E700BF0D971608169716081F97160828971608002A38B50C4621DBED
:209A8000C36993421ED9CD79206802FA05F50022294606F05FFB431C04D1F8F787F900681E
:209AA000404238BD854210D12269E169206806F0B1FF0028F1DB236983420CBF00206FF0F5
:209AC0003C00EEE76FF01C00EBE76FF01500E8E72DE9F84F0C4606460127FFF7F9FE0022B3
:209AE00021463046FFF7C8FF226905460021E069F8F7BBF8738A9F420CDA002D02DA2846AF
:209B0000BDE8F88F3A46214630460137FFF7B4FF0546EFE7002DF2DB7378202B13D0B6F8F9
:209B200012A04FF000084FF0F80B3378984575DB62694FF00008B6F81290F71CDFF85CA1C9
:209B400002FB03999EE0F38923BB22690021E069F8F78BF8E3694F4A214630461A6002F1FE
:209B6000FF52E36902F500522032C3F8E421D4E90632013BC2F8E8310222E369C3F8EC21B1
:209B8000454AE369C3F8FC210122FFF775FF051EB5DBC4E721463046FFF79AFEF2892146DA
:209BA0003046FFF769FF051EA9DBCEE722690021E069F8F75AF8EFB922693946E069F8F755
:209BC00054F87278E3690C2A0DD0102A4FF0FF3222D01A605A60E36983F808B0E369A3F8BA
:209BE0000990DA7203E0A3F8009083F80290E36983F800B02A4621463046FFF73DFF051E4C
:209C0000FFF67DAF013763690AEB0705BB42CDD808F10108AA4688E71A60E8E700276FF04C
:209C20007F49F0E722690021E069F8F71EF8B8F1000F1DD10B225146384604F0EAF940B1DB
:209C40003A68E3691A607A685A603A891A81BA7A9A72E3690822DA72E369E268DA81E36963
:209C6000E268DA82E369E2891A82E369E2891A832A4621463046FFF7FFFE051EFFF63FAF51
:209C800008F10108237A08EB09059845CADB002535E700BF52526141000055AA3197160877
:209CA000044B1B680360C3F1105303F500230B60704700BFE884160808B54FF490214FF0E2
:209CC000405002F0F9F80748C0F1605101F5803102F0F2F84FF400314FF00050BDE80840ED
:209CE00002F0EAB80000003808B50CF0D9FD002008BDFFEC10B5084B4FF0E024002207496C
:209D000063610F20A261F9F7CDF807230F202361BDE81040F7F79EBCFF520700E99C020897
:209D20000023092802DC40EA0310704701330A38F7E7FFEC08B50120F7F7ACF8024BCA2215
:209D40005A6253225A6208BD0040005813B5FFF7F1FF0E4BDA6822F02002DA60002201924D
:209D6000019AB2F5003F09D36FF07304FF2200205A62F7F78FF8204602B010BDDA6892067F
:209D800002D4019A0132EAE70024EFE7004000580C4A82B0D36813F0400302D0002002B00F
:209DA00070478021D1600193019BB3F5803F02D36FF07300F3E7D3685B06EFD4019B0133D3
:209DC000F1E700BF004000583D4B01202DE9F0413C4E5F6DF7F75EF8B7424AD03A4B9F4251
:209DE00047D04FF4803200213848F7F7DDF800224FF480313548F7F7D7F84FF44072334833
:209E00001146F7F7D1F84FF4004200212F48F7F7CBF80025FFF79AFF044610B101350A2D3A
:209E2000F8D1B7421AD0284B9F4217D0FFF782FFFFF7AEFF044650B9214B9A6822F040020C
:209E40009A60234A1A61DA6822F08002DA601C4FFF2300207B62F7F71DF87E650020F7F792
:209E600019F804B145BB1B4B012200201A70BDE8F081194BD3F8703403F44073B3F5407FEF
:209E8000C7D00F4C4FF4803200211048D4F800806568F7F789F800224FF480310B48F7F783
:209EA00083F84FF4407209481146F7F77DF8C4F8008065606665A6E76FF07300D7E700BF7F
:209EC00000400058EDFECEFACEFA0DF0704402583F1F7C0065540024004002582DE9F843C2
:209EE00006460D46314F7B683A68BC6A39688A42F9D179688B42F6D10A20C2F3021C02F0FD
:209F00000F0103F00F09C3F3032800FB0C11C2F3023C3160C2F3032100FB0C117160C2F332
:209F20000151C2F3034200FB0122C3F30351B260C3F3011200FB0299C3F3003200FB0288CF
:209F4000C3F30342C3F34233C6F80C9000FB012008F1FF3800F16402C6F8108000F5FA6041
:209F600072610722B3FBF2F2C2EBC2029B1AB36104F0B4F9011E404618BF012104F0A2F94B
:209F8000002348443362F0613A6965B1C2F30E02A3B2074CD31A01326343B3FBF2F342F279
:209FA000107253432B600020BDE8F88300400058A0860100FFF792BF2DE9F84F8269076900
:209FC000D0E9009AD0E902B6002A4FD0520395B2D0F81480FFF7AEFEFFF7DAFE044688BB7F
:209FE0005846FFF79DFE014650460904FFF798FE41EA00214846FFF793FE08431D4900F0BA
:20A000007F3020F0FE400860A8F16400FFF788FE8046781CFFF784FE04463046FFF780FE5C
:20A0200040EA050242EA084343EA042020F07F4020F0C0004860CB6823F08003CB60FFF7F6
:20A0400085FE04460B4D0C4E6B6DB34206D00120F6F720FF00206E65F6F71CFFFF23002074
:20A060006B62F6F717FF2046BDE8F88F4FF46045AEE700BF00400058CEFA0DF000B58DB0F3
:20A0800001A904F059F901A8FFF796FF0DB05DF804FBFFECF0B504460D46124E89B024F0B1
:20A0A0001F0425F01F05104F04F090FEA54201D809B0F0BDE3693246394600200793A36934
:20A0C00006936369059323690493E3680393A368029363680193236800932346F7F724FEE9
:20A0E0002034E3E7F79916083D9716082DE9F8430D4614461E4602EB03081B4903461B4A36
:20A10000074600209DF82090F7F70EFE2B46174A00201749F7F708FE2346144A0020154908
:20A12000F7F702FE3346114A00201349F7F7FCFDAC4207D8A84505D941462846BDE8F8438D
:20A14000FFF7A8BF3B46094A0C490020F7F7ECFDB9F1000F06D03146204600F007FB41469D
:20A16000081AEBE7BDE8F88379971608059A1608889716089B971608AE971608C19716087A
:20A180002DE9F0439BB0044600213C220BA80A91F7F76BFD204600F01FFBE56C35B10028EF
:20A1A00035D04FF47A735843B0FBF5F5A38E0AAF03F00303012B2CD1D4F8AC3040211F4ABC
:20A1C000384602F0D1FBE3682046267C8C3454F8408C099300F000FB0A22B5F5487F099B50
:20A1E00007970096B5FBF2F102FB11522CBF21252025CDE90312CDE90180114A00201149EB
:20A20000CDE90554F7F790FD1BB0BDE8F0830546CCE7A3680026DFF830909B6AD3F80880B3
